:020000040800F2
:10000000F8FF012009470A08A5470A0835710508C5
:10001000A5470A08A5470A08A5470A0800000000E6
:10002000000000000000000000000000A5470A08D2
:10003000A5470A0800000000A5470A082D68040823
:10004000A5470A08A5470A08A5470A08A5470A08B8
:10005000A5470A08A5470A086D3304089533040824
:10006000BD330408E53304080D340408BD03000063
:10007000D1030000E5030000F90300000D040000B7
:100080002104000035040000A5470A08A5470A0816
:10009000A5470A08A5470A08A5470A0835340408F1
:1000A000A5470A08554A0408A5470A08454A04080E
:1000B000654A0408754A0408854A0408352104087D
:1000C00029210408692104085D210408A5470A08BC
:1000D000A5470A08613D0000B13E00001D40000038
:1000E00075340408A5470A0800000000414B0408C5
:1000F000194B0408514B0408094B0408490400003B
:10010000A5470A08A5470A08954A0408A5470A080A
:100110008D410000FD420000A54A0408BD80090889
:100120005D040000710400008504000099040000D3
:10013000AD040000A5470A08A5470A08A5470A0814
:1001400000000000000000000000000000000000AF
:10015000C1040000D5040000E90400006D44000063
:100160009D21040891210408A5470A08A5470A080B
:10017000A5470A08A5470A08A5470A080000000085
:10018000A5470A08A5470A08DD4500004D470000BD
:10019000A5470A08A5470A08A5470A08A5470A0867
:1001A000A5470A08A5470A08A5470A08A5470A0857
:1001B000A5470A08A5470A08A5470A08D121040847
:1001C000C5210408A5470A08A5470A08A5470A0843
:1001D000A5470A08FD760908A5470A08A5470A08A1
:1001E000A5470A08A5470A08A5470A08A5470A0817
:1001F000A5470A08A5470A08A5470A08A5470A0807
:10020000A5470A08A5470A08A5470A08A5470A08F6
:10021000614B0408714B0408814B0408A5470A0888
:10022000A5470A08A5470A08A5470A0800000000D4
:10023000A5470A08A5470A0800000000A5470A08C4
:10024000A5470A08A5470A08A5470A08A5470A08B6
:10025000A5470A08A5470A08A5470A08A5470A08A6
:10026000A5470A08A5470A08A5470A08A5470A0896
:10027000A5470A08A5470A08BD480000000000007D
:10028000A5470A0800000000A5470A080000000072
:0802900000000000A5470A0868
:020000040804EE
:10000000114A037A0168D35C10B4CC58CA1824F0A2
:100010000104CC501368DB07FCD4037D1F2B09D9E6
:10002000203B20225DF8044B02FA03F343F018034F
:10003000CB60704720225DF8044B02FA03F343F0D3
:1000400018038B60704700BFC8090B084368426DF6
:1000500030B49A61EFF31182502383F31288416820
:10006000D2B2856C0B68046D23EA050323430B6051
:1000700082F31188436981681A68096822F00102D5
:10008000D0E908541A60826A1D605C615A60D0E948
:100090000B429C60DA600023B0F86C2030BCCA626E
:1000A00003777047002A4FEA014C034630B508BF7A
:1000B000E64600F1C00514BF8E468C460024196840
:1000C0000C3353F8042C43F8084C41EA0C0142EA83
:1000D0000E02AB4243F80C1C43F8042CEFD1D0F8CD
:1000E000C03043EA0E03C0E93144C0F8C03030BD2F
:1000F00010B40C4C6368002B11DD002004F1080CD7
:100100000146DCF8AC3003F1C00259600C33934275
:10011000FBD1013063680CF5867C8342F1DC5DF82D
:10012000044B704704000020F0B5404C04EB401332
:1001300093F8543403B9F0BD3D4B42011D7893F858
:1001400001C065450CD00CEB4C0E03EBCE0E9EF8B7
:1001500004604FEA4C0E771E012F5AD9032E52D05D
:100160002244A2F83814EFF31181902383F312880C
:1001700092F83A34C9B2B2F8380443EA4003002096
:100180009BB282F83A0481F311881909207881EA38
:1001900013215940D8B1C9431B01D2F8505401244E
:1001A000D2F83C049BB201F00F01D5F8AC2084409A
:1001B0000B4302F1C000590013F4004F8BB202D17F
:1001C0005168214351600C329042F4D1F0BDD2F815
:1001D0003C041B01D2F8502401F00F0110309BB2F7
:1001E0000124D2F8AC200B43844002F1C000590036
:1001F00013F4004F8BB202D15168214351600C328D
:100200009042F4D1F0BD0CF1010606F00306AE42B7
:10021000A6D0E64403EBCE030344597C00299FD0CB
:10022000A318012083F83A049AE700BF04000020D5
:10023000D81C0024704700BF024B03EB401393F817
:100240005504704704000020D0E90920131A5842D1
:100250005841704790F8573830B53BB990F8551869
:10026000012490F85638DAB2914200D830BD04FA31
:1002700003F2B0F85E5801332A43A0F85E28F2E793
:100280000379024613F0010006D0D2E90731D268A3
:100290005B1A013A03EA0200704710B5037904467D
:1002A00013F001030ED0FFF7EBFF034650B1226AB3
:1002B0006369E1689B5C0132B2FBF1F0DBB201FBE8
:1002C00010222262184610BD03799B070AD5436AA3
:1002D0008269D154436A02690133B3FBF2F102FB34
:1002E00011334362704770470171704703790146CB
:1002F00013F0020007D00B69D1E90921013B521A22
:100300001A40D2B2981A70470C4B4FF0E02C10B440
:100310005A6EDCF81800596E8A42F9D1996E8842FB
:10032000F6D8DC6E4FF47A7101FB04F31B1AB3FBB1
:10033000F4F35DF8044B01FB02307047D81C002435
:100340002DE9F04F4C484FF0010A4C494FF002099B
:100350004B4B4FF0040808271026202540244FF06F
:10036000800EDFF820C130F8022F12F0010F03D009
:100370001960083323F804AC12F0020F03D019609F
:10038000083323F8049C12F0040F03D019600833DB
:1003900023F8048C12F0080F03D01960083323F8F7
:1003A000047C12F0100F03D01960083323F8046C9A
:1003B00012F0200F03D01960083323F8045C12F008
:1003C000400F03D01960083323F8044C12F0800F5B
:1003D00003D01960083323F804EC12F4807F05D0B1
:1003E0004FF4807B1960083323F804BC12F4007FBB
:1003F00005D04FF4007B1960083323F804BC12F4D5
:10040000806F05D04FF4806B1960083323F804BC6B
:1004100012F4006F05D04FF4006B1960083323F815
:1004200004BC12F4805F05D04FF4805B1960083380
:1004300023F804BC12F4005F05D04FF4005B196090
:10044000083323F804BC12F4804F05D04FF4804BDE
:100450001960083323F804BCD20B05D04FF40042D6
:100460001960083323F8042C01F5806161457FF49D
:100470007AAFBDE8F08F00BFEE740A0800000258A2
:10048000481D00240024025810B584464FEA810E0E
:10049000102312F4004F4FEA420214BF0E24072427
:1004A000013B92B2CCF80040F444F2D100EB81124F
:1004B0008C010351122042F8213010BD10B5844642
:1004C0004FEA810E0424130B013C4FEA021203EBA6
:1004D000430392B203F11803CCF80030F444F2D194
:1004E00000EB01130A018450062043F8214010BD9F
:1004F000704700BF704700BF00EB4000024B03EBAA
:10050000C00393F84905704704000020064B93F898
:10051000F825824206D900EB400003EBC003D3F874
:100520004C05704700207047040000201D4B93F8D5
:10053000FC25AAB3D3F8381509B100200860012AB8
:100540002ED0D3F8501509B100200860022A27D018
:10055000D3F8681509B100200860032A20D0D3F829
:10056000801509B100200860042A19D0D3F8981525
:1005700009B100200860052A12D0D3F8B01509B1DE
:1005800000200860062A0BD0D3F8C81509B1002056
:100590000860072A04D0D3F8E0350BB100221A60B6
:1005A000704700BF040000201D4B93F8FC25AAB340
:1005B000D3F8381509B100200860012A2ED0D3F8ED
:1005C000501509B100200860022A27D0D3F8681519
:1005D00009B100200860032A20D0D3F8801509B1A2
:1005E00000200860042A19D0D3F8981509B100201A
:1005F0000860052A12D0D3F8B01509B100200860B0
:10060000062A0BD0D3F8C81509B100200860072AC4
:1006100004D0D3F8E0350BB100221A60704700BF58
:1006200004000020C44B1B78002B40F04F81C34BCB
:1006300093F8FC25002A00F0498193F8481530B55D
:1006400000294ED1D3F838150020012A086047D977
:1006500093F86015002966D1D3F850150020022ABE
:1006600008603DD993F87815002940F0CB80D3F885
:1006700068150020032A086032D993F890150029E4
:1006800040F0E280D3F880150020042A086027D9C2
:1006900093F8A815002940F0F880D3F898150020A9
:1006A000052A08601CD993F8C015002940F00F8175
:1006B000D3F8B0150020062A086011D993F8D81590
:1006C000002959D1D3F8C8150020072A086007D996
:1006D00093F8F025002A73D1D3F8E03500221A6090
:1006E00030BDD3F83C25910AA1F58011522940F282
:1006F0000F814FF0FE0CEFF31181502080F3128830
:100700008F4C4FF02C0E556AC9B250690EFB0C4C41
:10071000013540F00100CCF81855506181F3118883
:1007200093F8FC258EE7D3F85425910AA1F58011A2
:10073000522940F2F2804FF0FE0CEFF3118150206D
:1007400080F312884FF02C0E556A7D4CC9B2506967
:1007500001350EFB0C4440F00100C4F818555061FF
:1007600081F3118893F8FC250020D3F85015022A54
:1007700008603FF677AFB3E7D3F8CC25910AA1F52F
:100780008011522900F2EA806E48014491F814C0A9
:10079000EFF31181502080F312884FF02C0E556A30
:1007A000674CC9B2506901350EFB0C4440F00100A2
:1007B000C4F81855506181F3118893F8FC2581E73E
:1007C000D3F8E425910AA1F58011522900F2C980DD
:1007D0005C48014491F814C0EFF31181502080F37C
:1007E00012884FF02C0E556A554CC9B2506901352C
:1007F0000EFB0C4440F00100C4F81855506181F321
:10080000118869E7D3F86C25910AA1F58011522966
:1008100040F288804FF0FE0EEFF31181502080F3FC
:1008200012884FF02C0C556A454CC9B250690135FD
:100830000CFB0E4440F00100C4F81855506181F3E0
:10084000118893F8FC2512E7D3F88425910AA1F5C5
:10085000801152296BD94FF0FE0CEFF3118150201B
:1008600080F312884FF02C0E556A354CC9B250698E
:1008700001350EFB0C4440F00100C4F818555061DE
:1008800081F3118893F8FC25FCE6D3F89C25910AA6
:10089000A1F58011522957D94FF0FE0CEFF31181C9
:1008A000502080F312884FF02C0E556A244CC9B2A8
:1008B000506901350EFB0C4440F00100C4F8185596
:1008C000506181F3118893F8FC25E6E67047D3F870
:1008D000B425910AA1F5801152293AD94FF0FE0CA6
:1008E000EFF31181502080F312884FF02C0E556ADF
:1008F000134CC9B2506901350EFB0C4440F00100A5
:10090000C4F81855506181F3118893F8FC25CFE69F
:100910000C48014491F814C0EDE60A48014491F8EE
:1009200014C00AE70748014491F814E074E7054849
:10093000014491F814C090E7000000240400002056
:10094000D81C0024F0740A080748014491F814C028
:10095000A4E70548014491F814C0C1E74FF0FE0C2C
:1009600016E74FF0FE0C37E7F0740A0800EE100AA5
:10097000B8EE400A704700BFBCEEC00A10EE103A55
:1009800098B2704707280AD84FF4B472054B02FB9F
:100990000033B3F80006B0FA80F040097047002039
:1009A000704700BF04000020072807D8044B4FF40D
:1009B000B471012201FB003383F80226704700BFA7
:1009C00004000020072808D8044B03EB401393F8D9
:1009D000542412B1012283F83A2470470400002005
:1009E000072808D8054B03EB4013B3F83804B0FAD6
:1009F00080F0400970470020704700BF04000020CD
:100A0000054B93F8F825824204D903EB4013D3F841
:100A1000440470470020704704000020436A0246E7
:100A20001B681B6A5B689B7813F0010008BF507756
:100A3000704700BFC2628161704700BF0346012258
:100A400000205A77704700BF826908B50346006BE3
:100A5000D96A02449A6101B18847002008BD00BFED
:100A6000704700BF043070470C4B93F88827D3F8C9
:100A7000841702440144D2B2C3F8841783F888274C
:100A800093F88827120605D593F8882782F080020C
:100A900083F88827024B01225A707047D81C002423
:100AA000000000242DE9F84F164FD7F88C57ED0AB7
:100AB00023D00026DFF850A007F5F269B04674197C
:100AC000D7F890174FF01003524648BF0134D1F8C1
:100AD00028B04846C7F8BC876410E102D8470F2801
:100AE0000BDD094B03F1100153F8042B013207D140
:100AF0008B42F9D12546B542E1DCE802BDE8F88F2A
:100B0000661CF8E7D81C0024A0F20024184B596E8C
:100B1000D3F8C4278A1A322A04D8D3F8D8278A42AD
:100B200011D37047D3F8C81749B193F8D4278888F0
:100B300002F001020968120100FA02F28A61002241
:100B4000C3F8D8277047D3F8C8276AB11068323184
:100B5000928810B44469C3F8D81722425DF8044B58
:100B600018BF1204826170473231C3F8D81770473A
:100B7000D81C0024074AD2F8C8374BB192F8D427C2
:100B80009988186802F001031B0101FA03F38361DD
:100B900000207047D81C0024044B4FF4007C002038
:100BA000D3F8E837A2F800C00B607047D81C0024C7
:100BB00000207047012070470120704700207047D7
:100BC00010B41C6994420CD394460A4661448C428A
:100BD000996938BFA4EB0C0261445DF8044B66F0E0
:100BE000B3B85DF8044B70472DE9F0414FF425721E
:100BF0008EB00021744866F005F9744B744D4FF0C7
:100C00000008D3F8F02040F27D27A5F1680605F62C
:100C1000F41442F00102C3F8F020D3F8F02002F0FF
:100C200001020092009AD3F8E82042F00102C3F8D2
:100C3000E820D3F8E82002F001020192019AD3F8EB
:100C4000E82042F00202C3F8E820D3F8E82002F0DE
:100C500002020292029AD3F8E82042F00402C3F89A
:100C6000E820D3F8E82002F004020392039AD3F8B4
:100C7000E82042F00802C3F8E820D3F8E82002F0A8
:100C800008020492049AD3F8E82042F01002C3F854
:100C9000E820D3F8E82002F010020592059AD3F874
:100CA000E82042F02002C3F8E820D3F8E82002F060
:100CB00020020692069AD3F8F02042F00202C3F80E
:100CC000F020D3F8F02002F002020792079AD3F83E
:100CD000E82042F04002C3F8E820D3F8E82002F010
:100CE00040020892089AD3F8E82042F08002C3F844
:100CF000E820D3F8E82002F080020992099AD3F89C
:100D0000E82042F48072C3F8E820D3F8E82002F427
:100D100080720A920A9AD3F8F02042F48032C3F823
:100D2000F020D3F8F02002F480320B920B9AD3F823
:100D3000F02042F40032C3F8F020D3F8F02002F49F
:100D400000320C920C9AD3F8F02042F48022C3F8BF
:100D5000F020D3F8F03003F480230D930D9B55F869
:100D60002810002302E00133112B29D054F833203E
:100D70009142F8D106EBC303B3F8600A08F1070803
:100D80005CF078FAB845EAD14FF0000840F27D27D0
:100D900055F82810002302E00133112B12D054F82B
:100DA00033209142F8D106EBC303B3F8600A08F18F
:100DB00007085CF05FFAB845EAD10EB0BDE8F081F3
:100DC0000020DBE70020F2E7C8210024004402589D
:100DD00058750A0810B5044664F07EFF01462046A7
:100DE00089B2BDE81040FFF79FB900BF38B50B4D81
:100DF00000EB400005F5A763C40003EBC0032544E6
:100E000093ED027AD3ED037AE7EE007AB0EE670A4B
:100E100064F062FFD5F83835186038BD0400002052
:100E200002692DE9F843C36812EA030828D0054691
:100E30000E464FF00047B8FA88F327FA03F21B3B3F
:100E4000D24308EA02082A61042B16D8DFE803F02F
:100E50003B30251A0300B36A002B3FD003F1FF3962
:100E600000231FFA89F9B362746A34B123682046FB
:100E7000494698476468002CF8D1B8F1000FDAD1E0
:100E8000BDE8F88370680028F7D0696B036889B201
:100E90009847B8F1000FCED1F2E7B0680028ECD047
:100EA000A96B036889B29847B8F1000FC3D1E7E78F
:100EB000F0680028E1D0E96B036889B29847B8F17F
:100EC000000FB8D1DCE730690028D6D0296C036860
:100ED00089B29847B8F1000FADD1D1E7EB6A1FFA9C
:100EE00083F9C1E72DE9F043134C83B0DFF84C9050
:100EF000DFF84C8004F5906602E00834B44218D064
:100F0000A579002DF9D12768083407EB08039B0A5F
:100F100009EB4303B3F8E40A5CF0ACF934F8041CC1
:100F200001232A463846CDE9005560F097FEB442C9
:100F3000E6D103B0BDE8F083481D0024F0740A0830
:100F40000000FEA78069B43054F032BAF8B5A0F5BD
:100F500007642379DB0725D5657994F8543805F0C3
:100F600001073D46FBB1D4F848341A68D36A5B08E0
:100F7000536294F8583823B1B4F862380133A4F8B6
:100F8000623885F00101606C5BF0F4F8012384F8AD
:100F90005738002384F8553884F85638A4F85E385A
:100FA00084F85438F8BD94F85768012E03D194F8AA
:100FB000553884F856382046FFF74CF94EB90123CE
:100FC00085EA030184F85738606CBDE8F8405BF0AF
:100FD000D1B80023394684F85738F5E738B5A0F57D
:100FE00007640022344D606C03685A62A1F1290342
:100FF000302B31D895F8B73895F8B8180133DBB2F3
:10100000012B85F8B73809D9B4F85E3885F8B728C8
:101010005B08A4F85E384B1C85F8B83895F8B828FA
:101020000023082AA4F8603815D185F8B838B5F837
:10103000BA3801339BB2032BA5F8BA3808D9237903
:10104000DB0705D5E36A94F85E0843B3216B984744
:101050000023A4F85E3838BD5B396C290CD8B4F88D
:101060005E3885F8B7285B0843F08003A4F85E3843
:1010700095F8B8380133CFE794F85938002BCDD123
:10108000012185F8B738A5F8BA38802384F85918B3
:10109000A4F85E3885F8B8185BF06CF8BEE7E36931
:1010A0006269D054E369E2680133B3FBF2F102FBF9
:1010B0001133E361CCE700BFD81C002470B50546AE
:1010C0000A26084C013E00D170BD94F9000019F0C9
:1010D000CFFF031E04DB6178EA185172A278EA544C
:1010E0000434EFE7E67F0A0838B555F04DFC0D49AA
:1010F0000D4CD1F8FC20A4FB00400C4D42F0807256
:101100000B4B800CC1F8FC204FF060420949E866A7
:10111000C2F8B01F00225A601A6842F001021A6039
:1011200038BD00BF00ED00E083DE1B43D81C002467
:10113000001000E055CEACC51B481C4AC1681C4BD2
:1011400010B44FF6FF0485B021401A4C0A43C26028
:10115000D3F8D010D3F8DC20C4F8BC1842F0005209
:10116000C3F8DC20D3F8DC2002F000520192019A8F
:10117000D3F8DC2042F08042C3F8DC20D3F8DC2036
:1011800002F080420292029AD3F8DC2042F0004240
:10119000C3F8DC20D3F8DC3003F000430393039B57
:1011A00005B05DF8044B9FE700ED00E00005FA058F
:1011B00000440258D81C00242DE9F04FAC4C83B0F9
:1011C000AC4D81464F1E10265AF008FB4FF4FA78BA
:1011D0004FF0E0214FF47A7C4FF0010E6B68C3F3BF
:1011E0000803002B40F06681EFF31183002B40F0E1
:1011F0006181636E8869626E9342FAD1A26E9042F9
:10120000F7D8E26E0CFB02FAAAEB000ABAFBF2FA7C
:101210000CFB03AA6B68C3F30803002B40F02C817E
:10122000EFF31183002B40F02781636E8869626EB3
:101230009342FAD1A26E9042F7D8D4F86CB00CFB6E
:101240000BF2121AB2FBFBF20CFB0323A3EB0A0313
:10125000B3F57A7FDED3B8F10108BFD1D4F8CC174B
:1012600094F8D4E7D4F8C82751B18EF00203B1F84E
:1012700004C00868C3F340031B010CFA03F3836145
:1012800032B10EF0010390881B01984013689861F9
:1012900048464FF0010C4FF0E02351B1D1F800E087
:1012A0008988DEF8148011EA080F18BF0904CEF807
:1012B000181042B111689288D1F814E012EA0E0FAA
:1012C00018BF12048A61B4F8C428002A40F06C8167
:1012D00094F8CC18D4F8C828002940F05E812AB1CF
:1012E0009188D2F800E00904CEF81810FA21BA4625
:1012F0004FF47A7E01900F466A68C2F30802002A12
:1013000040F01181EFF31182002A40F00C81626EEF
:101310009869616E8A42FAD1A16E8842F7D8E16E6F
:101320000EFB01FBABEB0008BB46B8FBF1F80EFB74
:1013300002886A68C2F30802002A40F0E180EFF3F5
:101340001182002A40F0DC80616E9F69626E9142DA
:10135000FAD1A26E9742F7D8E06E0EFB00F2D21BD4
:10136000B2FBF0F20EFB0122A2EB0802B2F57A7F8B
:10137000DFD35F46013FBFD1D4F8CC275746019851
:1013800042B111689288D1F814E012EA0E0F18BF2A
:1013900012048A61D4F8C82742B111689288D1F842
:1013A00014E012EA0E0F18BF12048A61B4F8C428C0
:1013B000002A40F0128194F8CC18D4F8C8280029EB
:1013C00040F0038122B1D2F800E09188CEF81810E5
:1013D000FA21BA464FF47A7E01900F466A68C2F34A
:1013E0000802002A40F0BC80EFF31182002A40F08E
:1013F000B780626E9869616E8A42FAD1A16E8842A6
:10140000F7D8E16E0EFB01FBABEB0008BB46B8FB67
:10141000F1F80EFB02886A68C2F30802002A5CD168
:10142000EFF31182002A58D1616E9F69626E91427A
:10143000FAD1A26E9742F7D8E06E0EFB00F2D21BF3
:10144000B2FBF0F20EFB0122A2EB0802B2F57A7FAA
:10145000E1D35F46013FC1D1019857460138C0B280
:10146000FF2800F0C680D4F8CC17D4F8C82714E7BA
:10147000D81C002400ED00E0EFF3118386F31288FE
:10148000D1F818B00A69D00303D5C4F8C0E8D1F880
:1014900018B0606EDBB2D4F8C02883F31188024420
:1014A000E06E0CFB00F3A3EB0B03B3FBF0F30CFBC0
:1014B0000233CBE6EFF3118286F3128888690B6959
:1014C000DB0302D5C4F8C0E88869636ED2B2D4F8F1
:1014D000C0A882F31188534493E6EFF3118286F398
:1014E00012889F691969C90302D5C4F8C0C89F69E9
:1014F000606ED2B2D4F8C01882F3118801449BE721
:10150000EFF3118286F312889F691969C90302D526
:10151000C4F8C0C89F69606ED2B2D4F8C01882F314
:101520001188014418E7EFF3118186F31288986956
:101530001A69D20302D5C4F8C0C89869626EC9B2EC
:10154000D4F8C08881F31188E16E4244BB460EFB9B
:1015500001F8A8EB0008B8FBF1F80EFB0288E8E6FA
:10156000EFF3118186F3128898691A69D20302D5C4
:10157000C4F8C0C89869626EC9B2D4F8C08881F353
:101580001188E16E4244BB460EFB01F8A8EB00084F
:10159000B8FBF1F80EFB02883DE7002A3FF4A6AE47
:1015A000D2F800E091889FE6D4F8E428002A3FF4BE
:1015B0009DAEB4F8E8E84B49D4F8D028B1FBFEF171
:1015C0004910116084F8E1C890E6002A3FF400AFAA
:1015D0009188D2F800E00904F8E6D4F8E428002A5B
:1015E0003FF4F6AE0021D4F8D028116084F8E11859
:1015F000EEE64FF47A7E4FF0E0214FF00108F4461A
:101600006B68C3F30803002B58D1EFF31183002B51
:1016100054D1636E8869626E9342FAD1A26E904291
:10162000F7D8E26E0CFB02FAAAEB000ABAFBF2FA58
:101630000CFB03AA6B68C3F308030BBBEFF3118326
:10164000F3B9636E8869626E9342FAD1A26E9042DA
:10165000F7D8D4F86CB00CFB0BF2121AB2FBFBF209
:101660000CFB0323A3EB0A03B3F57A7FE2D3BEF1AD
:10167000010EC5D1013FBFF4A7AD03B0BDE8F08FA7
:10168000EFF3118386F31288D1F818B00A69D203F8
:1016900003D5C4F8C088D1F818B0606EDBB2D4F8B6
:1016A000C02883F311880244E06E0CFB00F3A3EB27
:1016B0000B03B3FBF0F30CFB0233D3E7EFF3118220
:1016C00086F3128888690B69DB0302D5C4F8C088E9
:1016D0008869636ED2B2D4F8C0A882F311885344EB
:1016E0009FE700BF40420F0010B590F82830044635
:1016F000012B03D000230120637710BD406A0368EB
:101700001A7B42B95DF02AF800F00103C243637707
:1017100002F00100F1E71B6A002BF3D0002010BD9E
:1017200038B5114D044694F82830012B05D000231C
:10173000637700230120236238BD606A03681A7B47
:101740006AB95DF00BF800F001036377C307F0D5C9
:101750006B6E226A9B1A002BE5DB002038BD1B6AEA
:10176000002BEED0F4E700BFD81C002410B5FF22F8
:10177000044690F82810406A62F08AF90E4B204621
:101780005B6E03F5FA732362FFF7CAFF94F8283003
:10179000012B00D010BD0022A021606A62F02EF95A
:1017A00094F82830012BF5D1606A1822B021BDE8E9
:1017B000104062F023B900BFD81C002438B504469D
:1017C0000D46FFF7ADFF062294F82810606A62F01C
:1017D0005FF9012294F828306277934204D0064BD7
:1017E0005B6E0F33236238BDE288D821606AB5FB97
:1017F000F2F262F029F9F2E7D81C00242DE9F8434F
:10180000838853B304460025DFF85480012707E09E
:10181000D8F864300135A2880F33AA4223621CD95C
:101820002046268AB4F80690FFF77AFF062294F83D
:101830002810606A62F02CF994F828306777012B41
:10184000E6D109FB06F6E288D821606A05FB06F6B8
:10185000B6FBF2F262F0F8F8DAE7BDE8F88300BF11
:10186000D81C002470B5104D95F8EA3803B970BD46
:10187000C3880446D5F8EC68B6FBF3F60B4B5E6004
:10188000FFF74EFF94F82830012B06D06B6E002234
:10189000023385F8EA28236270BD32461021606A5F
:1018A00062F0D2F8F2E700BFD81C00240000002448
:1018B0002DE9F04F594F90461E46C38897F8EA2805
:1018C00099B004460D46B1FBF3FA002A40D1DFF887
:1018D0005891D9F80430534522D1E188B5FBF1F392
:1018E00001FB135594F82830491BB14234BF1FFA4D
:1018F00081F91FFA86F9012B4CD07B6E204602330A
:101900002362FFF70DFF38B194F82830012B34D053
:10191000484619B0BDE8F08F002019B0BDE8F08F3F
:101920002046FFF7FDFE0028F6D04FF0FF33C9F840
:10193000043094F82830012B6AD07B6E20460233A5
:101940002362FFF7EDFE0028E6D0C9F804A0C4E743
:10195000D7F8EC28DFF8D090B2FBF3FBC9F804B05D
:10196000FFF7DEFE94F82830012B4BD07B6E02335C
:101970002362002387F8EA38ABE7606A5CF0EEFE8A
:10198000C0F30113013B022BC2D82046FFF7EEFE45
:101990004846BEE78DF81C3000228DF8443004A97B
:1019A0008DF858301E4B8DF80E502D0A1B688DF89F
:1019B0000D50ADF808301B0C656A8DF80A30032312
:1019C00028468DF80F208DF80C300693154B0A929F
:1019D000089303AB8DF830200993042317920B93DF
:1019E00002AB049301ABCDE90F86CDE90D22CDE921
:1019F0001222CDE91422059350F0E6F9286860F030
:101A0000A9FB7AE75A461021606A62F01DF8ADE73B
:101A100052461321606A62F017F88EE7D81C002442
:101A2000A0080B081D0A0408000000242DE9F04F4F
:101A3000D0F8249083B03F4F0446D9F800000E46FA
:101A4000904660F087FB97F8EA38002B40D0D7F833
:101A5000F058E288DFF8E8B0DFF8E8A0B5FBF2F371
:101A600002FB13538BF822301B0A8BF821303368AA
:101A70005146314E4846C6F8A83006F1A802D8F8BB
:101A80000030C6F8B0300023C6F8B83050F050FA35
:101A9000D8F800200123E188154487F8EA38B5FB1F
:101AA000F1F301FB1353C7F8F0581BB3234BC6F8EF
:101AB000B830637F0BB90AF1140A514648462263D5
:101AC00050F082F9E36A6BB3206B03B0BDE8F08F8E
:101AD000A569E288DFF868B0DFF86CA0C7F8EC58B9
:101AE000B5FBF2F302FB13538BF842301B0A8BF861
:101AF0004130BCE7D7F8EC2848460193B2FBF1F23D
:101B0000726052BA06F1A801ABF8622006F1D00269
:101B100050F00EFA019BD8F8002087F8EA38C7F891
:101B2000EC58C6E7636A186860F014FB206B03B0DA
:101B3000BDE8F08FD81C002400000024490A0408E6
:101B4000A0F20024080000245800002433B910B586
:101B50001C46C36A20469847204610BD66E700BF72
:101B600010B582B00C46019201A9049A8461C26248
:101B70006A460093FFF75AFF02B010BD2DE9F84303
:101B8000DDF820800F4616460021202204461D461F
:101B900065F038F9B8F1000F0CD0D8F80030B8F87B
:101BA0000A20E3811B0C2382D8F804306282E3828E
:101BB0001B0C2383384662F059F8F30619D4431EF0
:101BC000B8B107EB000C01E0013B12D31CF801EDAA
:101BD000BEF12E0FF8D1C01A03F10109421EB9441B
:101BE000032AA8BF0322082BA8BF082390461A4641
:101BF00006E008280246B9464FF00008A8BF0822B0
:101C00004FF02033394620462360636065F09CF82E
:101C1000164B04F10800424649462381837065F063
:101C200093F8611EE21D11F801CFACF16103ACF134
:101C3000200C192B98BF81F800C09142F3D104F118
:101C40000A0011F8013FA3F16102203B192A98BF55
:101C50000B708142F5D1182365832D0CE672237336
:101C6000099BA582E361BDE8F88300BF2020200026
:101C70002DE9F04FDFF8589485B0D9F86400C9F821
:101C8000C407002B60D00C46154601F5FE7603EB29
:101C9000020B1FE0002D64D0D9F8F437AB4200F0FE
:101CA000C780D9F8F037AB4200F0F980D9F8F8379F
:101CB000D9F8FC17AB424BD88D42C0F07481691A39
:101CC000204659F0D9F9013504F5007406F500767F
:101CD0005D4539D0D9F80028AA42DBD8AA1AD9F82C
:101CE0001078D308396B02F0070802338B4202D315
:101CF000BA6B93420BD939461846039359F08CF9C5
:101D0000039B0746002800F06E81C9F810083A7955
:101D1000002A40F01F81D7F828A0BAF1000F00F088
:101D20005B813A6B013520464FF400719B1AFA68CB
:101D300004F5007406F5007608EBC3083B4602EB99
:101D40004822D0475D45C5D1002005B0BDE8F08FE1
:101D50008D42B4D24FF400720021204665F052F853
:101D6000B1E74FF400722946204665F04BF8802316
:101D7000CB4A84F8BE310C2384F8C231D9F8F0176D
:101D8000D9F8E8379142C4F8C611C4F8CA3100F353
:101D90000F81C44A013BC44F82FB0102C81787FB75
:101DA00001C70A44C0EB6212C0EB2730BF4F87FB6C
:101DB00002C7C2EB821C84F8C1018010A1EB0C01A8
:101DC000174420F03F0001310843D117C1EBE71160
:101DD00084F8C0010A4484F8BF21B14A934200F359
:101DE000F380B04AB04882FB0312D91780FB03701E
:101DF0001A44C1EB6212C1EB2031AC4880FB027087
:101E0000C2EB821784F8C5118910DB1B104421F046
:101E10003F0101331943D317C3EBE01384F8C41116
:101E20001A4484F8C3214AF65523A4F8FE314AE740
:101E30004FF0FF3300274FF4F072201D84F8EC318F
:101E4000394684F8ED3184F8EE3184F8EF315223CD
:101E5000237063706123A37084F8E7314123E3703A
:101E600084F8E631722384F8E43184F8E531D9F856
:101E70000838C4F8E83164F0C5FF5523C4F8F071A0
:101E800084F8FE316FF05503C4F8F471C4F8F871AA
:101E900084F8FC7184F8FD7184F8FF3113E74FF486
:101EA00000720021204664F0ADFF814B022203CB7B
:101EB00045F6EB032274227323809023A273A37050
:101EC000F82384F82C200822C4F803006273C4F8B5
:101ED00007106375D9F8F017D9F8E8375B1AD9F805
:101EE000F8172362D9F8FC375B1A4AF6552163626A
:101EF0000023E372E3736377A377E37784F82D30ED
:101F000084F82E3084F82F3084F83130694BA36187
:101F10003E232377012384F83030802384F8403037
:101F2000654BC4F84230654B84F84620A4F8FE1196
:101F3000634A03CBC4F84B101988C4F847009B7858
:101F4000A4F84F1084F8513003CAC4F85200C4F802
:101F50005610B8E64FF400720021204664F052FF9C
:101F60003B6CB8F1000F45D104F1200A002B00F0C2
:101F700081803B6B112253492046CDE90088FFF751
:101F8000FDFD3B6C1A6C002A00F081801B6B5046F3
:101F900011224D49CDE90088FFF7F0FD04F1400A18
:101FA0004FF4E07871E0E91A204659F065F88AE6C6
:101FB000FF22013B84F8C1214FF6FF72A4F8BF2134
:101FC000374A93427FF70DAFFF2384F8C5314FF6B0
:101FD000FF73A4F8C33126E751464FF40072204640
:101FE00064F010FF6FE6231F384A43F8042F9E4227
:101FF000FBD168E6002B7F6C14BF02230123C3EBE7
:102000000813002F3FF45FAE013BBF6C002B01DDD6
:10201000002FF9D1A2464FF40078002F3FF453AEC1
:102020000AEB080303959A460BE00025A8F1200867
:10203000CDE900E5FFF7A2FDBF6CCFB1B8F11F0FEE
:1020400016D93D7907F11C0E112239683B6BAAEBBA
:102050000800002DE9D17A79A8F120083D6942F005
:102060002102CDE900E5FFF789FDBF6C002FE5D126
:10207000039D28E6CDE9008843464FF4F078082216
:10208000D9F8EC172046FFF779FD7F6CC5E750467D
:10209000434611220C49CDE90088FFF76FFD7DE72B
:1020A000FF03FB0083200882975545418180808093
:1020B000AC080B083F00FF0029940E0DB8080B0870
:1020C000C4080B08A4080B08A8080B08DEADBEEF77
:1020D000D81C002410B40F4CBFF34F8F0E4BC3F825
:1020E0005C42BFF34F8FBFF36F8F0C4B03F1300097
:1020F000A3F6F40C5A7A3AB11A7A34F812100CEBAF
:10210000420289B2A2F848190C338342F2D15DF839
:10211000044B704780F4002400ED00E0CC2500243F
:1021200000207047704700BF014854F0E9B800BF75
:1021300048260024084810B4D0F87039D0F8A449D3
:1021400099691A682CB1234600F517605DF8044BB5
:1021500018475DF8044B7047D81C0024014854F020
:10216000CFB800BFAC260024084810B4D0F8D4394A
:10217000D0F8084A99691A682CB1234600F6D410A1
:102180005DF8044B18475DF8044B7047D81C0024D9
:10219000014854F0B5B800BF10270024084810B417
:1021A000D0F8383AD0F86C4A99691A682CB12346AD
:1021B00000F638205DF8044B18475DF8044B704773
:1021C000D81C0024014854F09BB800BF7427002499
:1021D000084810B4D0F89C3AD0F8D04A99691A68E7
:1021E0002CB1234600F69C205DF8044B18475DF89F
:1021F000044B7047D81C00242DE9F04784B08DF8BB
:102200000F30431C00F09F800328044600F39B809E
:10221000824E642303FB0063D3F87009002800F0AA
:10222000928093F8B159202D40F0878093F8B059EF
:10223000012D00F082800125D6F8E87A83F8B059A4
:1022400004E0D6F8E83ADB1B192B66D8856915F44B
:102250000045F6D14FF0640A714B00974FEA4108F0
:102260000AFB04FA41460AEB0309B244212348461B
:10227000CAF8A4598AF8B13940238AF8B2390DF165
:102280000F03CAF8B459CAF894390123AAF89A3945
:102290000A235AF00DFF002873D1BAF89A399BB27D
:1022A000FF2B40F29180DAF87019FF235D48AAF8FD
:1022B00098394B685C4A034043EA08031A434A6072
:1022C000642505FB046505E0B5F89A399BB2002B3F
:1022D00000F08C803A460A21484654F04FF860BB23
:1022E000D5F89439D5F8701913F8010BB5F8982979
:1022F0008862C5F89439013AB5F89A3992B2013B2F
:10230000A5F898299BB2A5F89A39B5F89A399BB2E5
:10231000002BD9D0002AD7D11EE064232020002131
:1023200003FB0463D3F8B42983F8B0190243C3F85C
:10233000B42983F8B10983F8B219B6F8EC3A01333D
:102340009BB2A6F8EC3A002004B0BDE8F087D6F8BE
:10235000E83ADB1B0A2B27D88A6912F08002F6D0F4
:10236000B5F89A399BB2FF2B0ED94B682D4A134012
:102370002D4A43EA08031A43FF23A5F898394A6017
:10238000A2E78AF8B059D8E7B5F89A3925489BB240
:102390004A68A5F89839DBB2024048EA0343134380
:1023A00043F000734B608FE76423202103FB046438
:1023B000D4F8B43984F8B0290B43C4F8B43984F89C
:1023C000B11984F8B229B8E7BAF89A39DAF870196D
:1023D0009BB214484A68AAF89839DBB2024048EA2E
:1023E0000343134343F000734B6069E739464846A3
:1023F0005AF00AFE034600289FD1D5F87029202400
:102400000A48D461516801400120516085F8B14902
:1024100085F8B03985F8B23996E700BFD81C00249A
:1024200048260024009C00FC0000FF0100E800FE9C
:10243000B0F1FF3F00F00A8103282DE9F04706467E
:1024400082B000F3A3808F4C642000FB0640D0F8DC
:102450007079002F00F09A8090F8B159202D40F04B
:102460008F8090F8B059012D00F08A80012580F806
:10247000B059D4F8E85AB86910F4004909D0D4F832
:10248000E80A401B192800F28580B86910F4004959
:10249000F5D14FF0640A7C4F4FEA41080A990AFBD4
:1024A00006FA00955744A244CAF8941922213846E6
:1024B000CAF8A4998AF8B11940218AF8B21941469C
:1024C000CAF8B499AAF89A390A235AF065FD002887
:1024D00040F0BE80BAF89A399BB2FF2B6BD8BAF89D
:1024E0009A39DAF870199BB268484A68AAF898399C
:1024F000DBB2024048EA03431343654A1A434A6089
:102500004FF0640909FB064904E0D4F8E83A5B1B84
:102510000A2B26D88A6912F00402F6D04A6AD9F842
:1025200094391A70B9F89A39D9F89429013B0132D3
:102530009BB2C9F89429A9F89A39B9F89839B9F829
:102540009A29013B92B29BB2A9F898390BB9002A9B
:102550003FD1B9F89A399BB2002B7CD0D9F87019C9
:10256000D8E76423202003FB0643D3F8B41983F88B
:10257000B0290143C3F8B41983F8B10983F8B2292B
:10258000B4F8EC3A01339BB2A4F8EC3A002002B064
:10259000BDE8F08764232020002103FB0643D3F825
:1025A000B42983F8B0190243C3F8B42983F8B109F8
:1025B00083F8B219E4E7DAF87019FF233348AAF870
:1025C00098394B68334A034043EA08031A434A6088
:1025D00096E7D9F8701904E0D4F8E83A5B1B0A2BA7
:1025E00024D88A6912F08002F6D0B9F89A399BB2E1
:1025F000FF2B0BD94B68284A1340284A43EA0803AB
:102600001A43FF23A9F898394A60A2E7B9F89A3922
:1026100021489BB24A68A9F89839DBB2024048EADF
:102620000343134343F000734B6092E7642320217C
:1026300003FB0646D6F8B43986F8B0290B43C6F832
:10264000B43986F8B11986F8B22999E700207047A5
:102650008AF8B09994E7294638465AF0D5FC0346E3
:1026600000288DD1D9F8702920240D48D4615168F3
:1026700001400120516089F8B14989F8B03989F8E1
:10268000B23984E7D81C002448260024009800FCB6
:10269000002400820024FF81009C00FC0000FF0158
:1026A00000E800FE2DE9F0410468D4E90435A86192
:1026B0001A7D1F681F2A49D9203A20212E6801FA65
:1026C00002F242F01802FA602A7D1F2A48D9203A05
:1026D000202101FA02F242F01802F2606A68002139
:1026E0005868016038461160116841F010011160AE
:1026F00093F80880A26941465EF06EFA2D7AE2698D
:10270000304629465EF068FA226A63689468184A7F
:1027100012F80800515D5A686FF30F0222435A60A5
:102720003A5842F001023A50725842F00102725097
:102730009A6842F440429A601A6842F001021A60B4
:102740001A6842F400721A60BDE8F08120212E68F8
:1027500001FA02F242F01802BA602A7D1F2AB6D8A6
:10276000202101FA02F242F01802B260B6E700BF7F
:10277000C8090B08D3B20F2B22D8124B00B503F1B6
:102780007E0E02E00333734517D093F800C08445F2
:10279000F8D193F801C08C45F4D102EB42020A480B
:1027A000997800EB820300F59070C3F8281100EBD4
:1027B000820083F820115DF804FB00205DF804FB23
:1027C000002070470C800A080000002410B40C4C54
:1027D000002304F52F6C01E0152B0CD003EB430212
:1027E00001331CF802108142F6D1144494F9F20A24
:1027F0005DF8044B70474FF0FF305DF8044B7047B5
:10280000D81C002430B5134D002305F69C3C02E093
:1028100001331A2B1BD05CF833408442F8D10CEB07
:10282000C30EDC009EF804E08E45F1D102EB4202BB
:10283000094B254403EB820103F5907395F8A14BF6
:1028400003EB8200C1F8284181F8204130BD00200F
:1028500030BD00BFF0740A0800000024F0B100236E
:1028600010B504460E4894F804E000F52F6C01E022
:10287000152B11D003EB430201331CF802107145F4
:10288000F6D183186179206893F9F22AD3B20F2B1D
:1028900002D8BDE81040B5E7002010BD0020704709
:1028A000D81C002401380E4B0E4A00EBC000D2F8B1
:1028B000D81003EB800310B4D3F8E03183B00A4C96
:1028C000A34214BF022301231943C2F8D810D2F83F
:1028D000D82013400193019B03B05DF8044B70476F
:1028E0000000002400440258000002400138F8B5FE
:1028F00000EBC000124C1D46124B04EB800417463F
:102900000E46D4F8E001984214BFA120A0205AF04E
:10291000B1FCB4F9F601B909C4F8F061C4F8F85192
:102920005AF010FBB4F9F631002B07DB03F01F005F
:1029300001225B090449824041F82320F8BD00BF11
:10294000000000240000024000E100E02DE9F04F0B
:10295000BF4B85B0DFF80CA34FF001090026BD4F37
:102960000AF1F00BA3F5907809E0013609F10109AD
:102970000AF1280A0BF1050B062E00F0FC809AF8EC
:102980000030022BF1D19BF90320541C00F0F6809B
:10299000D2B29446AE4B02EB4204F1B203EB840494
:1029A00033465E46D346CA4699460F2A5FD8AA48A0
:1029B00002E00330B8425AD00378002BF9D14578B1
:1029C0008D42F6D1857801936068D8F8E431A5602E
:1029D0009842257000F04881D8F80832984200F0FB
:1029E0006A81D8F82C32984200F06E81D8F85032C3
:1029F000984200F06E81D8F87432984200F07881E5
:102A0000D8F89832984200F08C81D8F8BC329842BD
:102A100000F08281D8F8E032984200F08C81D8F83A
:102A20000433984200F08281D8F82833984200F0AD
:102A30009981D8F84C33984200F08D81D8F87033E2
:102A4000984200F0B481D8F89433984200F0A881FD
:102A5000D8F8B833984200F0B881D8F8DC339842FF
:102A600000F0BA81D8F80034984200F0A781013212
:102A70000C34D2B2624598D94B46D146DA46B346B9
:102A80001E46002303939BF90420531C7AD0D2B234
:102A9000964602EB42046E4BF1B2B44603EB84045B
:102AA0000F2A5DD86C4802E00330B84258D0037852
:102AB000012BF9D145788D42F6D18678D8F8E451CA
:102AC0006068A660A842267060D0D8F80852A84274
:102AD00000F0F680D8F82C52A84200F0FF80D8F819
:102AE0005052A84200F0FF80D8F87452A84200F07B
:102AF0000481D8F89852A84200F00981D8F8BC5255
:102B0000A84200F0FF80D8F8E052A84200F01E81F1
:102B1000D8F80453A84200F01381D8F82853A842EB
:102B200000F02D81D8F84C33984200F02281D8F87B
:102B30007033984200F02E81D8F89433984200F018
:102B40002381D8F8B833984200F05981D8F8DC33A3
:102B5000984200F04E81D8F80034984200F043814A
:102B600001320C34D2B272459AD966460022002353
:102B7000CAE90423F9E605B0BDE8F08F4FF00F0C69
:102B8000002207E74FF00F0E002282E700231846CD
:102B9000029300EBC0050130019008EB850090F82E
:102BA000FC51002DDCD1324680F8E8312B4B6646D3
:102BB000C0F8EC21029A80F8FD911344CAF8143051
:102BC000132380F8FC310198FFF76CFE039B002B68
:102BD000CCD0DAF814402046FDF712FADAF81000EB
:102BE000FDF70EFADAF81830C168DAF804205962F5
:102BF00040215D60996002F120019D631960C3E985
:102C00000355C3E90555C3E90755C3E90A55C3E9A7
:102C10000C5594B1E1683032DAF81C3059621D620B
:102C20009D63C3E90025C3E90255C3E90455C3E91F
:102C30000655C3E90A55C3E90C5500230198084914
:102C40001A46FFF753FE01238AF80C308DE600BFC9
:102C5000200100248A800A080C800A08E001002470
:102C6000390A0000082800240198029000EBC00EE9
:102C7000431C08EB8E0E03939EF8FC0100287FF4A2
:102C8000F6AE4A461846019BD146DA46B3468EF860
:102C9000E83116465D4B029ACEF8EC5113448EF89B
:102CA000FD91CAF8103014238EF8FC31FFF7FAFDBD
:102CB00001230393E7E601202423CDE90103D5E7AF
:102CC00024200290184664E702204823CDE901033E
:102CD000CCE703206C23CDE90103C7E7482002239A
:102CE0000290184655E76C2003230290184650E7DF
:102CF00004209023CDE90103B8E79020042302903B
:102D0000184646E7D82006230290184641E7B4202B
:102D10000523029018463CE70620D823CDE901039D
:102D2000A4E70520B423CDE901039FE74FF4907396
:102D3000082002939AE70720FC23CDE9010395E7D9
:102D40004FF4907000230290082022E7FC20072314
:102D5000029018461DE702204FF4B473CDE9010339
:102D60000A2083E701234FF4A27E0920CDE9013E2A
:102D70007CE74FF4B470022302900A2009E74FF475
:102D8000A2700290092004E74FF4D8700423029047
:102D90000C20FEE64FF4C670032302900B20F8E6E9
:102DA0004FF4D8700423CDE901300C205EE70323F3
:102DB0004FF4C67E0B20CDE9013E57E74FF4077074
:102DC0000723CDE901300F2050E705234FF4EA7EB9
:102DD0000D20CDE9013E49E74FF4FC700623CDE913
:102DE00001300E2042E74FF40770072302900F20B6
:102DF000CFE64FF4FC70062302900E20C9E64FF494
:102E0000EA70052302900D20C3E600BFE001002414
:102E1000234B5B68C3F3080310B4DBB9EFF31183F2
:102E2000C3B9204B4FF0E02C5A6EDCF81800596EF5
:102E30008A42F9D1996E8842F6D8DC6E4FF47A71E5
:102E400001FB04F3181AB0FBF4F05DF8044B01FB2E
:102E500002007047EFF31181102383F312884FF0C3
:102E6000E0229469136913F4803F0E4B03D00120D4
:102E7000C3F8C0089469586EC9B2D3F8C02881F36A
:102E80001188D96E4FF47A73024403FB01F0001BE2
:102E90005DF8044BB0FBF1F003FB0200704700BF8C
:102EA00000ED00E0D81C0024BE4803780BB90120D7
:102EB000704743682DE9F04F002BDFF8109387B07F
:102EC000D9F8646018DD00F108050024B649D5F88A
:102ED000F430BFF34F8F03F59072C1F85C322033AA
:102EE0009342FAD1BFF34F8FBFF36F8F0134436822
:102EF00005F586759C42EADB90F8F815AB4A04911B
:102F0000A2FB0612AA4BAB4E5209DFF8C4A2A3FBE8
:102F10000213DB0803EB8303A2EB4303DAB206EBF5
:102F2000830B06F538730592009300239846049BA3
:102F3000984500F01481DAF81830DAF80470D3E913
:102F40003D45FFF765FF9C4999F83FEC0122691860
:102F50000190BEF1540F99F83E0C02FA07F204EB0F
:102F6000410104EB400301D1A9F8460C994240F21B
:102F70006A811F88174200F05F815F88174200F066
:102F800070819F88174200F06E81DF8808331742F6
:102F9000ECD11C1B99424FEA640440F25481281B77
:102FA000452828BF452003EB4000834280F04F8135
:102FB00000251F46AC462946CDE9028EB3F800E055
:102FC0000EEA020E8E451CD1B3F802E00EEA020EA4
:102FD000714540F01A81B3F804E00EEA020E714523
:102FE00040F01581B3F80680083308EA020841452D
:102FF00008D1984209D9B3F800E00EEA020E8E45D6
:10300000E2D00233984200F2E580BCF1110FDDE915
:10301000028E40F21C81DCF1150200F11881674933
:10302000D9F8500CD1F820349C4238BFC1F8204464
:10303000019C231A002B14DB614B03449C4201D9F1
:1030400023460533C9F8503CD1F82034052B40F213
:103050000C81053BDBB289F83E3C4FF0FF33C1F8F1
:1030600020343AB105FA02F2CCF1140C012505FA2C
:103070000CF51543534BC5F3C43203EB8202D2F86F
:103080006C0C05F01F0203EB8202D2F86C1CC5F336
:103090004412C5F3842503EB820241EA0031D2F8E1
:1030A0006C2C03EB850341EA0211D3F86C3C41EA36
:1030B0000321454B81EA1122D3F81C3A82EA12120D
:1030C000013302F00F020F2A40F0A380B1F5803FD8
:1030D00080F09F80BEF1540F4FEA111147D03A4A59
:1030E000B1F5606FC2F81C3A4DD0009B998196F8FB
:1030F00058300598834210D0DBF8082033689B1ABB
:1031000033607368DBF830209B1A73600023CBF8C0
:103110000830CBF8303086F858003368013333601C
:10312000DBF808300133CBF808304FF6FF739942D3
:1031300007D1736801337360DBF830300133CBF8AB
:103140003030009B08F101085C360BF15C0B143346
:10315000B8F1080F0AF1200A00937FF4E8AE0123CA
:10316000194A012082F8183B07B0BDE8F08FB9F882
:10317000402CB1F5606F02F10102A9F8402C124A0F
:10318000C2F81C3AB1D199F8013003EB430309EBC3
:10319000C30343445B7C0D2BA7D18023009A937714
:1031A000A5E700BF0400002000ED00E01F85EB5103
:1031B000CDCCCCCC30180020C7FFFF7F000000240E
:1031C00020A10700F0740A08FC100020D81C00247D
:1031D0003C040020A3EB070E254F33F8021C4FEAF6
:1031E0006E0E11400EF1010E87FB0E87A7EBEE77F6
:1031F0004FF0010E012FB8BF0127BD40BC44013F75
:103200000EFA07F73D431F46D8E60433FAE60633C5
:10321000F8E6BEF1540F04D1B9F8402C0132A9F8F8
:10322000402C144A4FF6FF71C2F81C3AD2F8183AF3
:103230000133C2F8183A5AE702331C1B99424FEA8D
:1032400064043FF6ACAE10B1013889F83E0CBEF113
:10325000540F7FF476AFB9F8423C0133A9F8423CF1
:103260006FE7043395E6063393E60023F3E600BFE9
:1032700056555555FC100020264B70B51A785B78D2
:103280009A4242D1244E7368002B22DD06F10800D9
:103290000025224CD0F8AC30BFF34F8F03F1E00291
:1032A000C4F8683220339342FAD1BFF34F8FBFF393
:1032B0006F8F337813B1037F012B20D04269013522
:1032C000716800F586701368A94243F0010313602A
:1032D000E0DCFFF79DFD124BD3F81C4B002C0DDDFD
:1032E00003F5326303EBC4041968083333F8042C84
:1032F000C8689C4242EA0002CA60F5D170BD002352
:1033000080F8FC30FCF7A2FED8E75FF02DFF002824
:10331000B8D170BDD81C00240400002000ED00E0EE
:10332000FC100020800AA0F58010522807D8054B19
:1033300003441B7D0D2B02D8034AD0567047002052
:10334000704700BFF0740A08B8090B0860B18288A2
:103350004FF0B0414FF00043B2FA82F2D1F8800052
:10336000D3400343C1F88030704700BF4FF0B042F4
:10337000D2F88030D2F888100B4003F00103C2F875
:10338000883023B1024BD3F8540C036818477047B8
:10339000D81C00244FF0B042D2F88030D2F8881008
:1033A0000B4003F00203C2F8883023B1024BD3F87C
:1033B000580C036818477047D81C00244FF0B042DF
:1033C000D2F88030D2F888100B4003F00403C2F822
:1033D000883023B1024BD3F85C0C03681847704760
:1033E000D81C00244FF0B042D2F88030D2F88810B8
:1033F0000B4003F00803C2F8883023B1024BD3F826
:10340000600C036818477047D81C00244FF0B04286
:10341000D2F88030D2F888100B4003F01003C2F8C5
:10342000883023B1024BD3F8640C03681847704707
:10343000D81C0024F8B54FF0B043D3F88050D3F82F
:103440008820154005F47875C3F888507DB1084F81
:103450000126B5FA85F4C4F11F0407EB840306FACC
:1034600004F4D3F8540C03689847A543F1D1F8BD90
:10347000D81C0024F8B54FF0B043D3F88050D3F8EF
:103480008820154005F47C45C3F888507DB1084F6D
:103490000126B5FA85F4C4F11F0407EB840306FA8C
:1034A00004F4D3F8540C03689847A543F1D1F8BD50
:1034B000D81C002430B1036882881B691A4214BFEB
:1034C00001200020704700BF10B1036882889A6114
:1034D000704700BF18B1838802681B04936170476E
:1034E00070B50D4682B00446164640B101680C4BDB
:1034F0000C4A0B449B0A02EB4303B3F8E40A59F06D
:10350000B9FEC5F38101C5F3411305F01302CDE9FE
:103510000016A18820685EF0A1FB02B070BD00BF5C
:103520000000FEA7F0740A0800B1D9E770472DE942
:10353000F84FC14F6423044603FB0073D3F8586966
:10354000002E00F06481D3F86089B8F1000F04D038
:1035500098F80630002B40F05A81642303FB047373
:10356000D3F864591DB1AB79002B40F05081631C36
:10357000DBB2B8F1000F04D0152288F8073088F8C4
:10358000062015B11622EB71AA714FF0640A308B38
:1035900059F070FE29460AFB04FA40465FF064FDCC
:1035A000404607EB0A09DFF8B48299F86A3999F8BE
:1035B0006829002B0CBF4FF01E0B4FF03E0B5946F5
:1035C000FFF7B2FF28469D4D594699F869295544A1
:1035D000FFF7AAFF4C220021284663F013FCD9F81C
:1035E0005839974A5B689342C9F87039DFF870928E
:1035F00040F00F8153F0EAF9D9F82030C3F30213F9
:10360000434493F8EC3C03F01F039FED8E7A9FED4B
:103610008E5AB0EE084AD8406423F7EE003A4FF0D5
:10362000000C07EE900A03FB047340F21458F8EE06
:10363000677AB3F86CA9C7EE275A07EE90AA9FEDF8
:10364000837AF8EEE77AC7EE274ADFED817AB0EEAB
:10365000007AE5EE877AA5EE875A25EE844A37EEA2
:10366000856A74EEE72ABAF5C87F0CF1010ED5BF62
:103670004FF4967278226423322307EE90EAD8BF83
:103680004FF416791344A2F13202F8EEE76AC8BF8C
:103690004FF4827907EE903AD4BF41464FF4FA7165
:1036A00066EEA56AB8EEE77AC7EE267A07EE102A2C
:1036B00001EB0902B8EEC77A37EE447A77EEE37A87
:1036C000FCEEE77A17EE903AC7EE267AFCEEE77A40
:1036D00017EE900A07EE909AB8EEE73A07EE902AB6
:1036E000F8EEE77A23EE243A83EE277A37EE453A6E
:1036F00032EEC77AC3EE267A77EEE37AFCEEE77A0B
:1037000017EE901AC7EE267A77EEE37AFCEEE77AA8
:1037100017EE902A02F1020909EB010BB0EE467A8E
:1037200007EE90BAF8EE677AA6EEA77AF4EEC74AEB
:10373000F1EE10FA79DC43EA00095FFA89F9B9F190
:103740000F0F74D841EA02091FFA89F9B9F1FF0F86
:103750006DD81B05000403F07F6392B200F47F0074
:1037600003433C4843EA0C7300EA01210B43134333
:103770006422284602FB04740027C4F8743901232C
:10378000C4F87879C4F87C39C4F88079C4F88479AD
:10379000C4F88C79C4F890795EF012FA94F8B139D3
:1037A000202BD9B21AD194F8B039012B16D024238A
:1037B00084F8B139D4F870391A6822F001021A601D
:1037C0001A6822F480521A601A681A601A6842F065
:1037D00001021A6084F8B11984F8B0790021F07EF2
:1037E00059F0B0FBF37E01241B4D5A0903F01F036F
:1037F000002104FA03F345F82230B07E59F0A2FB11
:10380000B37E5A0903F01F039C4045F82240BDE8EF
:10381000F88F53F0DBF8D9F81C30C3F30213984447
:1038200098F8EC3CEFE6F4461DE7013174E7BEF191
:103830000F0FF8D100239BE7D81C00244826002452
:10384000001C0058286B6E4E00001643002474497B
:103850000000704200FFFF0000E100E0F0740A0881
:103860000044025808B100223AE6704770B50E4C89
:1038700094F8F865AEB104F58764002503E00135DE
:103880002034B5420DD0237F002BF8D0E068002211
:103890000028F4D00135217DFFF722FE2034B54207
:1038A000F1D1012070BD00BF0400002070B590F878
:1038B000EE311C09013C082C0DD8194E054603F0C9
:1038C0000F0336F8140040FA03F2D20703D595F837
:1038D000F921012A01D0012070BD9A402644013A05
:1038E000104063F03FFC96F8FC3C0E4A034402EBA8
:1038F000C30452F83320A38810691840ECD0002389
:1039000095F8EF210221204685F8F931FFF7E8FD0F
:10391000D5F85021136843F008031360DBE700BFBC
:10392000F0740A08481D0024014B53F8200070472A
:1039300050400058014B43F8201070475040005849
:1039400019481A4B01681A4A41F4807130B482B0A8
:103950000160D3F8F410FF24CA2041F48031C3F889
:10396000F410D3F8F41001F4803101915321019D3A
:10397000546250625162D3F8D030DB010CD40C4B4E
:1039800000220C495A659A65DA651A665A669A6683
:10399000196502B030BC7047126D064B9A42EED1E9
:1039A00002B030BC704700BF0048025800440258C3
:1039B00000400058316665422DE9F84FD0F85C713F
:1039C0000446534B00F59676FDB227F0FF09826856
:1039D00000F1E00A103D4846D2F80080A3FB05350F
:1039E0002D0929465DF054F9D4F81C210023B2F5C5
:1039F000807F84F820317FD00DD8102A00F0848099
:103A00005DD8012A46D0042A16BF6FF400616FF01A
:103A100008013C230EE0B2F5805F71D0B2F5803F23
:103A20003BD0B2F5806F15BF6FF400616FF00801F5
:103A30003C230423324608F11806404656F803C0DA
:103A400001EA0C01F150D4F81CB159465CF0CEFDEE
:103A5000BBF5807F2ED024D8BBF1100F3FD037D8D4
:103A6000BBF1010F02D0BBF1040F34D14FF0080CB1
:103A7000336852462946484643EA0C0333604023E4
:103A8000C4F8E8305DF0A8F83B6843F010033B60F1
:103A9000BDE8F88F6FF00801CCE76FF008013C2318
:103AA000C8E7BBF5805F22D0BBF5803F1AD0BBF5DD
:103AB000806F10D108F11C064FF0080CD8E7402A9F
:103AC00015BF6FF400616FF008013C230023B1E7DC
:103AD000BBF1400FCAD03C364FF4006CC8E74FF43E
:103AE000006CC5E708F154064FF0080CC0E708F178
:103AF0001C064FF4006CBBE76FF00801042399E744
:103B00006FF40061042395E76FF4006192E700BF52
:103B1000ABAAAAAA2DE9F04F474D85B02B781BB967
:103B2000012005B0BDE8F08F444B5C6EFFF770F9E3
:103B300095F8F8350193002B00F0C781404B05F54F
:103B4000C065404E0027A3FB042300955B09A6FB3C
:103B500003263D4AF60802F2347806EB8606A3EB0C
:103B60004606D2F8483BC11A1346F2B203F6142AAD
:103B700008EB860689460392B9F1000F05DB009B2E
:103B8000D3F824314B4500F387814FF4B4732A4AAC
:103B900003FB072393F82037002B00F0BF80009D24
:103BA0002A48D5F85C11AB681A68CBB221F0FF0146
:103BB000103BA0FB030326481B09C35C0B44A989E7
:103BC0005C68D368A4B223EA0103C4F11604D3608D
:103BD000072C40F2A3801C4A0121D5F86451D2F889
:103BE0001C3A8B46AE4602970133C2F81C3A0022BB
:103BF0002868944614E0BCF1140F2BDC13F108077D
:103C000048BF03F117073B110CEB271C5F1E013166
:103C100002FA03F30BFA07F78C4247EA030219D3BF
:103C200003468C425EF8040FA0EB0303E3D8CCF10B
:103C300015034FF0150CE9E704000020D81C002400
:103C40001F85EB51CDCCCCCCFC100020ABAAAAAA8E
:103C5000C8090B08BCF1150F029F40F013819F4863
:103C6000C2F38423C2F3441100EB830300EB810110
:103C7000D3F8083DD1F8081D1B0243EA011302F0F6
:103C80001F01C2F3C43200EB810100EB8202D1F8C4
:103C9000081DD2F8082D0B4343EA023383EA1322AE
:103CA00082EA121202F00F020F2A40F0EB80C3F3F7
:103CB0000F134FF6FF72934200F0E480B3F5606F8C
:103CC00000F0EE80AAF80C3098F858200398824251
:103CD00010D0B168D8F80020521AC8F80020D8F8DF
:103CE0000420316B521AC8F804200022B2603263FB
:103CF00088F85800D8F800200132C8F80020B268CF
:103D00000132B2604FF6FF72934207D1D8F8043007
:103D10000133C8F80430336B01333363009C01373F
:103D200008F15C085C3620460AF1140AFFF744FEED
:103D300004F5B4730093019BBB427FF41DAF684947
:103D40000122002381F8182BC1F8483B6549D1F8BE
:103D5000083691F8D8261B6812F0020FD1F81C170C
:103D60001A6A0CBF0A4342EA81021A62019B012BC4
:103D70003FF4D6AE5B49D1F8703791F840281B6804
:103D800012F0020FD1F884181A6A0CBF0A4342EAF3
:103D900081021A62019B022B3FF4C2AE5149D1F855
:103DA000D83891F8A8291B6812F0020FD1F8EC1945
:103DB0001A6A0CBF0A4342EA81021A62019B032B72
:103DC0003FF4AEAE4749D1F8403A91F8102B1B684A
:103DD00012F0020FD1F8541B1A6A0CBF0A4342EAD0
:103DE00081021A62019B042B3FF49AAE3D49D1F83F
:103DF000A83B91F8782C1B6812F0020FD1F8BC1C7C
:103E00001A6A0CBF0A4342EA81021A62019B052B1F
:103E10003FF486AE3349D1F8103D91F8E02D1B6890
:103E200012F0020FD1F8241E1A6A0CBF0A4342EAAC
:103E300081021A62019B062B3FF472AE2949D1F828
:103E4000783E91F8482F1B6812F0020FD1F88C1FB2
:103E50001A6A0CBF0A4342EA81021A62019B082BCC
:103E60007FF45EAE204A52F8203C92F8B0001B6806
:103E7000D2F8F41080071A6A4CBF42EA81020A4362
:103E80001A624DE6164AD2F8183A0133C2F8183AC7
:103E9000AFB14FF6FF7317E7002005B0BDE8F08F14
:103EA00012494A7802EB420201EBC2023A44527CC8
:103EB0000D2A7FF407AF80228AF81E2004E72946E6
:103EC00058220B4862F040FFE3E719460122044BF9
:103ED000C3F8481B83F8182B22E600BFF0740A08C9
:103EE000FC1000200400002004100020D81C002436
:103EF000BC1B00202DE9F8432422D0F850510023A8
:103F00008168C0F8D02104462A6800F5A87622F01E
:103F100001022A602B606B60AB604279C0F8D83137
:103F200080F8CC31C0F8D031C0F86831C0F8D43155
:103F3000C0F870319302C0F8541103F48053BC49A7
:103F4000C0F8583113038D4203F40053C0F85C31BC
:103F50004FEA022303F48063C0F8603100F0AB81C4
:103F60002379D80703F0020100F14081002940F0D5
:103F70007181C4F8641194F8F8314BB1D4F87831F8
:103F800043F00803C4F878314FF40043C4F8883193
:103F900012F00802D4F8D03100F06E81002B00F04E
:103FA000AD8124233046C4F8D0312B6823F00103BF
:103FB0002B6053F033F9012817D0D4F87831002B57
:103FC00040F09F816B68304623F490436B60AB6890
:103FD00023F02203AB60AB6843F00803AB602B68AF
:103FE00043F001032B605CF015FF94F8048018F097
:103FF000010F6FD0D4F82C71002F00F06C810023DA
:104000004FF4807C04F13C09E7632366E36648468D
:10401000C4E91133C4E91433C4E91933D4F8343191
:10402000C4F8B8304FF48063E3644FF48033C4E9DC
:1040300016C35DF05FFF48464EF0A0F8D4F8D431C7
:10404000C4F8C891202B666741D1E368626998B2D1
:10405000EAB3B0FA80F14909C8B394F8CCC1BCF115
:10406000010F34D04FF0220CC4F8D811A4F8AC01E1
:104070000120C4F8D4C1DFF8D0C1C4F8A821C4F825
:1040800078C0DFF8C8C1C4F88C10C4F87CC0DFF871
:10409000C0C184F8CC01C4F888C094F870C08445CD
:1040A0000CD084F8700094F87100012800F0318180
:1040B0004FF4006384F87010C4F890301023C4F8F3
:1040C000D831002384F8CC312023C4F8D0317B6868
:1040D000C4F8443118F0020F00F08680D4F8305153
:1040E000002D00F0EC80D4F83821002304F1B4074F
:1040F000C4F8C0303846C4F8C830C4E92D52402254
:10410000C4F8BC204FF48062C4F8C4204FF480325D
:10411000C4E93333C4E93633C4E93833C4F8D420AE
:104120005DF0E8FE38464EF029F8002840F0A38004
:10413000404B4149414A8D4218BF9D42404801F1E0
:104140006001C4F8C4710CBF01230023C4F8EC6003
:10415000954208BF43F001033032854208BF43F067
:1041600001036030954208BF43F0010330328D42B5
:1041700008BF43F0010301F56871954208BF43F0A1
:10418000010302F55C72854208BF43F0010300F5AC
:104190006870954208BF43F0010330328D4208BF7A
:1041A00043F001036031954208BF43F00103303210
:1041B000854208BF43F00103954208BF43F0010365
:1041C00030328D4208BF43F00103954208BF43F0EF
:1041D00001033BB91B4BEB1AB3FA83F35B09002BCA
:1041E00000F0AF8000236B60BDE8F8830423C4F8BF
:1041F000643171B10C23C4F86431D3077FF5BBAED1
:10420000D4F878314FF4803143F00203C4F88011C0
:1042100028E0D3077FF5AFAED4F8783143F002033E
:10422000C4F878314FF48033C4F88031A3E600BF7E
:10423000000C0058100002402800024040000240DC
:1042400058000240B8040240ED2F09082130090847
:10425000253009080823D107C4F864317FF58BAEF7
:10426000D4F8783143F00103C4F878314FF40033C7
:10427000C4F87C317FE6FEE70BB194F8CC2124230F
:1042800084F8CC213046C4F8D0312B6823F00103E8
:104290002B6052F0C3FF01283FF4A7AED4F8783169
:1042A000002B32D16B68304623F490436B60AB68CF
:1042B00023F02A0392E60423C0F8743150E6D4F8C0
:1042C000DC311A6842F080021A601A6842F040023B
:1042D0001A60BDE8F883D4F8DC311A6842F48072C1
:1042E0001A609A6842F001029A601A6842F020024D
:1042F0001A601A6842F010021A60EBE684F8CC31BA
:104300004FE6304653F084F95CE6304653F080F9CE
:10431000C8E79BB2484605F1240151F093FB002801
:104320007FF4CCAE84F8CC012B6843F480732B600F
:10433000AB6843F00103AB60AB6843F04003AB6094
:10434000C5E66B6050E700BF38B50409013C082C96
:1043500018D80E4D00F00F0335F8140040FA03F2A0
:1043600012F0010210D00122254402FA03F3013BAE
:10437000184062F0F7FE95F8FC3C054A034402EB56
:10438000C30038BD002038BD104638BDF0740A089F
:10439000481D00242DE9F047984D05EB0013D3F894
:1043A000944C002C00F08F80B3F89E7C06464FEAB8
:1043B0000019384658F05EFF01227B0907F01F07FD
:1043C000023BBA40082B0FD8DFE813F0BF00C7004C
:1043D000CF00D700DF000900E700EF00B7008849F1
:1043E000CB6F23EA0203CB6705EB0903013693F891
:1043F000980CF6B2FFF7A8FF074610B11223C6715A
:10440000837105EB090393F8990CFFF79DFF824632
:1044100010B11323C671837105EB090393F89A0C4D
:10442000FFF792FF804610B11423C67183714D448B
:1044300050462E2195F89C2CFFF776F895F89D2C88
:1044400040460E21FFF770F895F89B2C2E21384638
:10445000FFF76AF823686B4A23F001039442236054
:1044600033D0694B9C423ED1654BD3F8902042F447
:104470008042C3F89020D3F8902022F48042C3F801
:104480009020E36843F00043E360A36823F4F073F3
:10449000A3602368DA0716D4A1685C4A5C4B0A4023
:1044A0001343A360E368DB0042D5E268594B134035
:1044B00043F0E863E360236823F400632360236D23
:1044C00023F001032365BDE8F0874D4BD3F8982016
:1044D00042F48052C3F89820D3F8982022F48052F6
:1044E000C3F89820CDE74C4B9C4213D04B4B9C42D9
:1044F00063D04B4B9C426ED1414BD3F8982042F491
:104500008012C3F89820D3F8982022F48012C3F8C0
:104510009820B6E73A4BD3F8902042F40042C3F813
:104520009020D3F8902022F40042C3F89020A8E70E
:10453000236843F480532360B7E73149D1F89C30B6
:1045400023EA0203C1F89C304EE72D49D1F8983098
:1045500023EA0203C1F8983046E72949D1F89030A0
:1045600023EA0203C1F890303EE72549D1F89430A0
:1045700023EA0203C1F8943036E72149D1F88030AC
:1045800023EA0203C1F880302EE71D49D1F88430B8
:1045900023EA0203C1F8843026E71949D1F88C30A8
:1045A00023EA0203C1F88C301EE71549D1F88830A0
:1045B00023EA0203C1F8883016E7114BD3F898209C
:1045C00042F40052C3F89820D3F8982022F4005205
:1045D000C3F8982055E7134B9C427FF452AF03F584
:1045E0000C33D3F89C2042F02002C3F89C20D3F86F
:1045F0009C2022F02002C3F89C2042E7D81C002413
:10460000004402580030014000380040E0FFBF8FF6
:1046100007000020FFFF39D8003C00400034014073
:10462000005001400014005808B51D20FFF78CFE13
:1046300008B183794BB11E20FFF786FE08B183795C
:1046400003B108BD5523C38008BD5523C380F2E7DD
:10465000F8B50E4C94F8F875A7B104F5C064C7F12D
:1046600009070925013D0FD0A6683079FFF76CFED8
:1046700094F8DC10F27908B1FEF732FFAF4204F58E
:10468000B474EFD10120F8BDAB68FFDE0400002058
:1046900008B553F06FFE1B20FFF756FE08B1292323
:1046A000C38058F0E3FD08B12923C3805AF092F883
:1046B0000B485AF07BF80B4B93F8F92C012A01D0E8
:1046C000012008BD084AD3F8D80FC3F8D42F5DF0F5
:1046D0001BFA0023054A184682F8233008BD00BFA4
:1046E00024040024D81C00245C04002400ED00E015
:1046F000F8B50446EFF31185502383F31288D0F800
:1047000030311B6803F001031BB1EDB285F3118852
:10471000F8BDD0F8D021D0F8D4110A4302F021021C
:10472000212AF2D0D0E90912914250D090B24BD850
:10473000194623691B1A9BB2A162002184F8E0117B
:10474000D4F8D0112029E0D1A1698918DDD0B3FABD
:1047500083F25209002BD8D094F8CC010128D4D090
:104760002120A4F8A6314FF0010CC4F8D821C4F8D8
:10477000D001D4F8C401D4F85061C4F8A011A4F851
:10478000A43184F8CCC160B31B4F90F834E0C76308
:104790001A4FE64502650764194FC7640AD090F8BE
:1047A000357080F834C0674515D04FF4006380F849
:1047B00034204365102100222023C4F8D81184F846
:1047C000CC21C4F8D031A0E7081A83B2B4E70123A2
:1047D00080F8E03199E706F1280251F033F900281A
:1047E000E8D100234022326284F8CC31B36843F030
:1047F0008003B36089E700BFC52F0908E92F0908C6
:1048000025300908BFF34F8F0549064BCA6802F4EB
:10481000E0621343CB60BFF34F8F00BFFDE700BFE3
:1048200000ED00E00400FA050021032008B5FFF7C1
:1048300081F872B6FFF7E6FF08B51D480023C0F8FF
:104840008430BFF34F8F436923F480334361BFF358
:104850004F8FD0F8803043F6E074C3F34E3CC3F37F
:10486000C90E4FEA4C1C0CEA0401734641EA8372FC
:10487000013BC0F874225A1CF8D1ACF1200C1CF199
:10488000200FF0D1BFF34F8FBFF36F8FBFF34F8F68
:10489000BFF36F8F4369002223F400334361C0F8F4
:1048A0005022BFF34F8FBFF36F8F72B6FFF7AAFF8F
:1048B00000ED00E003689B0AA3F58013522B57D844
:1048C00070B5384C23441B7D0D2B50D840794FF0E8
:1048D0004C0C354C4FF0020E86080CFB034C03EBDE
:1048E00083000EFA06FEDCF8DC5F03EB4000304488
:1048F000EE68002942D004EB800C46EA0E06CCF8A4
:10490000F414CCF80425EE60EFF31186502282F304
:1049100012882C2101FB0340D0F8F0244AB3111D6A
:10492000C0F81425214A03EB8300214D03EB40001E
:10493000800005441030024452F8040F08B10860AA
:10494000011DAA42F8D10022F6B20A6086F311884E
:104950002C2202FB0342D2F81425CAB14C2202FBDE
:104960000343D3F8DC2FD36843F00103D36070BD59
:1049700070470E4A01FB03212431D4E726EA0E06D4
:10498000EE6004EB8005C5F8F414C5F80425BBE718
:104990004C2202FB0344D4F8DC2FD36823F001033C
:1049A000D36070BDF0740A08D81C0024C82100240C
:1049B000E821002403689B0AA3F58013522B00D939
:1049C00070470F4A13441B7D0D2BF9D84FF04C0C48
:1049D00010B40C4C42790CFB03400223D0F8DC0FDE
:1049E000DA409340C26829B922EA03035DF8044B18
:1049F000C360704713435DF8044BC360704700BF4A
:104A0000F0740A08D81C002403689B0AA3F58013DD
:104A1000522B11D8094A13441A7D0D2A0CD840791B
:104A2000022307494FF04C0CD8400CFB0212834084
:104A3000D2F8DC2FDB431361704700BFF0740A0823
:104A4000D81C002401490248FCF7EAB9C821002417
:104A50000000014001490248FCF7E2B9C8210024E6
:104A60000000014002494FF08040FCF7D9B900BF77
:104A7000F421002401490248FCF7D2B92022002485
:104A80000004004001490248FCF7CAB94C22002446
:104A90000008004001490248FCF7C2B9782200240E
:104AA000000C0040F8B5164D164E2A69EB681A4006
:104AB0004FF00040B2FA82F3EAB120FA03F3012A80
:104AC0006FEA030302EA03012B610A46F2D1D6F82A
:104AD000F4758FB1013F0023BFB2C6F8F435D6F8A4
:104AE000F04534B123682046394698476468002C65
:104AF000F8D10022DCE7F8BDEF6ABFB2EFE700BFF4
:104B000000100040D81C002401490248FCF788B975
:104B1000FC2200240004014010B5064C064804F2B3
:104B20002461FCF77DF904F27C610448BDE8104083
:104B3000FCF776B9D81C002400040140001C00409A
:104B400001490248FCF76CB92823002400180040F2
:104B500001490248FCF764B980230024002000408A
:104B600001490248FCF75CB9AC2300240040014035
:104B700001490248FCF754B9D823002400440140FD
:104B800001490248FCF74CB90424002400480140C4
:104B9000800AA0F5801052280ED8084B03441A7DD5
:104BA0000D2A09D8064B4C2101FB0233D3F8DC2F28
:104BB000136843F001031360704700BFF0740A08E4
:104BC000D81C002410B590F83DE0BEF1020F76D05D
:104BD000144690F83D208446012A02D1022280F832
:104BE0003D200C2921D8DFE801F0072020202220D9
:104BF00020203A2020205200DCF824003449DCF840
:104C00000020C1633349C16490F8341001290CD0ED
:104C1000012180F8341090F83510012952D000227B
:104C20004FF4006380F834204365002010BDDCF8A9
:104C300028002749DCF80020C1632649C16490F8A8
:104C400034100129F1D0012180F8341090F835108A
:104C50000129E4D13832214650F0F4FEE5E7DCF8D2
:104C60002C001B49DCF80020C1631A49C16490F88C
:104C700034100129D9D0012180F8341090F8351072
:104C80000129CCD13C32214650F0DCFECDE7DCF8E6
:104C900030000F49DCF80020C1630E49C16490F870
:104CA00034100129C1D0012180F8341090F835105A
:104CB0000129B4D14032214650F0C4FEB5E75FFA75
:104CC0008EF010BD3432214650F0BCFEADE700BF7F
:104CD000652F09080D2F09081F4B984210B50ED0FB
:104CE00003F5806398420AD01C4A03F5804398423A
:104CF00018BF904203D003F5806398421BD151F056
:104D000065FE174B1749DC69DA69C4F3022CC2F35C
:104D1000022201EB0C0393F8EC3C03F01F03D84094
:104D20000F4B11491B69C3F3C03342EAC303CB5C89
:104D300003FB00F010BD51F049FE094B0949DC6945
:104D4000DA69C4F30214C2F302120B1993F8EC3CB3
:104D500003F01F03D840E3E700000140004001409A
:104D600000440258F0740A08A4090B082DE9F04F1A
:104D7000002393B0AD4C0193AD4BAE4FA3F6A856B4
:104D8000AB4D4FF00009AC4BD5F800A093F86A2367
:104D90004FEA9A23A3F58013522B00F2D0803344BC
:104DA0001B7D0D2B00F2CB80012A17F903B000F018
:104DB0000F81022A02D1BBF1080F3CD14FF000084D
:104DC0004146584611F0ECFB11F072FC90F800C01F
:104DD000BCF1000F18BFBCF1540F14BF4FF0010C11
:104DE0004FF0000C40F0E88008F104081FFA88F842
:104DF000B8F1100FE4D1019B002B00F0AB808B4A7F
:104E00000BE033441B7D0D2B0ED8FB565B450ED0BB
:104E100002F58672944200F0998091680B689B0AB3
:104E2000A3F58013522BECD900235B45F0D14B79CD
:104E300069799942ECD109F101091C35B9F1080FE2
:104E4000A1D1019B04F586740133042B019397D102
:104E50007A4A4FF0010B92F8F83502F58769013371
:104E60000493049B5B4567D0734B99F81020D9F8E5
:104E70000C6093F87E330192002E5DD06F4AD6F815
:104E800000A055686E48B288002D504402924FEA47
:104E9000902040F3AC80654A002405E0013402F51F
:104EA0008672AC4200F0A08011688142F6D15F4B5F
:104EB0004FF48672029D02FB0434019B0322C9F861
:104EC0000C6089F81030029BC9F81840B3FA83F7D8
:104ED000C7F11F035800C9F80430B27186F807B053
:104EE00002FA00F6A16C0122D4F854C0314302FA50
:104EF00000F002FA03F3A164216D0143D4F8AC0081
:104F000021654E490E7899B2002E00F04D8143EA9A
:104F10000C036365CAF81850FBF7C4F80BF1010BDA
:104F20002046FBF793F809F1200940F20113BBF189
:104F3000090F29F8043C94D113B0BDE8F08F013A71
:104F4000012A7FF678AF4FF0000B37E7BCF1000F76
:104F50007FF471AFA86800223A4904E001320C31B5
:104F6000102A00F086834B689842F7D152B250461F
:104F70006979FDF747FC344A4068002351680133E2
:104F8000884216D0102B02F12402F7D14FF0FF33E4
:104F900003EBC3032D4A02EB830393F8FC31002B90
:104FA0007FF449AFC9EBC909214B03EB8903A36027
:104FB00047E7DBB2013BEBE7019B002B7FF41FAF20
:104FC00009F101091C35B9F1080F7FF4DCAE38E7AF
:104FD000BBF1010F3FF4F2AE09F101091C35B9F143
:104FE000080F7FF4D0AE2CE7042C00F049824FF478
:104FF0008671124A01FB052211690591002900F012
:105000000483906001304FF054019C46C4B20D48B7
:1050100082F8101182F811416A1C08494A60059A09
:105020001168976803915179002216E00C00002066
:1050300098820A08B8090B08D02D0024040000202B
:105040000000FEA720010024E0010024000000244D
:1050500001320C30102A00F00C8343689F42F7D1D4
:1050600052B20398CDF818C0FDF7CCFB944B4FF427
:105070008672DFF87C8202FB05310022069B01323A
:10508000D0E90170C1E9077041464868874208D0FD
:10509000102A01F124013FF44FAF486801328742E2
:1050A000F6D1D2B28749013A02EBC20201EB820289
:1050B00092F8FC11089100297FF43EAF4FF48671FD
:1050C00082F8FD410793542401FB05F37E4882F8E2
:1050D000FC419A107D49069300FB02F201F56074D1
:1050E0007748C2EBC20C02EBC202184401EB4C1130
:1050F00004EB4212C0F80CA0C0F8B410C0F8FC20B9
:105100003322C0F8B8208C22C0F80021704A0398DE
:10511000D418FFF7E1FD079B062B00F0B881072BA1
:105120006C496D4B6D4A18BF1A466D4B18BF0B4644
:105130004FF48671DDF80CA0B0FBF3F3B0FBF2F294
:10514000013B5F48013A01FB05019BB2A1F8BC207D
:10515000A1F874302366069B03F1580100F108039F
:10516000504619440023A4F858306366E3655BF0A9
:10517000BBFBDAF8003043F08003CAF80030059B2F
:105180005B791A4607930C2A1CD8DFE812F002025A
:105190001B001B001B00DC011B001B001B00BA01D5
:1051A0001B001B001B009501C7F12F072D0402FAFD
:1051B00007F3324643EA0C036365CAF81850FAF75E
:1051C00071FFABE63E4A4FF4867303984FF0000A36
:1051D00003FB05230222CDF830A059690368099129
:1051E00023F00103CDF83CA0CDF844A00360602378
:1051F0000A934FF48073109301230B930A23CDE994
:105200000D320AAA5BF0F2F90999B1F5807F00F03E
:10521000278240F23F81B1F5805F00F00D82B1F549
:10522000803F00F00382B1F5806F15BF4FF400633B
:1052300008234FF03C0A4FF0040A039A183252F840
:105240000A100B4342F80A30059B1879002840F0F9
:10525000CA81039A136843F0010313600023D8F84E
:1052600004200133974200F0BA81102B08F1240882
:10527000F5D14FF0FF33134A03EBC30302EB830373
:10528000D3F8E001174B984214BFA120A02057F09B
:10529000F1FF079A0C2A00F2A081134B03EB4203A3
:1052A000B3F8887E4FF48673054A104803FB052344
:1052B000DDF80CC000F532611F83002321E000BF40
:1052C00004000020000000246B4CA407C04101240E
:1052D0000C000020D0DD0600449508001055220087
:1052E00040771B0000000240F0740A08FC10002008
:1052F000E0010024944500F09D810133042B00F06F
:10530000BB8151F83320002AF4D1D0F81C2B013294
:10531000C0F81C2B00EBC300039ADB00C0F8202B65
:105320001944089823469022B1F804C047EA0C07B4
:105330008F800027C349FDF7D9FA4FF48673C24A1C
:1053400040214FF4403CC14803FB052A4FF48052F2
:10535000DAF81C502B6843F010032B602B6843F0E5
:1053600014032B60C4E91F77C4E92777C4E92977C0
:10537000DAF82030A167E9B2C4F894300793103905
:105380004FF48063C4F898C0A0FB01014FF4804C37
:10539000C4F88430DAF8B8000909069BC4F8900014
:1053A00025F0FF00DAF80C80C4F8882008F1180214
:1053B0000591039008F11008226703F17002A44BD5
:1053C0001A44DAF8B430C4F88CC063675BF004FCAC
:1053D000D5F800C0069BC4F820C0D5F814C003F16E
:1053E000B8029B4BC4F824C0D5F804C01A44079BEC
:1053F000C4F828C0D5F808C00599C4F82CC0D5F861
:105400000CC0C4F8DC304FF48063C4F8C870C4F832
:10541000CC304FF40033C4F830C0C4F8E030039807
:10542000C4E93077C4E93977C4E93B774FF40067C2
:10543000DAF80031C4F8B880C4F8D0704FF480476F
:10544000C4F8D830DAF8FC30C4F8D470C4F8BC30F2
:105450005BF0C2FB2B68D6F800A063636B69A363A3
:105460006B68E363AB682364EB6863642B6843F0A9
:1054700010032B602B6843F014032B60B5881CE5E8
:105480000323744A82F87F3313B0BDE8F08F724A69
:10549000724B4DE6102900F0E98000F2BD80012931
:1054A00000F0E280042915BF4FF4006308234FF099
:1054B0003C0A4FF0000AC0E603984FF48672624936
:1054C0004FF0020A036802FB05124FF4805123F0EB
:1054D000010351610AAA036000230C930F931193F7
:1054E00060230A934FF48073109301230B930A23D4
:1054F000CDE90D3A5BF07AF84FF0040A4FF40063FF
:105500009BE603984FF486724F494FF0020C0368F4
:105510004FF0040A02FB05124FF4807123F00103DF
:10552000516160220360002310910C930F9311933B
:105530000123CDE90A230A230AAACDE90D3C5BF039
:1055400055F8082379E603984FF486723E494FF0E8
:10555000000A03684FF0020E02FB0512102123F02F
:105560000103CDF830A051610AAA03606023CDF891
:105570003CA00A934FF48073CDF844A0109301230C
:105580000B930A23CDE90D3E5BF030F84FF4006336
:1055900053E603984FF486722B494FF0000A0368D4
:1055A0004FF0020E02FB0512012123F00103CDF89A
:1055B00030A051610AAA036060230B910A934FF453
:1055C0008073CDF83CA010930A23CDF844A0CDE918
:1055D0000D3E5BF00BF808232FE6002762E6DBB2F6
:1055E0000893013B47E6FEF7AFFE824638B1059BC4
:1055F0000221DA79FDF774FF5423AAF80630039AE2
:10560000536C43F40043536423E60223114A82F8A7
:105610007F3313B0BDE8F08F402915BF4FF400630E
:1056200008234FF03C0A4FF0000A06E608234FF02B
:105630003C0A02E6DB0073E64FF400634FF0040A15
:10564000FBE500BF0100000004000020ABAAAAAAED
:105650000C000020D02D0024882A1100A0BB0D00D2
:1056600008234FF0040AE8E50823E6E54FF4006359
:10567000E3E500235B68FFDE00239B88FFDE00BFBD
:1056800008B9002070472DE9F04F00228FB02F217C
:10569000044611F063F80646C8B190F80590A74F8C
:1056A000D0F800A0A7F86498FDF7D8F878B1D0E951
:1056B000015301935DB1DFF8C082002342464146A9
:1056C000486801332431854205D0102BF8D10020E1
:1056D0000FB0BDE8F08FDBB29949013B03EBC30388
:1056E00001EB83019B0091F8FCB1BBF1000FEED1FF
:1056F0001A442F23C7F818A850469383FFF7ECFAF3
:10570000904B984280F0F980012303935B4650460A
:105710000293FFF7E1FA029B8B490022C7F81C387D
:10572000039BC7F82828C7F82028B0FBF3F31B0A0F
:105730008648A1FB0331864B0A090909A0FB020236
:10574000C7F824185208A3F882235200A3F8802334
:1057500097F8552802F0FF01002A00F0DC800222B1
:1057600050467C4987F8552851F006FC0122204616
:1057700087F8602887F8562887F8572887F8582828
:1057800087F8592887F85A2887F85B2887F85C2813
:1057900087F85D2887F85E2887F85F2887F85528FE
:1057A000FEF7D2FD6A4BC3F8840330B12F21C180CC
:1057B0004E21F279FDF794FE654B019A00214FF4DA
:1057C0008064B9F10C0FC3F89413C3F8A413C3F8A1
:1057D000AC13C3E9E252604AC3E9ED11D2F8D80034
:1057E00040F00100C2F8D800D2F8D80000F0010063
:1057F00005900598D2F8D80040F00200C2F8D80011
:10580000D2F8D82002F002020692069A4FF0400227
:10581000C3F890234FF48052C3E9E6424FF480422C
:10582000C3F8A0234FF40032C3F8A8234FF00302BB
:10583000C3F8B02372D8494A02EB4902B2F8A44E29
:10584000A24608344649474AC3F8C01307EB84030D
:10585000C3F8182843460022596824338D4260D08B
:105860000132102AF8D14FF0FF33354A03EBC3035E
:1058700002EB8303D3F8E0013B4B984214BFA12015
:10588000A02057F0F7FC0023D8F80420013308F1DA
:105890002408954249D0102BF6D107EB84075846CF
:1058A000534660223149FDF721F8D7F818084CF02B
:1058B00065FC00287FF40BAFB47960210C904A4658
:1058C000630007910D9007A903F0020308900B9065
:1058D0000993E300224803F008030A9356F084FF7B
:1058E00000287FF4F4AEA30749461D4820D551F0A7
:1058F0004BFCB0FA80F04009EAE65046FFF7ECF9BD
:105900001B4B1C4A0344A2FB03239B0D013B9BB290
:105910005A1C0392FBE687F8541820E78A460C4687
:105920008FE7531CDBB2013B9FE75FFA83FBB4E7D1
:1059300051F096FAB0FA80F04009C9E6D81C00246C
:1059400000000024006CDC02598B4F01ABAAAAAA0C
:10595000D02D0024F424002400440258F0740A08D6
:10596000F02400245831002400000240D502000039
:1059700000366E01819F5E16E0010024830AA3F5C4
:105980008013522B00D970472DE9F0410F4C23446E
:105990001E7D0D2E18D80E4C4FF04C0801391546BF
:1059A00008FB064789B2C7F8E81FFFF795F907F526
:1059B0007E61B0FBF5F2013AD7F8DC0FC7F8E02FB3
:1059C000BDE8F04151F0D8BABDE8F081F0740A08A2
:1059D000D81C0024830AA3F58013522B7DD82DE90F
:1059E000F0437B4D85B02B441F7D0D2F72D84C2387
:1059F000DFF8F881044603FB07F908EB0905D5F841
:105A0000DC3F834266D001391646C5F8DC0F89B207
:105A1000C5F8E81FFFF760F909F1080308F6DC7123
:105A200000220B44C5F8E42FB0FBF6F00138C5F8AE
:105A3000E00FC3E9022241F21903EB5C03F0FF021D
:105A4000002B4BD04C25022341F2190605FB071110
:105A500005FB07850431D5F8DC9FAB55484651F06E
:105A60008BFA012341F22402AB5441F21A02AB54E7
:105A700041F21B02AB5441F21C02AB5441F21D0235
:105A8000AB5441F21E02AB5441F21F02AB5405F578
:105A90008152137041F22102AB5441F22202AB5405
:105AA00041F22302AB54AB554A4B9C421AD0B4F19D
:105AB000804F17D0A3F57C439C4213D003F580633D
:105AC0009C420FD003F580639C4263D003F578437A
:105AD0009C425FD005B0BDE8F083704741F21803E7
:105AE000EA54AFE74C2341F2180103FB07835A5CE9
:105AF000012AEFD041F2190002221A54364AD9F88D
:105B000008402240C9F8082001221A5400225A54A1
:105B100000224C23022103FB07830392CDE90122DB
:105B200041F2190299542B49D9F804208945D9F832
:105B300008302AD001F58061894526D022F0700214
:105B4000C9F80420254A91450DD0B9F1804F0AD0FB
:105B5000234902F50062914518BF894503D002F53B
:105B60004062914503D123F08003C9F808304C23EB
:105B700041F21902012103FB0783995441F21802F3
:105B80000021995405B0BDE8F08316491140C9F8C9
:105B90000410E8E74C2341F2180103FB07835A5C29
:105BA000012A97D041F2190002221A540A4AD9F860
:105BB00008502A40C9F8082001221A5400225A54D9
:105BC000094B9C42A4D003F578439C42A0D081E7C6
:105BD000F0740A08000001408800CEFF0004004075
:105BE000000800408FFF0FFF000C0040D81C00246D
:105BF0002DE9F0410468A30AA3F58013522B04D8C1
:105C00002D4D2B441E7D0D2E01D9BDE8F08120467F
:105C1000FFF7E0FE4C22294B02FB063341F219024A
:105C2000995C012927D00023254902E00133112B7B
:105C300032D051F833209442F8D105EBC305012648
:105C4000204F95F8624A314604F01F05204657F070
:105C500079F91B2C4FEA541806FA05F547F8285035
:105C600022D02E2CD1D131462C2057F06BF94FF495
:105C700080537B60C9E702219954D3F8DC2F124B83
:105C800091680B40062BCED0B3F5803FCBD0136884
:105C900043F001031360C6E70121002057F052F9D9
:105CA000084B01221A60B0E73146192057F04AF933
:105CB0004FF000733B60A8E7F0740A08D81C00247A
:105CC0004C7F0A0800E100E007000100F8B5134C22
:105CD00094F8B63803F0FF05002BF9D1104B0126DC
:105CE00093F8003484F8B66803B9F8BD0D4AB4F8E7
:105CF000B478138E34320C483946FEF763FF0346FE
:105D000010B184F8B658F8BDD4F868483246394620
:105D100005486362BDE8F8405DF0DCBED81C002495
:105D2000D02D002480F400244025002437B590F8BD
:105D300067380446032B2FD10023204D8DF8073000
:105D40009DF8073094F868289A4201D803B030BD16
:105D50009DF8073005EBC30393F808348BB181F04D
:105D6000010383B19DF8073005EBC303D3F80404A6
:105D7000FDF7AAFB9DF807300133DBB28DF8073041
:105D8000DEE70B46EDE79DF8073005EBC303D3F8DC
:105D90000404FDF79FFBEDE7D0E910039B7903F0C6
:105DA0000103994204D003B0BDE83040FDF78CBB3D
:105DB00003B0BDE83040FDF78DBB00BFD02D0024FF
:105DC00038B5044600790D4650B1FEF7BDFA08B16A
:105DD0000323C380E2792946BDE83840FDF7A4BB20
:105DE00038BD10B504462221FFF7EAFF2046FEF732
:105DF0000BFE20460121BDE81040FEF7DBBD10B5CB
:105E000004460121FFF7DCFF00212046BDE81040D9
:105E1000FEF7D0BD38B510F8133CA0F66C041BBBE0
:105E200094F858388BBBD4E909239A421CD05A1CE9
:105E3000A169A262CB5C21695B008A4228BF002273
:105E400043F40073A262A4F85C380A2384F85A3839
:105E5000012384F8583894F86738012B01D0042BBB
:105E600002D1606CFFF7CBFF94F85438002B6DD152
:105E700094F855380133DBB2092B84F8553825D115
:105E80002046BDE83840FAF7E5B994F95A586DB1A3
:105E9000B4F85C18013D20464B0801F00101A4F85C
:105EA0005C38FFF743FF84F85A58DDE7D4E909234B
:105EB00084F858589A42D7D194F86738012B01D00A
:105EC000042BD1D1606CFFF78CFFCDE70A2B3DD1BD
:105ED00094F857382BB9B4F85E3843F00103A4F8AE
:105EE0005E382379D9070AD5B4F85E08820501D453
:105EF000C30718D4B4F864380133A4F86438012215
:105F0000002384F8542894F8572884F85538012A37
:105F10001CD16179606C84F8573801F00101BDE84B
:105F2000384056F027B9E36AC0F3470013B1216B3C
:105F30009847E4E7E3696269D054E369E2680133B2
:105F4000B3FBF2F102FB1133E361D8E738BD2DE971
:105F5000F84310F8133CA0F66C047BB1B4F8603839
:105F600001339BB2082BA4F860381BD90021606C68
:105F700084F85918A4F8601856F0FCF8374F97F8D1
:105F80004484B8F1000F03D101212046FFF7CEFE73
:105F900094F858384BBBD4E909239A4204D1002322
:105FA00087F84434BDE8F883B8F1020F12D808F13D
:105FB000010814BFFF237F2387F84484A4F85C38CA
:105FC0000823606C84F85A38012384F85838BDE8F7
:105FD000F84314E75A1CA169A262CB5C2169DBB2C9
:105FE0008A42EBD30022A262E8E794F95A685EB3D2
:105FF000B4F85C9897F8455419F001010BD0012DC5
:1060000001D8012103E0AB1E012B09D80021204655
:10601000FFF78CFE04E015F0FD03F2D0012BF6D063
:106020000135EDB2032D87F84554BBD9013E4FEA47
:106030005909002376B2A4F85C9887F8453484F8AF
:106040005A68002EA7D0ADE7D4E909239A42A9D116
:10605000606C84F85868BDE8F843C2E6D02D00248F
:106060002DE9F043BFB0BFF35F8FA24A0020516A11
:106070000346044621F4803151620146C2F894007F
:10608000C2F898300133C2F89C10112BC2F8A0104E
:10609000F6D10523C2F89430536A43F48033536237
:1060A000BFF34F8FBFF36F8F9348944A9449121AEE
:1060B00060F04AFE9348944A9449121A60F044FEF4
:1060C000934BDA6D042A00F0FB8005D8012A00F01A
:1060D0007283022A00F08583864A00238D4C0120BA
:1060E000D2F888108C4E41F470018C4DC2F88810A3
:1060F00020602361216841F0800121602168014313
:106100002160216841F480312160216841F480518F
:106110002160A361E3612362A362E362236363639B
:10612000A363E36323646364216821F48021216015
:106130007B492366C1F808014FF000614FF6FF006C
:10614000784B9160D16801400B43D36050F01CFC48
:10615000A36902460F20C3F30323A169334493F8D4
:10616000EC3C03F01F0322FA03F3C5F8A4344BF010
:10617000D9FF6D4AD36813F0040FD36840F0A280B2
:106180006A4B0021684A0591D96A21F00101D96260
:10619000DB6A03F001030593936943F44043936181
:1061A000936903F440430593059B93699B04FCD5D5
:1061B0004C2200210EA85E4C60F024FE5D4A42F2A3
:1061C00003031268B3EB124F4FF000030893A4F1DE
:1061D000140308BF1C46E268002A4DD0534B5249B5
:1061E000D86A20F00100D862DB6A03F0010308934B
:1061F0008B6923F4404313438B618B6903F4404361
:106200000893089B484A93699F04FCD5414B4FF47F
:10621000403749480321D3F8E02042F08002C3F818
:10622000E0200122D3F8E03003F080030793079BBE
:1062300087610D9B0091019300235BF00FFD02230A
:1062400022690EA8CDE91733A3781E920122199373
:10625000A3881A93A3791B93E3791C93237A1D9344
:1062600000231F934FF48033CDE90E2350F0D4F870
:1062700003283BD098B1FEE72B4A2C4B916941F49F
:1062800040419161926902F440420892DA6A42F018
:106290000102DA62DB6A03F001030893B1E7274BDE
:1062A0001A6812F00E0F4DD11A6822F00F0242F058
:1062B00002021A601B6803F00F03022B42D0FEE7B4
:1062C000DC6509E723F007031D4C43F00203D360AC
:1062D000D4F8E81A06E0D4F8E83A5B1AB3F57A7F06
:1062E0003FF64EAF53689804F5D549E772B6FEF70E
:1062F00089FA00BF00ED00E000000000284B00001C
:1063000080A50B08000000200400002059190C088B
:106310000040005800440258F0740A0800000024AD
:10632000008000510003FA0500480258000400589C
:10633000900400240010005C001C02580020005251
:10634000D81C00246E4A936903F070033F2B05D8D4
:10635000936923F0700343F040039361684AD36963
:1063600003F070033F2B05D8D36923F0700343F08B
:106370004003D361624AD36903F4E063B3F5806FED
:1063800005D2D36923F4E06343F48063D3615C4AAC
:10639000136A03F070033F2B05D8136A23F07003D0
:1063A00043F040031362564B9A69100705D49A696B
:1063B00022F00F0242F008029A61514A936923F4D5
:1063C00070639361136899017FF579AF136941F2A6
:1063D00088304C4C23F0070343F003031361D4F8D7
:1063E000E81A05E0D4F8E83A5B1A834200F29B8190
:1063F000136903F03803182BF4D1936903F00F03EA
:10640000082B05D9936923F00F0343F00803936128
:106410003D4A136803F00F03022B0BD9136823F0D6
:106420000F0343F002031360136803F00F03022B02
:106430007FF445AF324A936903F07003402B05D9CE
:10644000936923F0700343F0400393612C4AD369AE
:1064500003F07003402B05D9D36923F0700343F098
:106460004003D361264AD36903F4E063B3F5806F38
:1064700005D9D36923F4E06343F48063D361204AF0
:10648000136A03F07003402B00F245811C4F50F05B
:106490007BFA0346D5F8A804BA69B969C2F30322A6
:1064A000164496F8EC2C02F01F02D340C5F8A43431
:1064B0004BF038FE002840F07D8110231590179096
:1064C0000EA80E934FF0A8FF002840F023813B68F0
:1064D0000E4A43F080033B60D7F8F43043F00203E8
:1064E000C7F8F430D7F8F43003F002030493049BA8
:1064F000136A43F001031362054BD4F8E81A0CE069
:1065000000440258D81C0024002000520004005807
:1065100000E20400013B3FF4E9AED4F8E82A9142DE
:10652000F8D0D4F8E82AD4F8E83A9B1A0A2BFAD91A
:10653000AF4C4FF480224FF440130EA80E924FF050
:1065400000082F935AF03CFDD4F8EC3041F20302DE
:10655000A849032643F002030EA8C4F8EC30D4F88F
:10656000EC3003F002030393039BD4F8943043F020
:106570000203C4F89430D4F8943023F00203C4F832
:1065800094300B689C49B2EB134F9C4B9C4A28BF3C
:106590000A465A601A6822F47C5242F400521A6089
:1065A0001A6842F060021A600E96CDE92B885AF004
:1065B00007FD4FF4E0430EA8CDF8E4800E93CDE93B
:1065C00025885AF0FDFC18230EA8CDF8B8800E934C
:1065D000CDF8CC805AF0F4FC4FF400230EA80E93B3
:1065E0004FF4003336935AF0EBFCD4F8E0304FF41C
:1065F0008071844843F00103C4F8E030D4F8E030FF
:1066000003F0010309934346099A0222CDE9006889
:106610005BF024FB23694FF400717B4823F0FE7389
:1066200043F088732361D4F8E03043F00403C4F8E6
:10663000E0304346D4F8E02002F004020692069AC5
:106640000222CDE900685BF009FB236923F07E4359
:1066500043F0FC43236150F097F96C4B6C4A414680
:10666000C5F8A4041846D21A60F0CCFB69486A4AFF
:106670006A49121A60F068FBBFF35F8F684D4646A7
:10668000684C01276B6A23F480336B62C5F89480F1
:1066900023E0002946D0D4F80090637A103414F82F
:1066A000060C1B0643EA007343EA410314F8051C79
:1066B00043EA814314F8041C43EA414314F8031CE1
:1066C000C5F89860013643EA0143C5F89C90032E53
:1066D00043F00103C5F8A03026D06368217A002B6F
:1066E000D7D0D4F800900029D7D129F01F01A3EB0F
:1066F0000108B8F1200F38BF4FF02008404660F085
:1067000061FB431E014607FA03F0804508BF1946A6
:10671000C9B2C2E7FEE7136A23F0700343F04003F7
:106720001362B3E6FEE7CAE50523C5F894306B6A49
:1067300043F480336B62BFF34F8FBFF36F8FBFF3B0
:106740004F8FBFF36F8F0022C5F85022BFF34F8FDA
:10675000BFF36F8F6B6943F400336B61BFF34F8FEF
:10676000BFF36F8FC5F88420BFF34F8FD5F88050EB
:1067700043F6E0762A49C5F34E34C5F3C9056401F2
:1067800004EA06002B4640EA8372013BC1F860220E
:10679000F9D2203C14F1200FF2D1BFF34F8F4B6997
:1067A00043F480334B61BFF34F8FBFF36F8F3FB024
:1067B000BDE8F08383E50E4A02201B49D865D2F874
:1067C000F4300343C2F8F430D2F8F43003400E93AF
:1067D0000E9AD1F8003883F30888D1F80438984726
:1067E000FEE704210320FDF7A5F872B6FEF70AF8CC
:1067F000004402580010005C7FBB2200008400406F
:106800007FBB2230000002580008025800F4002428
:1068100080F40024A0F2002400F400245D190C0888
:1068200000ED00E0AC0400240090F01F10B4EFF382
:106830001182102383F312880B4B4FF0E0200024C9
:10684000D2B2596E0131596681699966C3F8C04860
:10685000016982F31188D3F8E82A5DF8044B01320C
:10686000C3F8E82A704700BFD81C002410B4EFF327
:106870001181102383F312884FF0E0229469136989
:1068800013F4803F0C4B03D00120C3F8C008946977
:10689000586EC9B2D3F8C02881F311880244D96E6A
:1068A0004FF47A7000FB01F31B1B5DF8044BB3FB44
:1068B000F1F300FB02307047D81C00242DE9F047AB
:1068C000DFF89080FCF7A4FA4FF4867900210646A1
:1068D000D8F804501D4F002D2DDD00231C4609FB68
:1068E0000382013392F80521AB4244EA0204F6D157
:1068F00021435FFA81FA7B68C3F30803C3B9EFF35E
:106900001183ABB9F9F700FD801BB0F5FA6FCCBF6E
:10691000002104F001010029DDD1BAF1000F04D0FB
:106920000B4B93F83F2C542A08D05046BDE8F08713
:10693000FFF79CFFE8E78A460024DCE7B3F8442C25
:1069400050460132A3F8442CBDE8F08700ED00E08A
:10695000D81C002404000020454B5B68C3F30803E7
:106960002DE9F0430546002B5ED1EFF31183002B98
:106970005AD1404B4FF0E0245A6EA069596E8A42BA
:10698000FAD1996E8842F7D8DE6E4FF47A7101FB26
:1069900006F4241AB4FBF6F401FB0244344E10272B
:1069A0004FF0E02C4FF47A7E4FF001087268C2F38A
:1069B0000802CAB9EFF31182B2B95A6EDCF81800B6
:1069C000596E8A42F9D1996E8842F6D8D3F86C9004
:1069D0000EFB09F1091AB1FBF9F10EFB0212121BB1
:1069E000AA42E3D3BDE8F083EFF3118287F3128864
:1069F000DCF81800DCF81010C90303D5C3F8C08810
:106A0000DCF81800D3F86490D2B2D3F8C01882F33F
:106A100011884944D3F86C900EFB09F2121AB2FBAC
:106A2000F9F20EFB0122DAE7EFF31181102383F371
:106A300012884FF0E0229669136913F4803F0D4BE2
:106A400003D00120C3F8C0089669586EC9B2D3F8C4
:106A5000C02881F311884FF47A710244D86E01FB8B
:106A600000F4A41BB4FBF0F401FB024496E700BF62
:106A700000ED00E0D81C00242DE9F0473A4B471EFA
:106A80003A4D10264FF0E0204FF47A7C4FF0010889
:106A90006A68C2F30802002A52D1EFF31182002A79
:106AA0004ED15A6E8469596E8A42FAD1996E8C42DF
:106AB000F7D8D96E0CFB01FEAEEB040EBEFBF1FE67
:106AC0000CFB02EE6A68C2F30802E2B9EFF311822E
:106AD000CAB95A6E8469596E8A42FAD1996E8C424B
:106AE000F7D8D3F86C900CFB09F1091BB1FBF9F155
:106AF0000CFB0212A2EB0E02B2F57A7FE2D3013F49
:106B0000C6D2BDE8F087EFF3118286F3128884695C
:106B10000169C90302D5C3F8C0888469D3F864A0A9
:106B2000D2B2D3F8C01882F31188D3F86C905144D4
:106B30000CFB09F2121BB2FBF9F20CFB0122D9E7A4
:106B4000EFF3118186F3128884690269D20302D5BA
:106B5000C3F8C0888469D3F864E0C9B2D3F8C02808
:106B600081F311887244A4E7D81C002400ED00E0F2
:106B7000154C08B5D4F8483494F84E04ABB9142039
:106B8000FFF77AFF00BFD4F848345BB1196894F876
:106B90004E249B8809690B4012B91BB1FDF744FED6
:106BA000002BFBD0F9F7B2FFECE719689A880B6964
:106BB000134020B1002BE2D10B691340FAE7002B00
:106BC000DDD00B691340FAE7D02D0024704700BFD9
:106BD0000246074B02209A4208D801335B08400066
:106BE0009A4280B202D2FF28F8D97047704700BF9E
:106BF0007FF0FA02CB0700D5704710B50446FAF7CC
:106C0000B5FD94F82830012B00D010BD616A024810
:106C1000FFF7DEFF888010BD00E1F5052DE9F04F9C
:106C2000D0F8E85183B081601746B5491E46044646
:106C30000160D5E90E23C0E90532B5F84230C360E2
:106C4000B5F8403003616B68C0F8DC31C0F85031F2
:106C5000AC4BC0F8E431288E002840F0258195F92E
:106C60000080B8F1280F00F027815FFA88F9B9F1A8
:106C70003A0F05D8A44B434493F9F03E002B60D162
:106C80004FF0010894F8EE0184F8E081FDF75CFB19
:106C9000022394F8EC9184F8F93194F93830142BEC
:106CA00000F01481A3F13302D2B2072A40F2CB8064
:106CB000282B40F05E814FF05A0B16F0080394F831
:106CC000EDA194F8EF2100F0CA80002800F0D380F5
:106CD00016F0400306F0110140F00081B7060BD416
:106CE00006F00103884EC3F10203DBB206EB830317
:106CF000D3F82C3F5B01DBB2002980F806B080F8A6
:106D000007800CBF1A210A211943FCF7E9FBD4F8CC
:106D10002C31002B40F0C48095F8341095F83200E7
:106D2000890956F00FF995F832300122774903F0BE
:106D30001F005B098240204641F8232003B0BDE8D4
:106D4000F08F404603F1FF3A14F092F9B8F1140FB6
:106D50004FFA8AFA00F0BE80A9F13309B9F1070FA2
:106D600000F20B81A8F132084FF00B09DFF8ACB14B
:106D700043000BEB400090F95024511C0FD05FFAF8
:106D80008AF10420CDE90023FBF7F4FCDDE90023C0
:106D900028B14168C4F830118168C4F838119B44A7
:106DA0009BF9513401330BD05FFA8AF10520FBF7D0
:106DB000E1FC28B14368C4F82C318368C4F834314D
:106DC000D4F8300148B1524B0022596801322433C3
:106DD000884200F0A580102AF7D1D4F82C010028B1
:106DE0003FF44EAF4A4B00215A68013124339042A0
:106DF00007D010293FF444AF5A6801312433904240
:106E0000F7D1C9B2434B09F101095FFA88F801399A
:106E100001EBC10103EB810393F8FC21002A7FF40D
:106E20002FAFD3F8E00183F8FC9183F8FD813A4B52
:106E3000984214BFA120A02056F01CFA6B6824339E
:106E4000C4F84C311CE7A3F1320816F008034FF0E8
:106E50000B0B94F8EDA194F8EF217FF436AFB9074E
:106E600009D540B1310680F806B080F8078037D4E4
:106E70000221FCF735FB4846FDF766FA58B1FA07E0
:106E800009D50BF1010B5246022180F8078080F8EA
:106E900006B0FCF725FBD4F82C31002B3FF43CAFB7
:106EA000204603B0BDE8F08F56F0E4F995F9008074
:106EB000B8F1280F7FF4D9AE40464FF05A094FF091
:106EC000080A4FF0010814F0D3F84FE74FF0000B19
:106ED000D846F2E64FF00009C84647E740230BE7E3
:106EE000D4F850611A464FF0010C2021336823F08A
:106EF0000803336084F8F9C1FCF7F2FABBE700BF7E
:106F0000B0830A08AD380408F0740A0800E100E014
:106F1000E00100240000002400000240D02D0024E5
:106F20005FFA82FA174B5FFA88F10AF1FF3202EB3F
:106F3000C20203EB820393F8FC21002A7FF44DAFD9
:106F4000D3F8E00183F8FD1183F8FC910E4B9842D1
:106F500014BFA120A02056F08DF92346504695F885
:106F600033200A49FBF7C2FC6B682833C4F8483168
:106F700033E74FF00008C3469FE64FF00008C146D4
:106F8000F4E600BF0000002400000240450F0408A2
:106F90002DE9F0470546086888B00C464FEA902C6A
:106FA000BDF84080ACF5801C9DF844A0BCF1520FA8
:106FB00058D819462E4B63441E7D0D2E52D806EB31
:106FC000C6032C4F06EB430307EB8307FEF702FDD6
:106FD00094F80590A379BAF1000F01D083F0010372
:106FE0005A004FF48071DB00384602F00202CDF8FF
:106FF000088003F0080303924A4604936023019338
:107000004FF40073CDE90613002301A9059355F051
:10701000EBFBA379384649469F0726D44FF020FF63
:107020004C22154B02FB063341F21902995C0129EF
:107030000FD102219954D3F8DC2F104B91680B40EB
:10704000062B06D0B3F5803F03D0136843F001034D
:1070500013602168637901F1340269600021D0185E
:107060002860D15008B0BDE8F08750F08DF8D7E720
:10707000F0740A08B42C0024D81C00240700010076
:1070800010B4284C94F8303763B3226D904234D05A
:10709000012B27D0D4F82C21824236D0022B21D0CC
:1070A000D4F80822904232D0032B1BD0D4F8E4222B
:1070B00090422ED0042B15D0D4F8C02390422AD071
:1070C000052B0FD0D4F89C24904226D0062B09D053
:1070D000D4F87825904222D0072B03D0D4F8542638
:1070E000824210D0DC22591C02FB034284F8301784
:1070F000106518465DF8044B70470023DBB25DF85D
:10710000044B184670470723F8E70123F6E70223EC
:10711000F4E70323F2E70423F0E70523EEE7062371
:10712000ECE700BFFC1000200548D0F8903723B1F1
:10713000DB6A13B100F5F26018470248704700BFE0
:10714000D81C002428840A0870B5104C4FF0000C9D
:10715000234693F800E00633864512D00CF1010C6B
:10716000BCF1060FF5D10A4ED6F88854052D07D08C
:107170000CFB05430135C6F88854187059809A8075
:1071800070BD062303FB0C43F7E700BF3432002435
:10719000D02D002438B5174CD4F88C341B8843B953
:1071A000154D002384F8973485F88837C5F884375F
:1071B00038BDD4F88824002AF2DDD4F89014012ACE
:1071C000488806D001230C4DA4F8940484F8963422
:1071D000E7E78A880132121A9A42F3D1064D00225B
:1071E000D5F8903705F5F260C5F8BC271B699847BC
:1071F000D7E700BFD02D0024D81C00240748D0F8C2
:107200008C371BB1064B93F896340BB100207047B6
:10721000D0F8903700F5F2605B681847D81C00245E
:10722000D02D0024184A10B4184C92F888374460C6
:107230002344174C036092F8880794F897348342EC
:1072400018D892F88807834207D300235DF8044BCF
:107250001A461846C1E90032704792F888071A1E8C
:107260005DF8044BC0F180030CBF01200220C1E98E
:107270000032704792F88847002201201B1B5DF8FE
:10728000044BC1E900327047D81C002400F40024EC
:10729000D02D0024104B114A93F8881792F89704C8
:1072A00093F88827904293F888270FD8904204D308
:1072B000D3F8843700201844704793F88827D3F810
:1072C0008437C2F18002104418447047801AD3F802
:1072D00084371844704700BFD81C0024D02D0024E8
:1072E000F0B51C4C85B01C4B94F888271B4D0393BC
:1072F000134495F8971494F888270293914294F8D0
:10730000883716D899420CD294F888670F46C6F190
:107310008006D9B9334601223F2BCDE900670DD84D
:1073200060B994F88807401AB0FA80F0400905B0B7
:10733000F0BDCB1A002701221E46EDE76946002367
:1073400002A85CF009FB95F89714EAE7731802228B
:10735000E2E700BFD81C002400F40024D02D002454
:107360002DE9F047174684B000293DD0441E294D31
:10737000DFF8AC904FF0000A04EB0108264E0DE058
:1073800096F888370846994296F888371CD2C3F198
:10739000800318443F281AD8A04525D095F89704B3
:1073A00014F8013F411C09F80030C9B20B0685F8FA
:1073B0009714E5D5002096F8883785F897A40146FC
:1073C000994296F88837E2D3C01A3F28E4D996F854
:1073D00088379942E0D0114B5B78002BDCD000203D
:1073E000FFF77EFFA045D9D1694602A8FFF71AFF33
:1073F000DDE9003213443F2B00D910B904B0BDE8D9
:10740000F08702463B4602A85CF0A6FA04B0BDE84D
:10741000F08700BFD02D0024D81C002400000024D9
:1074200000F4002430B585B0694602A8FFF7FAFEE3
:1074300058B9094C04F5F265D4F8903728465B68D2
:1074400098470028F8D005B030BD0246012302A8B5
:107450005CF082FAEDE700BFD81C002438B50023A9
:10746000124C134DC5F88C3753F07CFEC4F89004D1
:10747000FFF75AFED4F89034C4F88C04A3B19A886C
:107480005B88D21A436802FB0333C5F88C37F9F7DF
:1074900009FB94F89724044695F888379A4201D05E
:1074A000FFF7C0FFC5F8844738BD00BFD02D0024CA
:1074B000D81C00242DE9F041104E154682180446D0
:1074C000D6F88C370F469A420D4A88BF1D1A92F89B
:1074D000972496F888379A4201D0FFF7A3FF00203F
:1074E00021462B463A46C6F8BC07D6F89007846A70
:1074F0000448A446BDE8F041604700BFD81C002402
:10750000D02D0024682400248C4613460146624690
:107510001846CFE72DE9F04F00218BB041F62C72D1
:10752000B7485FF06FFC0420FCF7FEF90146052028
:10753000FCF7FAF951EA000340F05581B14B03938F
:10754000039BE422B049AE48D3F80C455FF0FCFB46
:10755000AB4B1E465C621C67C3F8B440C3F8B8402E
:10756000C3F8BC40C3E90744C3E91A4457F02EF8F6
:10757000FFF774FF002108460EF002FCF9F792FABB
:10758000B0F1000840F399810024A04DDFF8A0C2BB
:1075900006F1E4092746A24605F5936B9C4E01943B
:1075A000CDF808C004E00AF5006AD04540F3AD808C
:1075B000029A536EC2F8C437F9F7A8FA2022594646
:1075C0005046FFF777FF1222924958465FF00AFDB6
:1075D0000028E8D1BA4525D001998F4B01EB410233
:1075E00003EB82034A1C8D4918460193AAEB07035B
:1075F0000592049301F0E8FB019B4946059A41F886
:107600004C3B049BC9F80C700192C9E90433D9F8CA
:107610001C30C9E908330123C9F80830804BC9F888
:1076200028308946039B57461222D3F80C35C9F8F7
:107630001C30A918335D013291F8981499420BD08F
:107640000024202AF5D120375946B845384653DB67
:10765000FFF730FF0022ECE70134152CF1D1D019EF
:1076600070492022FFF726FF00230A2209A96D484E
:10767000CDF824B001F0DCFC0746099800230A226B
:10768000013009A9099001F0D3FC07900023099863
:107690000A2209A90130099001F0CAFC06900023D2
:1076A00009980A2209A90130099001F0C1FC05904E
:1076B00009A9099800230A220130099001F0B8FCB9
:1076C0000023049009980A221946013001F0B0FC09
:1076D00097B10599DDE9063243EA4212049B5B014A
:1076E00043EAC123A7F2BC7143EA600342EA4122A4
:1076F00043EA0243C9F81C30019B642B43D0574630
:107700000AF5006AD0453FF753AF019B642B1ED0AA
:10771000BA451CD00C22404C4049AAEB070502FB9D
:107720000344013320461A46019301F04DFBD9F87A
:107730001C20C9F80040C9F81450C9E908220122E8
:10774000C9F80820364AC9E90375C9F82820019B01
:10775000002B03F1030117DC4FEA4803B3F1805F0C
:10776000C0F2AC80264B986830B91A461B791BB121
:107770001368002B40F0D880002108460BB0BDE80C
:10778000F04F0EF0FDBA67214C261D4BDFF8A49098
:107790004FF0010A06FB01F432460021224F1D1969
:1077A00028465FF02FFB3246002128465FF02AFB77
:1077B0001B4E134A04F11003019942F80490183447
:1077C000C5F808A004312F62AE6242F8038013446A
:1077D0000432C3F80480039BD3F80C3513511444CE
:1077E00063606B62B8E74FF47A7200235CF002FFCB
:1077F0000E4B40F2B27240F26D14B0FBF3F31DE099
:1078000058430024000000243C840A08D02D0024A2
:10781000F4080B08D0080B0888320024E4080B0891
:1078200009750408683200240068214C8051010069
:10783000D81C00240C090B085B1A013212F0030556
:1078400014BF21464FF4B7718B42F5DA8749002DFA
:1078500064D003910399D1F8DC148B42C0F29C8070
:10786000834D01245B1A55F8041F01349942F9DD58
:107870000133A2F2BC72039D43EA44133C2443EA61
:1078800042237C4AB0FBF2F102FB11024FF461602B
:10789000B2FBF0F100FB11221C20C5F8E004B2FBA2
:1078A000F4F004FB1022521042EA401242EAC122D4
:1078B00042EA0343C5F80C3542E603214C266E4BE1
:1078C000DFF8C091012706FB01F4324600214FF09A
:1078D000020A1D1928465FF095FA32460021284613
:1078E0005FF090FA644B039A04F1100143F804909E
:1078F000C8F10063D2F80C0504F11802BB405E4CDD
:107900005E4E85F805A0AF602E62635021444B6047
:10791000231D98501A445060686223E70C46039177
:107920001D21C4F8E01495E7534C002200230146C2
:107930000546A064E063C4E910232246D46C02F13A
:107940004C035CB39C684E1E9D64B442C2E923554F
:10795000DD630DD04E1CB44210D113F8481C002931
:107960003FF40AAF1A6421461A4643F8083CE5E79B
:1079700000293FF401AF53F80C2C2146A1427FF4BB
:10798000FBAE00293FF4F8AE146CE66B0136E663FB
:107990001C6493641A46D1E7012469E7364A02263B
:1079A000254613E0D36B16635B01C2E9045520D072
:1079B00003F6FF7301EB133319465363CB1A91633C
:1079C00052F84C7F4E1C1C440130C7B11379711E14
:1079D000002BE7D1136916637BB103F6FF7301EB4C
:1079E00013335769536337B107F6FF7701EB17314C
:1079F000E4E73346E0E73146E0E73346F1E7DFF816
:107A000088C001391E4B3F250CF5FC62CCF80848B4
:107A1000CCF8EC373E244023CCF81408CCF80418FA
:107A2000880FCCF8F8378B00C2E90445D9B140F291
:107A3000FF141B1940F100005B0A43EAC0530E48D3
:107A4000C2E90B0003F140000344CCF8FC0703EB50
:107A5000C101CCF800384802CCF8E817CB0DCCF8BF
:107A6000E007536088E60123E9E700BF0000002437
:107A7000DC04002480510100584300240068214C9C
:107A800028090B081C090B08D81C002410B50A4C47
:107A9000D4F890375B6A13B104F5F2609847074A4F
:107AA000D4F88437D2F88C24013B528813445242D4
:107AB0001340C4F8843710BDD81C0024D02D0024F6
:107AC0002DE9F047DFF8209192B0464EFFF762FBB8
:107AD00099F8883796F897249A4201D0FFF7A2FCCC
:107AE0000025D9F88C77C9F8845757B36C46DFF86E
:107AF000FC800AE099F8883796F897249A4201D0DA
:107B0000FFF790FC2035AF421BD92A46414620465C
:107B100001F05AF920465CF0A9F8012201462046FE
:107B2000FFF71EFCABB2002BE4D1D9F8C837002B0D
:107B3000E0D09A881B6859690A4218BF12049A61FA
:107B4000D8E7D6F88C349B7B012B44D099F8883742
:107B500096F897249A4201D0FFF764FC0020C9F8F8
:107B60008407002F3AD080466C460546DFF87CA09B
:107B70002A46514609A801F027F921220021204672
:107B80005FF040F9202221462846FFF793FC20228F
:107B9000064609A920465FF025FAABB2203550B958
:107BA000202E08D15BB1AF42E2D8B8FA88F0400984
:107BB00012B0BDE8F08708F10108002BF3D1D9F825
:107BC000C837002BEFD01A689B8851690B4218BF49
:107BD0001B049361E7E7FFF759FFB7E7012012B0F5
:107BE000BDE8F087D02D0024D81C002430090B08F4
:107BF0000A4B93F8100518B9094B93F868097047B8
:107C0000084AD16D0329F7D105494FF0010C81F8DD
:107C100068C90021D16583F8101570470000002461
:107C2000D02D0024004000580321044608B5084622
:107C3000FBF780FE72B6104AD2F87039D2F8741988
:107C400053EA01020AD1002211460420FBF772FE1A
:107C500011460520FBF76EFEFCF7D4FD074A4EF6F1
:107C60006020526E04FB00F0D21841F1000182182E
:107C700041EBE071E9E700BFD02D0024D81C0024BF
:107C8000704700BF2DE9F047002BDDF820A08846A3
:107C900007460CBF4FF020094FF030095646002A26
:107CA000144616F8011B23DD11B3334601E0002C06
:107CB00005DD13F8012B2546013C002AF7D1023DD2
:107CC0003CB149463846C047013DFAD29AF8001007
:107CD00059B13846C047334616F8011B0029F8D180
:107CE000A4EB0A041819BDE8F0872046BDE8F08728
:107CF000002C04F1FF35E4DC00240029E9D1F4E78D
:107D000003685A1C02601970704700BF024B186864
:107D100003681B68184700BF8862002410B56FF025
:107D200000440246044404E0B3EB0E0015D1A24225
:107D300014D012F8013BA3F14100192811F8010BEE
:107D4000A0F1410C98BF203300F1200EBCF1190FB7
:107D5000EAD91B1A04D10028E9D110BD002010BDBA
:107D6000184610BD884230B54FF001043AD301FBEC
:107D700004F4B0FBF4FC8C45F9D2BCB102BB06E0C4
:107D8000A14203F8015B11D81446B0FBF2FCBCF130
:107D9000090F0CF157050CF1300E04FB1C00B4FB6D
:107DA000F1F2EDDCA14203F801EBEDD900221A70EB
:107DB00030BDA14203F8015BF8D81446B0FBF2FCD9
:107DC000BCF1090F0CF137050CF1300E04FB1C005F
:107DD000B4FBF1F2EDDCA14203F801EBEDD9002296
:107DE0001A7030BD8446002AEAD1D0E7002870B569
:107DF00003DA2D23404201F8013B092886464FF063
:107E0000010307DD03EB83035B00B0FBF3F2092AF8
:107E1000F8D89BB10F4CA4FB030CBEFBF3F2092A6C
:107E20004FEADC0C02F1570602F1300503FB12EEBB
:107E300007DD092B01F8016B6346ECD800230B70BA
:107E400070BD092B01F8015B6346E4D800230B7079
:107E500070BD00BFCDCCCCCC0378202B03D110F863
:107E6000013F202BFBD0092BF9D02D2B00F0A9804E
:107E70002B2B75D0B7EE000AA3F13002D1B209293D
:107E800077D8F2EE046ADFED5F7A07EE102A10F879
:107E9000013FB8EEC77AA3F13002D1B2A7EEA67ABD
:107EA0000929F0EE477AF0D92E2B66D003F0DF03D4
:107EB000452B40F0838010B442782D2A00F0968044
:107EC0002B2A00F08380A2F130030130092B00F24D
:107ED00084800024002303EB830302EB430310F8A8
:107EE000012FA2F13001303B0929F4D9B3F59A7F73
:107EF0001A46B7EE007A28BF4FF49A72072B09D9B9
:107F00001346DFED416A083B27EE267A072BFAD8A5
:107F100002F00702DAB1F2EE046A012A27EE267AAD
:107F200015D0022A27EE267A11D0032A27EE267AC8
:107F30000DD0042A27EE267A09D0052A27EE267AC4
:107F400005D027EE267A062A18BF27EE267A002CBF
:107F500045D0C7EE877A5DF8044B20EE270A7047BC
:107F60004378B7EE000A0130A3F13002D1B20929FB
:107F700087D92E2BDFED237A98D143780130A3F1F6
:107F80003002D1B2092991D8B2EE047AF0EE475A04
:107F900006EE902A10F8013FB8EEE66AA3F130022F
:107FA000D1B2C6EE076A092927EE257A77EEA67ABE
:107FB000EED903F0DF03452B3FF47DAF20EE270A17
:107FC00070474378BFEE000A013055E782780230EF
:107FD000A2F13003092B7FF67CAFB7EE007A67EE93
:107FE000877A5DF8044B20EE270A704782780230CA
:107FF000A2F13003092B01D801246BE7B7EE007A18
:10800000A7E700BF0000000020BCBE4CF0B5067919
:1080100006F0E003402B03D145794FF0FF3406E032
:10802000602B4FF00105F8D1447905FA04F40023E0
:10803000012006F00706AB4200D1F0BD052E0FD897
:10804000DFE806F00308101D242448B1C85CD75CA3
:1080500078400FE020B1C856D756C71B7842784108
:108060000133E8E70028FBD031F8130032F8137031
:10807000784080B220420CBF01200020F0E70028A9
:10808000EED031F9130032F91370E6E70028E7D09B
:1080900051F8230052F82370DAE7F8B50C4E054684
:1080A00033798BB9F8BD25B12388C3F30B039D4207
:1080B00004D0A288D4E902015EF046FE1C34BC4222
:1080C000F1D300233371EDE7024C034FF7E700BF14
:1080D00088620024B0F00B0850FA0B08037903F013
:1080E0001803102B1DD003D833B9B0F80B0070471C
:1080F000182BFAD000207047114BB0F80B0093F901
:108100000030591C0BD10F4B1B7803EB430203EBE0
:10811000820303EBC30300EB430080B27047DBB282
:10812000F3E7074BB0F80B0093F901305A1C04D168
:10813000044B5B7800EB4310EFE7DBB2FAE700BFDC
:108140007805002448370024032870B518D80D4B53
:10815000C943C60003EBC00001F00101057B427B6F
:1081600081EA0504A2420BD082683AB14D1B106827
:1081700092886942694109018A40826133445C7393
:1081800070BD00BF88620024092917D0B1FA81F3BD
:108190005B0999B1013903604A0001F0030102F063
:1081A0000802C1EB01119300C1EB0111A3EB920393
:1081B0008900C3EB031381809B004380704700BF9D
:1081C000B5EEC00ADFED357A0023F1EE10FA30B5D6
:1081D000C8BF30EE270A87B0D8BF30EE670ADFEDA0
:1081E000307A054603A9029320EE270ACDE9003331
:1081F000FDEEC07A17EE904A84EAE470A0EBE470DA
:1082000051F038FA002C03A8B4BF2D2320238DF899
:1082100000305BF02BFD01282AD0022834D003283F
:108220001ED003A968465EF0F5FD68465BF01EFDB2
:10823000044669462846033CE4B222465EF084FDCB
:10824000002328462B555BF011FD2E22431C0DEB1D
:1082500004012A54E8185EF00AFE284607B030BD33
:10826000302303A968468DF801305EF0D3FDDCE7CA
:1082700043F23002302303A96846ADF801208DF89F
:1082800003305EF0C7FDD0E743F2300303A9684630
:10829000ADF801305EF0BEFDC7E700BF6F12033AD4
:1082A00000007A440DF07CBB38B5054658B14C1E31
:1082B00014F8011F284619B9BDE838400DF084BBF9
:1082C0000DF06EFBF4E738BD70B50546B0F8090057
:1082D00049F07CFE054B044628461E79FFF7FEFE5A
:1082E00016B1E368184470BDA368FBE788620024F8
:1082F00038B505460C46FFF7E7FF2A7902F0070379
:1083000002F0E002602A29D1052B0CD8DFE803F047
:10831000030B0F0B1B1B6A79012393400278DBB21E
:1083200014B11343037038BD22EA0303FAE76A79F4
:108330000123934002889BB214B113430380F2E7F8
:1083400022EA0303FAE76B7901229A40036814B129
:1083500013430360E7E723EA0203FAE7052BE2D8B9
:10836000DFE803F00303050507070470DBE704807B
:10837000D9E70460D7E708B520215EF05AFD03462F
:1083800018461BB102780133202AF9D008BD08B580
:10839000CB0701D4FCF750FA08BD2DE9F3410023C7
:1083A000124D044600EB8106114F05F8283FB442F8
:1083B00003D1104802B0BDE8F081394628464FF09D
:1083C00000085EF027FD214668465EF050FD202142
:1083D00068465EF02EFD28B96946284604345EF0F2
:1083E00019FDE4E780F80080F1E700BF886200240F
:1083F00077890B08B06200242DE9FF471E46C36849
:10840000044689469246BDF83070DDF8348043B3A7
:108410000D2924DC1A4B5D56BAF1FF3F23D0194ACF
:1084200031463846CDE9005A2368C04752465FFAC4
:1084300089F12079FAF79EF9024600B10288D3B299
:10844000314638460393C2F30323120B0293CDE95E
:1084500000520D4A2368C04704B0BDE8F0870025EC
:10846000DAE74D1CD8E77B06F6D40C953146236835
:108470003846064AC44604B0BDE8F047604700BF2E
:10848000B8090B08477D0B08547D0B08787D0B0855
:108490002DE9F043154685B0894619466A1CBDF89A
:1084A00030600D9F28D04FEA101800F00F04194AD1
:1084B000304608F14008CDE900454346B847C0B111
:1084C000EBB2D9F8000099F805100F2B11D82A4605
:1084D000FAF798F968B103880021027830460392D0
:1084E000C3F303221B0B02920B4ACDE90043434620
:1084F000B84705B0BDE8F0837306FAD4030900F06D
:108500000F00064ABC460C904033304605B0BDE82B
:10851000F0436047877D0B08997D0B08C27D0B08EF
:108520002DE9F043070987B091461E46DDF83880F3
:10853000403700F00F0439B30DF0D8FFC37905467A
:10854000164A49463046CDE900433B46C047C0B1D4
:108550002868FAF7E7FEAA796B7912F0020F104942
:108560004FEA93030F4A18BF0A46E9790133009492
:10857000CDE90321CDE901030B4A3B4600213046FA
:10858000C04707B0BDE8F0833B46084A494630463D
:10859000C4460E9407B0BDE8F0436047D67D0B0893
:1085A000D7810B08A1930B08E87D0B080A7E0B0806
:1085B00010B58C18A14215D001F1FF3E013C41F2EB
:1085C000210C1EF8012F082380EA022002B240008D
:1085D000002A8CEA420180B2B8BF88B2013BF5D1D3
:1085E0007445EED110BD00BF0823484041B24000A1
:1085F0000029C0B2B8BF5040013BF7D1704700BF5F
:1086000030B5056804468D4218D901F1FF3E681E59
:1086100000231EF801CF082183EA0C034FFA83FCE4
:108620005B00BCF1000FDBB2B8BF53400139F5D19C
:108630007045EED16A1C22602B7030BD00236A1C8D
:1086400022602B7030BD00BF9FED067AF7EE007AF6
:1086500060EE870A60EE800A30EEA70A80EE800A9C
:10866000704700BFDB0FC94010B52DED028B08EE3F
:10867000101ADFED807ADFED800A0446B8EE488AF2
:1086800028EE008A28EE278AB0EE480A5DF0BCF991
:108690009FED7A7AF0EE407AB4EEC70AF1EE10FA66
:1086A00040F3BD809FED746ADFED756AB0EE677AC6
:1086B00077EEC67AB4EEE67AF1EE10FAF6DC9FEDCC
:1086C000717AF4EEC77AF1EE10FA40F3C5809FEDAF
:1086D0006B7A77EE677A27EEA76ADFED6B5ADFEDEC
:1086E0006B6A9FED6B7AE6EE256A9FED660A67EE90
:1086F000865ADFED610A38EE000AA6EE267AE5EE2C
:10870000877AB0EE678A5DF07FF9DFED5C7AB4EED0
:10871000E70AF1EE10FA5BDDDFED576A9FED587A5C
:10872000F0EE407A30EE660AF4EEC77AF1EE10FA17
:10873000F6DCDFED547AB4EEE70AF1EE10FA62DD12
:10874000DFED4E7A37EEC00AF7EE007A9FED517AF0
:1087500020EE004ADFED4C6ADFED4C4A0023B0EE1C
:10876000673A9FED4B5AE4EE264AC4ED097A60EE73
:10877000043AA361A8EE073A6361F0EE675A2362F8
:10878000F8EE006AE361A4EE245AE8EE475A87EE59
:10879000836AA3EE850AB6EE007ABDEC028B77EE13
:1087A000C07A26EE077A66EE266A27EE865A67EECC
:1087B000277A25EE866A26EE807A84ED015AC4ED8A
:1087C000007A84ED046AC4ED027A84ED037A10BD68
:1087D000DFED317AB4EEE70AF1EE10FAA9D5DFED5C
:1087E000266A9FED2E7AF0EE407A30EE260AF4EEFD
:1087F000C77AF1EE10FAF6D4DFED227AB4EEE70A8A
:10880000F1EE10FA9CDCDFED267AB4EEE70AF1EE29
:1088100010FA99D5DFED207A37EEC00A94E79FED84
:108820001E7AB4EEC70AF1EE10FA7FF548AF9FED5D
:10883000126ADFED1A6AB0EE677A77EE867AB4EEE6
:10884000E67AF1EE10FAF6D49FED0E7AF4EEC77ADE
:10885000F1EE10FA3FF73BAF9FED117AF4EEC77AD5
:10886000F1EE10FA7FF537AF9FED0B7A77EE677A6E
:1088700031E700BF27D4D236DB0FC940DB0F4940B8
:10888000E4CB1641DB0FC93F92E741B99730083C72
:1088900015A82ABEF304353FDB0F49C0E4CB16C14F
:1088A000DB0FC9BFDFED2D0A08B55DF0ADF8DFEDD8
:1088B0002C7AB4EEE70AF1EE10FA28DDDFED276A34
:1088C0009FED287AF0EE407A30EE660AF4EEC77A31
:1088D000F1EE10FAF6DCDFED247AB4EEE70AF1EE01
:1088E00010FA2FDDDFED1E7A37EEC00A20EE007A97
:1088F0009FED1E6ADFED1E6ADFED1E7AE7EE066A67
:1089000020EE076AE6EE877AA6EE270A08BDDFEDBD
:108910001A7AB4EEE70AF1EE10FADCD5DFED0F6A51
:108920009FED167AF0EE407A30EE260AF4EEC77A22
:10893000F1EE10FAF6D4DFED0C7AB4EEE70AF1EEC0
:1089400010FACFDCDFED0E7AB4EEE70AF1EE10FAA2
:10895000CCD5DFED097A37EEC00AC7E7DB0FC94097
:10896000DB0F4940E4CB1641DB0FC93F92E741B929
:108970009730083C15A82ABEDB0F49C0E4CB16C1CE
:10898000DB0FC9BFDFED2F7ADFED2F0A30EE270AAC
:1089900008B55DF039F8DFED2D7AB4EEE70AF1EEB7
:1089A00010FA28DDDFED286A9FED297AF0EE407A93
:1089B00030EE660AF4EEC77AF1EE10FAF6DCDFED7F
:1089C000217AB4EEE70AF1EE10FA2FDDDFED1F7A1F
:1089D00037EEC00A60EE006A9FED1E6A9FED1E7AB8
:1089E000DFED1E7AA6EE867A20EE266AE6EE877A1C
:1089F000A6EE270A08BDDFED1A7AB4EEE70AF1EE1B
:108A000010FADCD5DFED106A9FED167AF0EE407AB1
:108A100030EE260AF4EEC77AF1EE10FAF6D4DFED66
:108A2000097AB4EEE70AF1EE10FACFDCDFED0E7A48
:108A3000B4EEE70AF1EE10FACCD5DFED097A37EEA5
:108A4000C00AC7E7DB0FC93FDB0FC940DB0F494056
:108A5000E4CB164192E741B99730083C15A82ABEED
:108A6000DB0F49C0E4CB16C1DB0FC9BFB0EEC07A43
:108A7000F0EEE06AF0EE407AC6FE875AF5EE405A14
:108A8000F1EE10FA3BD086FEC75A85EE256A9FEDBF
:108A90001D2A9FED1D3A9FED1D4ADFED1D4ADFEDBA
:108AA0001D2AF7EE005ADFED1C3A9FED1C5AA6EE88
:108AB000423AE6EE223AA6EE034AE6EE235AE6EE04
:108AC000044AA6EE245A85EE250AF4EEC76AF1EEB2
:108AD00010FA03D59FED127A37EE400AF5EEC00A80
:108AE000F1EE10FA03D59FED0F7A37EE400AF5EE5E
:108AF000C07AF1EE10FA48BFB1EE400A70479FED20
:108B0000070AE2E739094E3DE3B59E3E88FA163E74
:108B100045FE7F3F99FB243F69A2163EA7DFA8349C
:108B2000DB0FC93FDB0F49402DE9F04F884689B084
:108B30001E461178531C0393002900F0168100256E
:108B400014460746A94609E038460135C047039C4C
:108B5000621C21780392002900F08F802529F3D12F
:108B60006078A31C3028CDE9033923D0A0F130036D
:108B70004FF0000ADBB2092B26D96C282AD07828BE
:108B80007FD8572878D9A0F15803202B79D8DFE86F
:108B900003F0BD7878787878787878787882AF78CC
:108BA0007878787878787878AA787878789E788ADB
:108BB0007878BD00E31CA0784FF0010A0393A0F180
:108BC0003003DBB2092BD8D804AA03A952F0A2FAC9
:108BD0006C28D4D1039B1A785C1C782A0394B7D8EC
:108BE000572A40F28E80A2F15803202BB0D801A161
:108BF00051F823F02B8D0408518B0408518B040885
:108C0000518B0408518B0408518B0408518B0408C4
:108C1000518B0408518B0408518B0408518B0408B4
:108C2000998C0408478D0408518B0408518B040863
:108C3000518B0408518B0408518B0408518B040894
:108C4000518B0408518B0408518B0408E98C0408EB
:108C5000518B0408518B0408518B0408518B040874
:108C6000D18C0408518B0408578D0408518B0408DB
:108C7000518B04082B8D040828B9284609B0BDE89B
:108C8000F08F039C64E72528FBD1039C25213846FF
:108C90000135C0475CE7039C56F8041B3846013594
:108CA000C9B2C04754E70DF1140B00220A2156F84F
:108CB000040B5B46039CFFF755F85346049A414664
:108CC0003846CDF800B0FEF7DDFF054440E7039CD1
:108CD00056F8040B0023049A414600903846FEF7EC
:108CE000D1FF054434E7039C56F8043B1D602FE791
:108CF0000DF1140B56F8040B039C5946FFF776F858
:108D0000DBE7002AB9D0252AC0D021E7A0F158021C
:108D10000DF1140B102156F8040BB2FA82F25B46E7
:108D20005209FFF71FF8039CC7E7A2F158020DF1A3
:108D3000140B102156F8040BB2FA82F25B4652096A
:108D4000FFF710F8B9E70DF1140B56F8040B59466C
:108D5000FFF74CF8B1E70DF1140B00220A2156F889
:108D6000040B5B46FEF7FEFFA7E70D4685E7F8B567
:108D7000104C07460D461646E06CA0B10E49FFF7B1
:108D800093FA3946E06CFFF78FFA0C49E06CFFF775
:108D90008BFA0B4933462A46E06CFFF7C5FE0949BA
:108DA000E06CFFF781FA94F8503013B1012384F896
:108DB0005130F8BD886200241C7E0B0898980B087F
:108DC000A5820408297E0B080EB400B584B00849BA
:108DD00005AB019001A853F8042B0393FFF7A4FE01
:108DE0000022019B1A7004B05DF804EB03B07047D9
:108DF000017D0408F7B5114E074600230C463046A6
:108E000015460F49523600F8523F04EB45050D4B0D
:108E1000002F18BF19460C4F5DF0FCFFAC4202D189
:108E20000A4803B0F0BD394634F8022B6846FFF714
:108E3000CBFF694630465DF0EDFFEFE78862002426
:108E4000367E0B082D7E0B083F7E0B08DA6200246D
:108E5000F7B500230B4E044600EB41050A4F06F818
:108E6000833FAC4202D1094803B0F0BD394634F823
:108E7000022B6846FFF7A8FF694630465DF0CAFF3F
:108E8000EFE700BF88620024E29F0B080B63002419
:108E9000F8B54E1E054601F11F04054F16F8012FC7
:108EA000284639460235FFF78FFFA642F6D1F8BDB6
:108EB000447E0B0802460846531C05D1034B1A6832
:108EC0001B790A600B71704701497DE7827D0B08B1
:108ED000E39F0B0810B5013114460DF007FB28B9CC
:108EE000054B1A681B792260237110BDC279204698
:108EF0000249BDE8104067E7827D0B08E37D0B085F
:108F000003685A1C02601970090A03685A1C02603F
:108F10001970704702681346511C016013F802CBA8
:108F20000360D31C5178036093781B0443EA012348
:108F3000111D43EA0C030160D07843EA00607047DA
:108F4000A0F13003092B07D920F02000413819285F
:108F50008CBF00200120704701207047303809285D
:108F60008CBF002001207047413819288CBF002099
:108F700001207047613819288CBF002001207047FC
:108F800020280BD0092809D00A2807D00D2805D0A1
:108F90000B3801288CBF002001207047012070474A
:108FA000A0F14103192B98BF20307047A0F1610355
:108FB000192B98BF2038704702B3844610B5841827
:108FC00003E0981A15D1A44514D01CF8013BA3F175
:108FD0004100192811F8010BA0F1410E98BF203370
:108FE00000F12002BEF1190FEBD91B1A04D10028A1
:108FF000E9D110BD002010BD184610BD10467047C5
:1090000070B5044608460D465AF030FE064602E0AA
:1090100014F8013F43B1324629462046FFF7CCFF02
:109020000028F5D1204670BD1C46204670BD00BF0B
:109030002DE9F043064686469EF800C074460EF1C0
:10904000010EBCF1200FF7D0BCF1090FF4D0BCF138
:109050000A0FACF10B00EFD0ACF10D05B5FA85F5B8
:109060006D09002DE8D10128E6D9BCF12B0F3DD0C8
:10907000BCF12D0F39D0102A3ED04FF0FF3E904664
:10908000BEFBF2FE02FB0EF7FF43FFB2002014F816
:1090900001CBBCF1390F4CF02009ACF1300C0DD8EC
:1090A0005FFA8CFC944510DA7045264602D819D137
:1090B000674517D21D404FF0FF30E8E7A9F1570C84
:1090C000B9F1600F5FFA8CFCECD801B10E6003F0CF
:1090D0000103D5B9002803DA002B18BF6FF0004058
:1090E000BDE8F08300FB08C0D1E70125102A94F801
:1090F00001C004F10104C0D1BCF1300F10D06FF0F9
:10910000704E0F274FF01008C0E7B0F1004F04D9A0
:109110001BB14FF00040BDE8F0834042BDE8F08352
:1091200060786FF0704E0F274FF01008A0F14106E5
:10913000192E04F1010698BF203078280CBF0234A4
:109140003446A3E773B50E4610490546FEF7E6FD23
:1091500018B93070012002B070BD2C78602C8CBF23
:10916000613C413C072C0FD8013501230A2201A99B
:109170002846FFF75DFF019BAB4205D00F2803D8BF
:10918000013440EA0410E4E70020E4E7827D0B08A4
:1091900001230A2200214BE770B50D461446FFF764
:1091A000EAF80646A0B1FFF7F3FF40F634031922B0
:1091B0009842A8BF1846B0F5617FB8BF4FF4617000
:1091C000A0F56173B3FBF2F32B70237801332370A6
:1091D0003046FFF7D0F80646A0B1FFF7D9FF40F6BA
:1091E000340319229842A8BF1846B0F5617FB8BF72
:1091F0004FF46170A0F56173B3FBF2F36B702378E9
:1092000001332370304670BD2DE9F04116461F46EC
:10921000404D0446394630464FF47A7200235BF0E5
:10922000E9F93D4B05443D4F3D4E83FB0510E917E1
:109230002844C1EB601183FB0103C8170B44C0EB4A
:10924000631087FB003CC317C3EBAC0386FB0376BC
:109250004FEAE37ECEEBE61EC1EB0116A5EB860CD2
:10926000C0EB00154FEA8E0684F806C0A1EB85011D
:10927000617103EB4301A0EBC10040F2B55101FB6A
:109280001E332071B3F5896F33DA40F2DA218B4255
:1092900037DCB3F5B77F234FB4BF4FF0000E4FF06C
:1092A000010E0EEB4E0175464FEA4E0807EBC10169
:1092B000C88A08EB0E0C0B2107EBCC0C0CF1160C3A
:1092C00001E03CF8020D984210DD0139F9D1F0447B
:1092D000012137F8380006F5FA6E0133A1707544A4
:1092E0001B1A22812580E370BDE8F0810131C9B2EB
:1092F000F1E7032540F296500A4F4FF00608AE46BC
:10930000D7E7022540F22940064F4FF00408AE4649
:10931000CFE700BF80BC92C789888888ABAAAA2AF9
:1093200073B06D16889A0A080D4B10B5D3E9004347
:1093300054EA03020AD10146002340F20112184602
:109340000B80C1F802208B710B8110BD054A126899
:10935000121943F10003FFF757FF012010BD00BFB2
:10936000403700243C1D00242DE9F04104461546F9
:1093700008469442B4FBF2F607D205FB1644134BA1
:109380001B5D00F8013BBDE8F0819642B6FBF2F7A9
:109390000CD20E4B05FB176705FB1644DA5D1B5D0F
:1093A00000F8012B00F8013BBDE8F081BA42B7FBA1
:1093B000F2F807D905FB1878044B13F8082000F8D9
:1093C000012BE7E74046FFF7CFFFF3E7D4090B088F
:1093D000794B9A88B2F57A7F02D94FF47A729A80E3
:1093E000DA88B2F57A7F02D94FF47A72DA80188976
:1093F000B0F57A7F03D94FF47A7210461A81B3F828
:109400000AC0BCF57A7F02D9002294465A819A8913
:10941000B2F57A7F4BD94FF47A72D98991429A8109
:1094200049D900228445DA8180F0B080598B9A8B2B
:10943000914201D900225A83604B1B88002B41D0F6
:1094400010B55F4C82B0A278062A63D92179002931
:1094500040F09E809FED5B7A5B4A07EE903AA379DD
:109460001178F8EEE77A06EE901AB8EEE66AC6EEE4
:10947000276A0BB137EE077AB4EEE67AF1EE10FA0E
:1094800067DC524A5378032B5FD8514901EB4311F3
:109490001078504B0328C3F8D4144ED8EA2203F5B1
:1094A000967300FB02334C4A136002B010BDD98999
:1094B000B1F57A7F3CD8844519D29142B6D30022C7
:1094C0009A81B3E7414A5378032B13D84049107867
:1094D00001EB43113F4B0328C3F8D41413D8EA22FD
:1094E00003F5967300FB02333B4A1360704700207C
:1094F0001881E2E700231078354953700328354B73
:10950000C3F8D414EBD9002103F596731170324AD5
:10951000136070473149207901EB820191ED187A8F
:10952000002899D0531F032BABD9002AA9D035E0CE
:1095300000218445D981C0D3D9E7002103F5967372
:109540001170254A136002B010BD002320495370EA
:109550009EE767EE877ABCEEE77A8DED017A9DF89B
:10956000043007EE103AB8EEC77AF4EEC77AF1EE9F
:1095700010FA01DD0133DBB2E3B1102BA8BF1023D9
:10958000DBB28B4238BF0B4613707AE71A814DE786
:10959000053A032A7FF675AF9FED0A7AB7EE000A07
:1095A00080EE070A5CF098FB2388834228BF0346BD
:1095B000238066E70123E3E7E8390024CC1D00207F
:1095C000283100246F1203389039002448370024D2
:1095D000346300248862002498390024889A0A0899
:1095E0002DE9F04FAB4B83B01B7800AFA3F117020E
:1095F000022A13D9A84A12F83310002940F0BF827A
:10960000DB001A4452784AB1A44A13443A6093F8F2
:109610007C302BB918239F4A137001E09F4B3B60AD
:109620009F4B4FF0000A9F4E03F178059E4BA5F12A
:10963000780B93F808801FE09BF90430142B00F09E
:10964000958220465DF08EFDA20323D5012800F00F
:109650008D82082800F38A82B9F1000F01D03442CC
:1096600006D14146204658F0B1FD002800F07E8228
:109670000BF10C0B5D4513D0DBF8004014F0010931
:10968000DAD020460AF1010A5DF06CFDA2035FFA10
:109690008AFADBD40128DCDC0BF10C0B5D45EBD145
:1096A0000AF1FF33022B00F2618200237F4D02207A
:1096B000DFF8149285F8543511F0F4FB95F858351D
:1096C000D9F80040022B00F0DA82002800F02E8347
:1096D000DFF8F8A1764B4FF47A7895F8B1C54FF0E2
:1096E000000E03F56A7B64222646C7F804C033F8EF
:1096F000081CB1F57A7FB3F8461088BF23F8088CB0
:10970000B1F57A7F33F8061C88BFA3F84680B1F51F
:109710007A7F33F8041C88BF23F8068CB1F57A7F72
:1097200002D9002123F804EC33F8060C8842B3F880
:109730005A00B3F85C1098BF23F806EC884293F8FF
:109740006B1003F1650001F1FF3188BFA3F85AE007
:10975000632993F86C1001F1010188BF83F86B2035
:10976000C9B209294FF0000188BF83F86CE013F8F3
:109770003140013110F801CFA44538BF80F800E036
:109780000329F4D17968EA33012918BF03F864EC9E
:109790009B45ACD13446474EB378042B00F0A182F0
:1097A00023B93388B3F5F07F00F2E581FFF710FEAF
:1097B000414895F8C415FEF7E7FC103095F8E3151D
:1097C000FEF7E2FC95F8F3151030FEF7DDFCB5F876
:1097D0000216B5F800360B43B5F804160B431BB25E
:1097E00013B10123A5F80636344B2340002B00F0BB
:1097F000AC82E30700F15F82600400F1CB812107B6
:1098000040F12D822E49DAF800300C400B40C9F8A7
:109810000040CAF80030230440F106820023224AA7
:10982000D373D377E00440F1098295F81336022B05
:1098300002D1012385F81336DFF88880434608F10A
:10984000780402E006339C420CD01A780A2AF9D137
:109850009978DA78914202D35A79002AF2D00A2014
:1098600021F026FB00234FF4806085F8543511F079
:1098700019FB002800F048821249C7F804A08B4663
:109880008A469AF8050078B39AF8001049B343461F
:1098900021E000BF2C38002428880A08889A0A088A
:1098A00060670024BC02020068370024886200243C
:1098B000BE630024283100245C6800240960000293
:1098C000FE9FFFFDA06800244C3E00246437002466
:1098D00006339C4208D01A788242F9D15A79002A7C
:1098E000F6D0084621F0E4FA0AF1060A5445C8D138
:1098F00096F802805946D7F804A0B8F1080F00F096
:10990000B38195F8B135DAF80020A3F10103C2F371
:10991000C030B3FA83F385F893065B0985F8903677
:1099200095F8B235A3F10103B3FA83F35B0985F827
:109930009636AA4B5878032801D900205870D9F8D8
:109940000030A74803401040A64AC9F80030927B77
:10995000CAF80000002A00F0B081B5F8AC36002B40
:1099600040F09D81A04A1368B3F1807F01D30023AA
:10997000136093689D48184010B140F20223936031
:109980001379013B042B01D901231371A8F10508B8
:10999000974BB8F1030F93F800B040F21581BBF17B
:1099A000000F27D04FF00008DFF878927C605C460B
:1099B000CB46894606E0AAF1060AAAEB060A5445F8
:1099C00040F2EA80DA461BF8010F0028F3D00CF0D1
:1099D000B1FD0028EFD082799307ECD549467C6829
:1099E0000122B8F1000F05D0737C3BB97379012BCC
:1099F00000D01AB1B3790BB10023B3717D4BDA8873
:109A000002F00F00042803D8C2F30312022A02D97D
:109A10004FF42062DA801A8902F00F00042803D87C
:109A2000C2F30312022A02D940F601221A8195F8E4
:109A3000B10695F8BD2695F8B036904205D90022BA
:109A400085F8B12653B1A5F8B42695F8BC269A42FC
:109A500004D2002385F8B036A5F8B43695F8B226BE
:109A600095F8A6379A4202D9002385F8B236624E9D
:109A7000D7F8008006F18009334613F8032D02EB76
:109A80004202424492F854E192F855C192F85601CC
:109A900013F801AF9A79F245A8BFF2466245A8BF14
:109AA000624683F800A09A71DA788242A8BF024623
:109AB000B342DA70ECD103F120064E45DCD14F4BB6
:109AC0001A6B002A00F002810026012002E0063114
:109AD0008C420ED00B782B2BF9D14B78043300FA43
:109AE00003F31342F3D0063122EA030201268C422B
:109AF000F0D10EB1414B1A63414C6E4604F1080897
:109B0000234601E098454BD013F8012F072AF9D9D5
:109B1000002304F8013F0133082BFAD1B5F8AA2538
:109B2000B546B5F8A8359A4202D3364BC5F8A835E4
:109B3000354BFF22354C03F1780085F8D82713F90F
:109B4000082C142A05D053F80C1C34EA010100F04B
:109B5000C5800C339842F2D12D4B5A79022A01D19B
:109B600000225A710C37BD46BDE8F08F29492A48BA
:109B700048F042FA99E54FF4F073338016E602EBB1
:109B8000C301DB00496800297FF43BAD172123485E
:109B9000017036E5224936E649467C68002220E716
:109BA00088B02022FF21E94648465DF02BF9144A8F
:109BB00003E0424549F82330B0D012F8013F59F88C
:109BC00023100131F5D0A3E700233371BBF1000F5F
:109BD00000F0B9804FF00108E6E600BFE839002444
:109BE000BDD7771848370024A0390024FDFDFFFFBA
:109BF000481C0020203D00243963002468370024DD
:109C00003A310024AE014A016C67002401000200D1
:109C1000CC2900246067002488F30B082C3800242A
:109C2000F6DFFFFD2F3100244C4BDB7B002B78D07F
:109C300000234A4AE004D3773FF5F7AD21067FF5CC
:109C4000F4AD474B1978182904D8464BCB40DA07B6
:109C50003FF5EBADDFF8188108F1780402E6A204C5
:109C60007FF5D9AD4049CEE5B379002B3FF449AE3D
:109C7000737C012B7FF445AE0223737441E6002808
:109C80003FF426AD90F904604FF0FF0801E080F842
:109C90000880304611F0F6F80028F8D118E595F85C
:109CA000A80679600CF046FC796800287FF45AAE6B
:109CB000A5F8AC0656E62D49A5E543F4A02340F4EB
:109CC000A020C9F80030CAF8000046E62B207960D1
:109CD00021F0EEF8214B79681A6BF5E685F8D82764
:109CE0003AE7DAF8003024F4805423F48053C9F8BA
:109CF0000040CAF80030338CB3F57A7FBFF456AD1C
:109D00004FF47A73338451E5D9F8003023F00063BF
:109D1000C9F80030DAF8003023F00063CAF80030E8
:109D2000AAE542F201031C4282D17BE5DFF844A0A0
:109D300024F08004DAF80030C9F8004023F08003F2
:109D4000CAF80030C6E45A464EE6DAF8003044F06D
:109D5000080443F00803CAF8003053E568370024CC
:109D60002C38002400410001F6BFFFFDF79FFFFDE6
:109D7000A0680024643700247E4B2DE9F04F93F84F
:109D8000DC3783B0013B012B40F2DE807A4F7B4B06
:109D9000FA68DFF8148202F2DC524345FA6080F080
:109DA000E680DFF8089201229B46754D09F1020614
:109DB0000192B9F80210002900F0B180052906EBE4
:109DC000010240F2AC80AA4280F0A980BBF80000FA
:109DD0003446C0F30B000BE0138814461A44002BE2
:109DE00000F09D80AA4280F09A80052B40F2978077
:109DF00063888342F0D163799B07EDD1238858466D
:109E0000DBF8081094F804A0009348F0F5F8BBF8CC
:109E10000010BAEB113F00F0888000230193BBF8DB
:109E200004100BF11C0B5BF8140CC1F30B015BF875
:109E3000044C50F061FEC3452060BAD3514A524BE6
:109E40001268524E524C1A60FFF7CAFB3278EA236E
:109E5000504D02FB034372782B60A4F1800303EBA7
:109E60004213C4F8A8331EF015FE4FF0FF332868E4
:109E7000494D6B602BF0CCFB21F060F804F2EC4311
:109E800004F2645102E00633994258D01A78002A4D
:109E9000F9D19C78D878844202D358790028F2D03E
:109EA000344C2A7294F81036B4F8142603EB83036A
:109EB00003EB83039B00642BB8BF64237B606423A4
:109EC00003FB02F20023642A7B61BB84B8BF6422D7
:109ED00087F82630C7E90333BA603A622F4AC7E9E8
:109EE000063304F5C063936230F022FE94F8021842
:109EF000B4F8000823F00EFC3BF06CF819F004FAFB
:109F000094F8DC37013B012B29D9254B012201981C
:109F10001B6887F82520FB6003B0BDE8F08FDBF8F5
:109F20000810584648F068F877E7009BA11D58468E
:109F30009A1F48F097F800287FF471AF6DE7F27B25
:109F4000003A18BF0122ABE7F8F762FF154B094949
:109F50000222034481F8FC27C1F8F83716E7F8F726
:109F600057FF0223C4F8F80784F8FC37CDE7012334
:109F7000019363E788620024B0390024B0F00B0835
:109F8000000004084C3E00246437002448370024B5
:109F9000B463002498390024780500245C23002051
:109FA0003C1D002460E3160050FA0B080000020874
:109FB000104B0122032810B504461A7005D9601C05
:109FC000BDE81040C0B211F09FB9EA210A480B4A1F
:109FD00004FB01000A4B147018602BF019FB2AF0E7
:109FE00071F92AF053FA601CBDE81040C0B211F0BC
:109FF0008BB900BF74350020B463002448370024B7
:10A0000098390024044A01200449136881F804089F
:10A0100043F40013136070478C39002488620024D5
:10A02000F8B5164D6B78BE2B26D1AC1C144F02220E
:10A0300029464FF6FF70FEF7BBFA22884AB1A618F0
:10A04000BE4219D2052A17D921463446FEF7B0FA86
:10A05000F3E721460222FEF7ABFA0222A1180634EA
:10A06000FEF7A6FA074B641BA3F8064841F60F5308
:10A07000C31A58425841F8BD0020FCE7000002080E
:10A08000000004088862002470B5046886B00546A4
:10A090000E46C4F310033BBB01220393CDE9013309
:10A0A0002023CDE9042304F17843B3F5801F19D3AD
:10A0B000A4F10163B3F5801F10D2A4F5801302222E
:10A0C00003F17843694601A802925B0C03934BF0BD
:10A0D000D7FF48B14FF0FF3006B070BD51F048FDDA
:10A0E00052F03CFB2346EBE73146204651F018FB8B
:10A0F00018B92B6820332B60EEE76FF00200EBE716
:10A100002DE9F0416A4E90B03378B12B7ED1FFF744
:10A1100087FF80F00104E4B2664B04F00104664D51
:10A12000B3F86331654FADF80030BD4270D3002CF9
:10A1300000F0BC802822002106A85CF063FE604B82
:10A1400004969B1B05935F4BDA68D40770D45D4B74
:10A15000D3F80C21D00774D44FF4807302226946DF
:10A1600004A8ADF83C3059F083F8022269464FF656
:10A17000FF70514DFEF71CFA4FF000080446BD4237
:10A1800069D30025022201A904A8ADF8045059F0B2
:10A190006FF8022201A92046FEF70AFA40BA02220D
:10A1A00002A9C043ADF8080004A859F061F80E9860
:10A1B00088B106ABC0F12002294618445CF022FEAB
:10A1C0009DF93C0018B906A904A8FFF75DFF00231C
:10A1D0008DF83C000E939DF83D307BB1394BDA6829
:10A1E00042F00102DA60DA68D20707D5D3F80C2111
:10A1F00042F00102C3F80C21D3F80C319DF93C0068
:10A20000B0FA80F0400910B0BDE8F081012483E786
:10A21000AB691C3535F8181CD3F8008055F8140CC0
:10A22000C1F30B0150F068FC804518BF01247CE7A6
:10A23000254A5A6002F188325A60DB68D90786D510
:10A240008AE7214AC3F8042102F18832C3F80421C5
:10A25000D3F80C3180E7AE8802A904A88DF80D80F0
:10A26000C6F30B061C35B31DADF8083035F81C3CA1
:10A27000C3F30B021B0BADF80A2006228DF80C303D
:10A2800058F0F6FF062202A92046FEF791F904468F
:10A2900055F8141C324604A858F0EAFF204655F839
:10A2A000141C3246FEF784F9044668E70120AAE749
:10A2B00000000208889A0A08B0F00B0850FA0B0850
:10A2C000000004080020005223016745F8B5264D20
:10A2D000FFF786F995F8DC37013B012B32D9234E85
:10A2E00001220324224FF36885F8082803F2DC5387
:10A2F000F360FFF705FF58B13B78B12B08D1FFF7AA
:10A300008FFE013C0AD058B9FFF7FAFE0028F3D1BE
:10A31000013CEED151F02CFC52F020FA0028F9D08B
:10A3200095F8DC370022013B85F80828012B13D96A
:10A33000104B012100221B6886F8251085F809289A
:10A34000F360F8BDF8F764FD0B4B0222034485F877
:10A35000FC27C5F8F837C2E7F8F75AFD0223C5F81D
:10A36000F80785F8FC37E3E788620024B039002459
:10A37000000002083C1D002460E3160010B5074AE7
:10A380000124074B14709C73FFF7A0FFFFF7F4FC48
:10A390002046BDE8104010F0B7BF00BF7435002064
:10A3A0004837002490F89230B7EE007ADFED6A6A01
:10A3B000014607EE903A90F89630684AB0EE476A48
:10A3C00005EE103A90F89430F8EEE77A04EE903A01
:10A3D00090F89530B8EEC55A05EE903A90F898305E
:10A3E00067EEA67A04EE103A25EE265AF8EEE44A15
:10A3F000F8EEE55AB8EEC44A25EE275A64EEA64AAE
:10A4000065EEA65A24EE264A64EE854A65EEA75A02
:10A4100024EE274AB0EE473AF0B590F8917000F17B
:10A420006F0602F11A050024137807EE903AF8EE51
:10A43000E77A67EE857A67EE867AFDEEE77A17EEC1
:10A44000903AFA2BA8BFFA2323EAE3730B725378EE
:10A4500007EE903AF8EEE77A67EEA47A67EE867A2E
:10A46000FDEEE77A17EE903AFA2BA8BFFA2323EA1B
:10A47000E3734B72937803EE903AF8EEE33A63EEAF
:10A48000A57A67EE877AFDEEE77A17EE903AFA2B17
:10A49000A8BFFA2323EAE3738B72938807EE903AFE
:10A4A000F8EEE77A67EE847A67EE867AFDEEE77A71
:10A4B00017EE903AD5ED007AB3F57A7FF8EEE77AA9
:10A4C000A8BF4FF47A7323EAE3738B812B68002BC8
:10A4D0003FDD90F89730B0EE436A02EE903AF8EE26
:10A4E000E22AA2EEE66A63EE863A83EEA76AA2EE5D
:10A4F000A66A65EEA77A013467EE877A67EE867AF8
:10A50000FDEEE77A17EE903AFA2BA8BFFA23BC4289
:10A5100023EAE37306F8013F00DDF0BD012C13D1FF
:10A5200090F8933007EE103A90F89B3006EE103A10
:10A53000B8EEC77AB8EEC66A27EE267A26EE266A05
:10A540000435083208316FE7B7EE007AB0EE476A9B
:10A55000F6E7B7EE006ACCE70AD7233CEE9B0A0881
:10A5600090F899306BB3B0F864308BB190F89A20C2
:10A57000642102EB8203C3EB0313B3FBF1F3A0F8F6
:10A580006430962312FB03F3B3FBF1F3A0F86630BB
:10A5900043884BB190F89A30642203EB8303C3EBFA
:10A5A0000313B3FBF2F34380B0F850304BB1962263
:10A5B00090F89A3013FB02F36422B3FBF2F3A0F895
:10A5C0005030704790F821304BB3438B83B190F8F3
:10A5D0002230FA22642113FB02F203EB8303B2FB65
:10A5E000F1F2B3F57A7F4283A8BF4FF47A73838385
:10A5F000838843B1FA2290F8223013FB02F36422DD
:10A60000B3FBF2F38380C3884BB190F8223003EBA5
:10A610008303B3F57A7FA8BF4FF47A73C380704782
:10A6200070B50A4C00250A4E94F8913013B12046BB
:10A63000FFF7B8FE20460135FFF792FF3046FFF7DF
:10A64000C1FF042D04F1EA04EED170BDB46300240F
:10A65000E839002410B5064C4FF48072002104F64E
:10A660000A005CF0CFFB0023C4F80C3910BD00BF1A
:10A6700088620024034BD3F8100908B10BF0A4B989
:10A68000704700BF8862002408B50B4605490246A2
:10A69000D1F8100928B10449FEF746FABDE8084090
:10A6A000E8E708BD88620024A5820408024B014641
:10A6B000D3F81009FDF7F8BD886200240048F5E7DB
:10A6C0009F930B080CB4C30607B500D561B905A963
:10A6D00004980191FFF7D8FFFFF7F0FF012003B0C6
:10A6E0005DF804EB02B070470020F8E70FB407B53F
:10A6F00004A951F8040B0191FFF7C6FFFFF7DEFF35
:10A7000003B05DF804EB04B070470349034801F55A
:10A7100000610EC9EAE700BF00E0F11F497E0B08A7
:10A7200010B57521044630F00BFD01460948FFF7CE
:10A73000DDFF1A21204630F003FD01460648FFF7F1
:10A74000D5FF1B21204630F0FBFC01460348BDE845
:10A750001040CBE75D7E0B08707E0B08837E0B08F4
:10A7600038B50B4DE87810F0FD0405D10948FFF726
:10A77000BDFF2046FFF7D4FFEB78013B012B06D845
:10A780000548FFF7B3FF0120BDE83840C8E738BDF2
:10A79000E8390024967E0B08A17E0B0808B5FFF768
:10A7A00085FFBDE8084089E72DE9F04385B0224EDA
:10A7B000FCF7BAFC026983890025018804460292ED
:10A7C0008268DFF8888001924288DFF884901B4F0E
:10A7D000009242681A48FFF789FF15B91948FFF738
:10A7E000DDFFD8F800309D4212DA3378052B20D8EF
:10A7F00009EB8303D3F88C21B38829460135384609
:10A800000093063636F8043CFFF770FF062DE4D1BE
:10A8100050F0A8FC4288838864689B1A03FB0444B8
:10A82000FCF738FD02460848214605B0BDE8F04374
:10A830005CE70022E0E700BF34320024167F0B08FB
:10A84000AC7E0B080A7F0B08257F0B0858320024CA
:10A85000889A0A0810B504460348FFF727FF2046E8
:10A86000BDE810409AE700BF427F0B0808B50346D9
:10A8700010460AB9002008BDDB0601D50029FAD030
:10A88000FFF7E8FFF6E72DE9F04F724C8DB0DFF8E7
:10A89000D0910A4604F1B00A00218346FFF7E6FF93
:10A8A00003900025A37A99F80460AB4200F39280EC
:10A8B00010345445F5D140F216200DF1180A47F036
:10A8C00085FB0027002E4FF015024FF00001D0E964
:10A8D0000245504604BF254634465CF093FA2E7874
:10A8E000002E3ED06978304605910BF0FFFD95F9BA
:10A8F0000290049009F1010253425341002C00F0F0
:10A90000A68000220599A05CB04240F09C802244C1
:10A9100092F90280C14540F0948052788A4208BF83
:10A920000123012203F001030AF8072083F001014B
:10A93000039A58460593FFF799FF059B039044B18E
:10A94000454A30460499CDE900B24246FDF7A0FDE4
:10A95000059B424A30460499CDE900B24A46FDF7CC
:10A9600097FD01370335152FB9D184B3564604F14D
:10A970003F07DFF8E480DFF8E49016F801ABBAF1A6
:10A98000000F21D12078F8B194F9023001331BD0A7
:10A9900061780BF0ABFD0546039A01215846FFF79D
:10A9A00065FF94F902205346294603902078CDE9AB
:10A9B00000B8FDF76DFD207853464FF0FF32294671
:10A9C000CDE900B9FDF764FD0334BC42D5D10DB02B
:10A9D000BDE8F08FE08847F0F9FA002E627AD0E9FE
:10A9E0000231207A04BF1946334605FB00228F56F8
:10A9F00023B39E56B742039A5846049313BF0121CE
:10AA000000214FF001084FF00008FFF72FFF049BD3
:10AA1000039043B1104B324629462046CDE900B39E
:10AA20004346FDF7E9FC0D4B29463A4620460135E1
:10AA3000CDE900B34346FDF7DFFC33E74FF0FF36C7
:10AA4000D8E700236DE703323F2A7FF45CAF4FF075
:10AA5000FF386BE784050024D5AB0408C5A60408BD
:10AA60008862002410B508460749FDF757F9002809
:10AA700015BF0124002405480548FFF7EBFE2046DA
:10AA8000BDE810400AF02ABC477F0B08507F0B0836
:10AA9000777F0B082DE9F04F0C4607468BB040F24C
:10AAA000162047F093FA2246054600213846FFF764
:10AAB000DDFE404B064615221B79002104A8002B21
:10AAC000D5E9024504BF25461C465CF09BF905F11B
:10AAD0003F03039395F80090B9F1000F30D095F83B
:10AAE00001A0002C63D0224600231178494557D19C
:10AAF000283392F8018001226B4403F8182CD045CA
:10AB00003246384613BF012100214FF0010B4FF0B0
:10AB1000000BFFF7ABFE064654B1B8F1000F07D0AB
:10AB2000254B5A464146484600933B46FDF7F8FC04
:10AB3000224B5A465146484600933B46FDF7F0FCEF
:10AB40000335039B9D42C5D13CB3651C0DF1100834
:10AB50004034DFF86490DFF864A018F8013BCBB90B
:10AB600015F8013CB3B116B13046FFF773FE2978F2
:10AB70003B4615F8010C0022CDF800900026FDF7A9
:10AB8000CFFC002215F8010C3B461146CDF800A081
:10AB9000FDF7C6FC0335A542DFD10BB0BDE8F08F51
:10ABA00001330332152BA0D14FF00008A7E7A046D0
:10ABB000A5E700BF88620024D5AB0408C5A6040839
:10ABC000034B0146D3F8100908B10AF0E9BE7047FB
:10ABD000886200240CB407B510F020000BD079B9BE
:10ABE0002320FFF7EDFF05A904980191FFF74CFD25
:10ABF000FFF764FD012003B05DF804EB02B070477D
:10AC00000020F8E72DE9F04F914687B00C461A4630
:10AC1000002180464D46FFF729FE00270646B9F180
:10AC2000000F63D02946062220465CF03FFA002838
:10AC30003246404613BF012100214FF0010A4FF078
:10AC4000000AFFF713FE0646287818F003FB834638
:10AC5000F8B1687918F0FEFA4FF461714FF0190CF1
:10AC6000AB78EA789BF805E01CFB03131CFB02128F
:10AC700095F801B0297900B14079CDE90410CDE90A
:10AC8000023251463B461A4A4046CDE900EBFFF7F7
:10AC9000A1FF207818F0DEFA8346F8B1607918F049
:10ACA000D9FA4FF461714FF0190CA378E2789BF850
:10ACB00005E01CFB03131CFB021294F801B0217980
:10ACC00000B14079CDE90410CDE9023251463B464E
:10ACD000074A4046CDE900EBFFF7F4FC01370634A4
:10ACE0000635142F9BD107B0BDE8F08FCA46D0E7D8
:10ACF000937F0B082DE9F04F904689B01A460C4619
:10AD0000002181464546FFF7B1FD3A4E08F1780330
:10AD10000746DFF8E4B0079394F9040010F0B2F8A6
:10AD200000285CD0B8F1000F61D029460C222046E3
:10AD30005CF0BCF900283A46484613BF01210021C7
:10AD40004FF0010A4FF0000AFFF790FD074695F912
:10AD500004004EF079FCEA790346514606EB820284
:10AD60004846D2F8A42104922A7A06EB8202D2F84D
:10AD7000A4210392AA7906EB8202D2F8A4210292BE
:10AD80006A7906EB8202D2F8A42101922A68009225
:10AD90005A46FFF71FFF94F904004EF055FCE27984
:10ADA0000346514606EB82024846D2F8A42104929B
:10ADB000227A06EB8202D2F8A4210392A27906EB52
:10ADC0008202D2F8A4210292627906EB8202D2F8C2
:10ADD000A4210192226800925A46FFF773FC0C35B9
:10ADE000079B0C34AB4297D109B0BDE8F08FC24647
:10ADF000D1E700BF889A0A08AC7F0B082DE9F04F15
:10AE000090468BB000264FF0190A45464FF4617901
:10AE10000C461A4600210746FFF728FD0990B8F1B5
:10AE2000000F49D029460A2220465CF03FF900284D
:10AE3000099A384613BF012100214FF0010B4FF052
:10AE4000000BFFF713FD2A890990334606925946F5
:10AE5000EA88384605922A790492EA780392AA7819
:10AE60001AFB029202926A781AFB029201922A78E5
:10AE70000092124AFFF7AEFE228933460136594648
:10AE800006923846E2880A35059222790492E278E1
:10AE90000392A2781AFB0292029262781AFB029243
:10AEA000019214F80A2B0092044AFFF70BFC1E2EA5
:10AEB000B5D10BB0BDE8F08FC346DDE7C97F0B0805
:10AEC0002DE9F04F804691461E460C461546002758
:10AED000DFF81CA12DED088B95B094ED008AB5EE3E
:10AEE000408AF1EE10FA7BD0D4ED019A94ED029AEB
:10AEF000D4ED038AB9F1000F49D0D5ED00BA95ED34
:10AF000001BAB4EE6B8AD5ED02AA95ED03AAF1EE73
:10AF100010FA6AD1F4EE4B9AF1EE10FA65D1B4EE64
:10AF20006A9AF1EE10FA60D1F4EE4A8AF1EE10FA64
:10AF30000CBF0121002132468B46404681F00101C1
:10AF4000FFF794FCB0EE6B0A064611A8FDF738F93E
:10AF5000B0EE4B0A07900EA8FDF732F9B0EE6A0A80
:10AF600006900BA8FDF72CF9B0EE4A0A059008A848
:10AF7000FDF726F90599069A079B03904046029132
:10AF800059460192524600933B46FFF723FEB0EE2E
:10AF9000480A11A8FDF714F9B0EE690A83460EA815
:10AFA000FDF70EF9B0EE490A06900BA8FDF708F977
:10AFB000B0EE680A059008A8FDF702F9069B059A0D
:10AFC0000021039040460292524610341035CDE9DC
:10AFD00000B33B460137FFF775FB082F7FF47DAFC9
:10AFE00015B0BDEC088BBDE8F08F0021A3E700BFD2
:10AFF000EC7F0B082DE9F74F92460C461A460021CC
:10B0000081465646FFF732FC00258046DFF864B0E3
:10B01000BAF1000F2CD03146042220465CF046F8ED
:10B0200000284246484613BF01210021012700277E
:10B03000FFF71CFC738880465A46019339463AF85C
:10B040002530484600932B46FFF7C4FD63885A46D7
:10B05000394648460193043634F8043B00932B46A6
:10B060000135FFF72FFB042DD2D103B0BDE8F08FDF
:10B070005746EBE700800B082DE9F04F8FB089466B
:10B08000174600211A4606460024FFF7EFFB0DF194
:10B09000240B0546DFF86CA059F82480594602A815
:10B0A000CDF808804EF07CFA4FB357F824302A468A
:10B0B00030469845039313BF012100214FF001084A
:10B0C0004FF00008FFF7D2FB04A9054603A84EF095
:10B0D00067FA04A923465246009130464146FFF7DD
:10B0E00079FD23460134524641463046CDF800B042
:10B0F000FFF7E8FA202CCFD10FB0BDE8F08FB846AB
:10B10000EFE700BF11800B082DE9F04F924685B0A4
:10B110000C461A46002181465546FFF7A7FB00263C
:10B120008046DFF86CB0BAF1000F2FD02946042218
:10B1300020465BF0BBFF00284246484613BF012172
:10B14000002101270027FFF791FBEB7880465A4644
:10B1500002933946AB78484601932B8800933346D7
:10B16000FFF738FDE3785A463946484602930435DE
:10B17000A378019334F8043B009333460136FFF77C
:10B18000A1FA102ECFD105B0BDE8F08F5746E9E700
:10B190001B800B082DE9F04F85B014461A46054672
:10B1A00002910021FFF762FB4FF0000806460623DC
:10B1B0004FF0000903FB08F7C037029B13F807B0F4
:10B1C000002C7AD0E35D324628469B45039313BF9B
:10B1D000012100214FF0010A4FF0000AFFF746FB62
:10B1E000039B0646374A51462846CDE9009343461D
:10B1F000FFF7F0FC4346334A514628460137CDE974
:10B20000009B09F10109FFF75DFAB9F1060FD4D1EE
:10B2100008F10108B8F1060FC9D1E427029BA7F194
:10B22000E40913F807A0002C49D014F807B03246FF
:10B230002846DA450DBF4FF001084FF00008012104
:10B240000021FFF713FB062306461E4A4146284607
:10B25000CDE9009BFFF7BEFC01370623194A4146A2
:10B260002846CDE9009AFFF72DFAEF2FD6D1029BA1
:10B2700093F8EF70ACB194F8EF803246284647451A
:10B2800013BF0121002101240024FFF7EFFA00235E
:10B290000C4A2146009328460723CDF80480FFF787
:10B2A00099FC0023074A214628460093072301976B
:10B2B000FFF708FA05B0BDE8F08FA2469AE7A0466E
:10B2C000CAE700BF2D800B082DE9F04F0E4615464A
:10B2D00089B01A4600210446B046FFF7C7FA2F4648
:10B2E00081464FF0000B002D7AD039460C224046A3
:10B2F0005BF0DCFE00284A46204613BF01210021F6
:10B300004FF0010A4FF0000AFFF7B0FA97F90B204F
:10B3100081465B460492514697F90A2020460392E3
:10B32000B7F908200292B7F906200192B7F9042074
:10B330000092364AFFF74EFC98F90B205B460BF162
:10B34000010B51460492204698F90A200C3708F167
:10B350000C08039238F9042C029238F9062C019259
:10B3600038F9082C0092294AFFF7ACF9BBF1080F15
:10B37000B9D14FF0000BDFF898800C2303FB0BF9D9
:10B3800085B3002755F80900012356F8092003FA70
:10B3900007FA42403AEA020214BF1946002110EAB5
:10B3A0000A0F07D05B464246204600970791FFF7F9
:10B3B00011FC079956F809201AEA020F05D05B46DE
:10B3C000424620460097FFF77DF901370E2FD9D16D
:10B3D0000BF1010BBBF1080FCFD109B0BDE8F08F25
:10B3E000AA46A9E72F46012356F8091003FA07F2E7
:10B3F0000A4206D05B464246012120460097FFF7ED
:10B4000061F901370E2FEED1E2E700BF41800B0852
:10B4100059800B082DE9F04F89468DB01646002162
:10B420001A4607460024FFF721FADFF8DCA005469C
:10B43000C4EBC40309EB030259F80300918840F3FD
:10B44000074892790890ADF824108DF82620B8F1BD
:10B45000000F53D0002E54D0F218F05891889379F1
:10B4600007220A9008A8ADF82C100AA98DF82E30F2
:10B470005BF01CFE00282A46384613BF012100213C
:10B480004FF0010B4FF0000BFFF7F0F99DF82E3055
:10B4900005465246069359469DF92D303846059388
:10B4A0009DF92C3004939DF82B3003939DF92A309D
:10B4B00002939DF8293001939DF82830009323468C
:10B4C000FFF788FB9DF826305246594638460693CA
:10B4D0009DF9253005939DF9243004939DF8233080
:10B4E000CDE902839DF8213001939DF8203000932F
:10B4F00023460134FFF7E6F8102C99D10DB0BDE8D2
:10B50000F08FB346DEE700BF6E800B082DE9F04FE9
:10B510009246002689B04FF019095546B3464FF4BC
:10B5200061780C461A4600210746FFF79FF90790FD
:10B53000BAF1000F27D02946062220465BF0B6FD5F
:10B540000028079A384613BF012100214FF0010B54
:10B550004FF0000BFFF78AF96A790790334619FB21
:10B5600002825946384605922A7919FB02820492D2
:10B57000EA780392AA7802926A7801922A78009275
:10B58000104AFFF727FB627933460136594619FB0B
:10B590000282384606350592227919FB028204920E
:10B5A000E2780392A27802926278019214F8062B54
:10B5B0000092044AFFF786F80A2EB9D109B0BDE817
:10B5C000F08F00BF8B800B082DE9F04F14468BB035
:10B5D0000F461A4600210646FFF748F90546002C9B
:10B5E00000F0D78022783B789A42024630460DBF61
:10B5F0004FF001084FF0000801210021FFF736F954
:10B60000237805469B4A41463046FFF7E3FA3B78EC
:10B610004146984A3046FFF755F8002C00F0BB80B1
:10B62000627830467B789A422A460DBF4FF0010877
:10B630004FF0000801210021FFF718F96378054653
:10B640008D4A41463046FFF7C5FA7B7841468A4A23
:10B650003046FFF737F807F1C90307F1020A04F192
:10B66000CA0B0593A31C4FF000090693822307938E
:10B670003B784B4500F39180002C00F0F58097F863
:10B68000EA30304694F8EA209A422A460DBF4FF03D
:10B6900001084FF0000801210021FFF7E7F894F8B6
:10B6A000EA300546754A41463046FFF793FA97F867
:10B6B000EA304146714A3046FFF704F8002C00F0AA
:10B6C000D58004F1EA0307F1EA0204F1FA014FF030
:10B6D000010833F802CF32F8020F844518BF4FF04B
:10B6E00000089942F5D188F001012A463046C9B2D6
:10B6F000FFF7BCF80821054604F1EC00FDF7A8FBB4
:10B700005F4A034641463046FFF764FA97F8EA106D
:10B7100007F1EC00FDF79CFB594A034641463046D1
:10B72000FEF7D0FF002C00F0A3804FF0FC094FF093
:10B73000010807EB090104EB0900FCF7EFFA09F136
:10B740000409002818BF4FF00008B9F58E7FF0D12A
:10B7500088F001012A463046C9B2FFF787F8082170
:10B7600004F1FC00FCF719FE464A03464146304608
:10B77000FFF730FA97F8EA1007F1FC00FCF70DFE2E
:10B78000404A0346414630460BB0BDE8F04FFEF755
:10B7900099BFA0463BE7A04657E7079BFB180993D4
:10B7A000002C5FD0079B0998E31819460893FCF713
:10B7B000B5FA059B5A789BF800309A424FD1B0FAFF
:10B7C00080F84FEA5818069AAAF102030AF10E010E
:10B7D000023A33F802CF32F8020F844518BF4FF017
:10B7E00000088B42F5D188F001012A463046C9B2E3
:10B7F000FFF73CF86278069905469BF81800FDF7BC
:10B80000F9FA02909BF8003041461F4A30460193F6
:10B81000089B009309F10103FFF7DCF9059B5146F2
:10B820007A7809F10109587E0AF1100AFDF7E2FA67
:10B83000059A0290414612F8013F30460BF1010B88
:10B840000193099B059200934B460F4AFEF73AFF7E
:10B85000069B10330693079B0933079308E74FF0C5
:10B860000008B0E7A046D9E7A04620E7A0464DE78C
:10B87000A0467FE7A4800B08B6800B08E4800B0885
:10B88000FC800B0813810B08CB800B082DE9F04FCF
:10B890000F46904689B0002187EA08080646139AA9
:10B8A00000250393FEF7E2FFDFF884906FEA0803B8
:10B8B0000446069328460FF0ADF8129B184230D08C
:10B8C000069BDFF870B0034014BF4FF0010A4FF041
:10B8D000000A049310EA070328460CBF4A465A465A
:10B8E000059307920FF0A8F8039B8046079A5146EC
:10B8F00000903046FFF76EF9049B22463046B3FABB
:10B9000083F14909FEF7B2FF059A0446039B002A1A
:10B910000CBF5A464A4651463046CDF80080FEF7E5
:10B92000D1FE0135182DC5D109B0BDE8F08F00BF9B
:10B930002A810B08FA7F0B082DE9F04F3B4C89B0A8
:10B940000A4600210546FEF791FF0590384A237804
:10B95000608802EB8303D3F8449346F037FB354B02
:10B96000D0F808B01F7917B15F46D0F80CB0A379B2
:10B970000026012B38BF012306932279637906FB49
:10B9800002331BF80380002F3AD0FB5C4345059A35
:10B990002846079313BF012100214FF0010A4FF001
:10B9A000000AFEF763FF079B0136059053B303F0CF
:10B9B0000F021B0951462846403302921E4ACDE928
:10B9C00000634B46FFF706F9B8F1000F24D008F0EA
:10B9D0000F034FEA1818184A5146029308F1400322
:10B9E0002846CDE900634B46FEF76CFE069BB3424A
:10B9F000C3DC0834114BA342A8D109B0BDE8F08FD5
:10BA00003B46C3E7002FDFD04B460D4A5146284640
:10BA10000096FFF7DFF8D7E76B06E7D44B46084AF6
:10BA2000514628460096FEF74DFEDFE76C9C0A085B
:10BA3000889A0A088862002431810B08CC9D0A0884
:10BA400047810B080FB407B504A951F8040B019105
:10BA5000FEF71AFE03B05DF804EB04B070472DE961
:10BA6000F041037903F0E002402A4DD009D83ABBF7
:10BA700003F00703052B1ED8DFE803F0181D181D7F
:10BA80000910602A47D0802A41D0BDE8F081D0F863
:10BA900005102348BDE8F041FEF728BED0F8052088
:10BAA00051422048BDE8F041FEF720BEB0F8072023
:10BAB000B0F80510F5E7B0F90720B0F90510F0E788
:10BAC00046790024184D194805EBC605FEF7EEFD32
:10BAD000012395F8BC74A74203D8BDE8F041FEF7F6
:10BAE000EDBDD5F8B8644FEA840856F824204AB171
:10BAF00013B90F48FEF7DAFD56F808100D48FFF7A6
:10BB0000A1FF00230134E6E741790B48C2E78279BF
:10BB100041790A48C6E70A48BDE8F041FEF7E6BDAC
:10BB20005B810B0871810B08889A0A0888810B08D1
:10BB300002840B0855980B0899810B08AA810B0801
:10BB4000C1810B08F8B5154B1B6833B30025144FA2
:10BB50001448FEF723FEFEF78DFDFBF71BFBFBF7FA
:10BB60004DFB044648B113200FF01CFBFEF7A6FD69
:10BB70000D48BDE8F840FEF711BE38466E1CFFF7D1
:10BB800061FF792D02D12646FEF798FDFEF772FD82
:10BB900064203546FAF770FFE1E7F8BD642400241D
:10BBA0001F990B08D9810B08F3810B086F4B42F2E8
:10BBB00001011A68B1EB124F4FEA12432DE9F04F21
:10BBC00091B000F0CE8042F20302934200F0CB80AD
:10BBD00041F20302991A4B424B41654A654D116887
:10BBE00005EBC303644A654C6548664FDFF8F08196
:10BBF000DFF8BC91B1FBF2F2D3F87C16FFF722FF1D
:10BC0000B4F814294FF47A730A20B2FBF3F103FB62
:10BC10001122B4F9163992B2B2FBF0F25A48FEF78B
:10BC200065FD5A4A5A495B48FFF70CFFFEF746FD8F
:10BC3000594B5A4A997B5A4B05EB81015948D31A03
:10BC4000B4F80628D1F89816FEF750FD5648FEF7CE
:10BC50002DFD94F818195548FFF7F4FE5448FEF7E7
:10BC600025FD94F819195348FFF7ECFEFEF726FD61
:10BC70005148FEF71BFD00210A46FB7F4E1C0B417D
:10BC800013F0010F08D012B14846FEF70FFD314600
:10BC90004046FFF7D7FE0122072E3146EDD1474E31
:10BCA00096F86A1506F13C0306F5EC72012908BF07
:10BCB000134693F8DC30032B02D04148FFF7C2FE55
:10BCC000404A96F86A1502F5CE73012918BF13464B
:10BCD00093F8DC30012B02D13B48FFF7B3FE394A21
:10BCE00096F86A1502F5CE73012918BF13461B6931
:10BCF0005B7B012B02D93548FFF7A4FE344FFEF7DA
:10BD0000DDFC0026D4F81C8907F12009DFF8D4A057
:10BD1000DFF8D4B057F8041B002967D00123B340E3
:10BD200013EA080F1BD0DA0619D01AF8062059F8C2
:10BD3000263053F8222036B12648CDE90212FEF70C
:10BD4000B5FCDDE902125846FFF77CFE012E06D154
:10BD5000214B93F8211011B12048FFF773FE0136F3
:10BD6000D8E7022339E7032337E700BF0010005C60
:10BD7000A4040024889A0A0840420F008862002424
:10BD800001820B08E839002414820B08F8FF012017
:10BD90000008000035820B08483700240000040822
:10BDA0000000020859820B0888820B089A820B084F
:10BDB000A2820B08A4820B08AC820B08CC1D0020C9
:10BDC000C5820B08081E0020CD820B08D2820B080A
:10BDD00028A10A0802840B0874350020E0820B08B1
:10BDE000BC820B0834060024DA820B08FEF766FCDE
:10BDF000794B7A481A687A4B1978137A05EB8101E6
:10BE0000527AD1F8D816FEF771FC764B764819684D
:10BE10004FF47A73B1FBF3F1FFF714FE05A8FDF7B9
:10BE200083FA38B105A908A857F04EFD08A96F4854
:10BE3000FFF708FEFEF742FCD4F8A829002A00F01C
:10BE4000858007EE902ADFED6A6AB8EEE77AC6EEE3
:10BE5000877AFDEEE77A17EE903A664E96F828015B
:10BE600030B1D6ED4B7AFCEEE77A17EE901A88B235
:10BE7000D4F828795FB107EE907ADFED5D6AF8EECD
:10BE8000E77A86EEA77AFDEEC77A17EE907A5A49DE
:10BE9000B1F870106429CDE90007A8BF64215748A4
:10BEA000FEF724FC96F8303196F8312105EB830338
:10BEB000B6F834115248D3F8EC36FEF717FC514B64
:10BEC0005148198889B2FEF711FCFBF72DF9016979
:10BED00021B182684D48120DFEF708FC4C48FEF770
:10BEE000E5FB4C4B1B681B0663D596F86031032BB2
:10BEF0008CBF49484948FEF7D9FB94F85835022BC6
:10BF000026D14748FEF7D2FB96F86031042B47D87C
:10BF10004448FEF7CBFB96F87031002B47D005EB79
:10BF2000C305D5F804174048FFF78CFDFEF7C6FBA4
:10BF30003E48FEF7BBFB3E4B01253E4E1C68002CE5
:10BF40003BD1FEF7BBFB11B0BDE8F08F134684E791
:10BF500002200EF0C5FF074608B93748D2E790F92E
:10BF600004004DF071FB804639F01EF805EB8000AF
:10BF70004146D0F8A4213148FFF764FD94F85B35C1
:10BF8000012B04D12E48FEF791FB2E48BAE7BB796E
:10BF90002D4805EB8303D3F8A411FFF753FDF4E715
:10BFA00094F85A350BB92948B3E72948B1E729492C
:10BFB000B9E72948FEF77AFBB8E794FAA4F0B0FA9B
:10BFC00080F005FA00F024EA00040EF009FD0146B5
:10BFD0003046FFF737FDB2E79C3D0024E4820B08B2
:10BFE000983D00243C1D0024F6820B0810830B08AA
:10BFF00000247449807300247435002023830B08C7
:10C0000069830B08C427002490830B089F830B08C7
:10C01000BA830B0864370024C0830B08CC830B0859
:10C02000DC830B08389A0B0820840B083C840B082F
:10C030008C3900242C840B08E2830B08EC830B085A
:10C04000FC830B0801840B08C57F0B0805840B08D3
:10C0500015840B08F9810B0830840B082DE9F04F8B
:10C06000DFF86C8199B098F80330002B00F09380D2
:10C070004E4800254E4EDFF85CB1FEF78FFB2F4691
:10C08000DFF85491DFF854A10BA9E8B217F0B4FB24
:10C090009DF83430002B53D0139C54B107EE904AD6
:10C0A0009FED440AF8EE677A80EE270A59F014FEF5
:10C0B00004460B9A29465846FFF7C4FC109A002AFA
:10C0C0006BD002FB04F04FF47A73B0FBF3F30993E7
:10C0D000DDF848C0BCF1000F61D00CFB04F142F266
:10C0E0001073B1FBF3F1082D98F8033018BF7F18D7
:10C0F000002B56D017984FF47A7E0A230790159894
:10C100000690169805901198B0FBFEFECDF810E051
:10C110000998B1FBF3FE03FB1E11CDE902E1099979
:10C12000B1FBF3F103FB1100BCFBF3F3CDE900100D
:10C1300021465046FEF7DAFA0023B362C6E90D3312
:10C1400001354036242D9FD198F8033003B31A4CA3
:10C150004FF47A731948D4E95D12B1FBF3F3D208B6
:10C16000D4F87C11FEF7C2FA0A22154897FBF2F1C7
:10C1700002FB1172FEF7BAFA124B1B78432B04D163
:10C180001148D4E96021FEF7B1FA0023C4F87C31EC
:10C1900019B0BDE8F08F0D486BE7099298E761464A
:10C1A000A1E721464846FEF7A1FAC5E752840B08ED
:10C1B000A86B00248096184B80730024F9840B0828
:10C1C00019850B08172900243D850B08B0840B083E
:10C1D00048370024BA840B0801880B08C9840B086F
:10C1E00010B5114B86B0114904460493104B114809
:10C1F0000393114B114A0293114B0193114B00937E
:10C20000114BFFF71FFCFEF759FA10491048FEF7D3
:10C210006DFA3CB10F4A1049104806B0BDE8104015
:10C22000FEF764BA06B010BDA7850B0871850B0830
:10C23000AC850B087C850B08B7850B0867850B0858
:10C24000C0850B08CC850B084F370024D2850B081E
:10C25000DA850B08EB850B08F8850B08FF850B08C2
:10C260000120BDE7264810B5FEF720FA254B93F8CC
:10C270002130002B42D02448FEF790FA234C1CF0CA
:10C280008DF970B12248FEF711FA224B93F828314C
:10C2900053B394ED450A59F01FFD01461E48FEF7C1
:10C2A00025FAB4F80C111D48FFF7CCFB94F80831BF
:10C2B000F3B11B48FEF772FAB4F810111948FFF7F2
:10C2C000C1FB94F80A31ABB11548FEF767FAB4F830
:10C2D0000E111548FFF7B6FB94F8093163B1104809
:10C2E000BDE81040FEF75ABA1048FEF757FAD8E7F3
:10C2F0000F48DFE70E48E8E70D48F1E70D48EFE7A4
:10C300002C860B086837002442860B087435002001
:10C3100049860B088073002463860B0872860B081D
:10C3200092860B08A2860B08BC860B0868860B0851
:10C330009B860B08B4A00B0838B50C4B0C4603EBDE
:10C34000C0050B4895F8E42103EB8203D3F84413AE
:10C35000FFF778FB95F8EA3133B1611C0548C9B2A3
:10C36000BDE83840FFF76EBB38BD00BF889A0A08A9
:10C3700055980B08E29F0B086B4B1B782DE9F04F8B
:10C3800087B0002B00F0CA80684D4FF00008684865
:10C39000A968FEF7ABF969686648FEF7A7F9664B2E
:10C3A0006648D3E90031C91A654B1A68B1FBF2F24D
:10C3B000FEF79CF9FEF782F96248FEF7EFF9624852
:10C3C000FEF7ECF9614B5FFA88F41B78A34221D8A1
:10C3D0005F4D00245F4EFEF771F9013455F8041FDC
:10C3E0003046FFF72FFB162CF7D15B4D0124594E39
:10C3F000FEF764F92B466968013430461B68043542
:10C40000C91AFFF71FFB162CF4D107B0BDE8F04F97
:10C41000FEF754B9514B14264FF03C0B671C03EB4D
:10C42000840306FB045693ED4A0A59F055FC96F82E
:10C430001EA081B2B6F80E901AF0010F80B20CBFA8
:10C440002D2252221AF0020F049045480CBF2D23D2
:10C4500054231AF0040FB1FBFBF10CBF4FF02D0C6D
:10C460004FF0560C1AF0080F05914FF064010CBF05
:10C470004FF02D0E4FF0430E1AF0800F01FB09F123
:10C480000CBF4FF02D0A4FF0530ACDE900CECDE995
:10C4900002A13946FFF7D6FAB37FDB073AD55C2312
:10C4A000304A6343D118D05891ED010A70B1B8EE0B
:10C4B000400ADFED2D7A20EE270A07EE900AF8EE0B
:10C4C000677A80EE270A59F007FC00B2642290FBDD
:10C4D000F2F102FB11022548FFF7B4FA14212448B7
:10C4E00008F1010801FB075701FB0454F988628A2F
:10C4F0000491218B02F0030392080391E18A0291D7
:10C50000A18B0191A18A009119214B43218AFEF749
:10C51000EDF857E71748FEF7C9F8DFE7164807B008
:10C52000BDE8F04FFEF73AB904000020101B0020D0
:10C53000DC860B08EC860B083C1C002003870B08EC
:10C54000441D002430870B088C870B08481C0020F2
:10C55000B81B00203C880B08BC1B00207435002051
:10C56000E8870B083018002000401C4605880B089F
:10C570001A880B0811880B0840880B080EB403B505
:10C5800003AA52F8041B0192FCF7F1FB064BD3F807
:10C5900010291AB90549D86CFBF786FE02B05DF880
:10C5A00004EB03B0704700BF886200249F930B0820
:10C5B0002DE9F04798460B7981460F4603F0E005D8
:10C5C0001646402D32D10024634DDFF8A881DFF8F4
:10C5D000B09116E03B7903F00703013B042B04D82C
:10C5E000DFE803F014171A1D2100315D5A48FFF7E8
:10C5F00029FA7B79013BA34202DD4846FEF756F853
:10C6000001347B79A342E5DCBDE8F0873157284649
:10C61000EDE736F81410FAE736F91410F7E756F894
:10C6200024104046E3E756F82410F0E703F0070330
:10C63000052B57D8DFE803F0031F27292C3E347859
:10C64000602D55D02CD8002D75D1B7F80550B7F80E
:10C65000076021464048FFF7F5F9AC4239DBB442A8
:10C6600037DCB8F1000FCFD0324629463B48BDE851
:10C67000F047FFF7E7B996F90040602D38D00FD8A2
:10C68000002D58D151E03488DAE7B6F90040F4E7DC
:10C69000D6F800A0202D54464DD034D9602D27D097
:10C6A000802DB1D132782E4B2E48002A14BF31464E
:10C6B000194635E0202D34683DD0EFD82146264874
:10C6C000FFF7C0F9D7F80510A14202DB4B42A342A5
:10C6D00021DDFDF7F3FF23463A6848462249BDE8CD
:10C6E000F0474BE7202D25D01ED9602DD8D100244E
:10C6F0007B7944FA03F3DB07BDE8F0474CBF1B48E6
:10C700001B48FFF79FB951461A48FFF79BF9D7F826
:10C7100005108A45DDD8B8F1000F3FF475AF164813
:10C72000BDE8F047FFF78EB90024B7F90550B7F917
:10C7300007608EE700247A79104B03EBC20393F86D
:10C74000BC24A242C5DDD3F8B83453F82400BDE8B8
:10C75000F047FDF7ABBF00BFE39F0B0884800B08D9
:10C76000089A0B0855980B0862880B08D6810B08AD
:10C77000B4A00B086E810B085C880B08889A0A0825
:10C78000A2820B082DE9F04F164685B0334C1A46AD
:10C790004FF00009A246CDE9010100213046FEF725
:10C7A00065F806F0100300900393FDF763FF23790B
:10C7B000029A03F01803934203D0002A44D1182BA5
:10C7C00042D14FF00D0B0BFB09A3B3F8090045F064
:10C7D000FDFB80462046FBF781FC0746D8E9022195
:10C7E000024401442046FBF711FC80F0010105469C
:10C7F000009AC9B23046FEF739F8039B009003B1A6
:10C8000015BB0BFB09FBB3065AF80BB00ED56DB97F
:10C8100059461348FFF716F9D8F808202B46214649
:10C820003A440198FFF7C4FEFDF748FF59460D480A
:10C83000FFF708F9D8F80C20002321463A44019864
:10C84000FFF7B6FEFDF73AFF09F1010940F2812337
:10C850000D349945A9D105B0BDE8F08F08AB0A08A1
:10C860007C880B087D880B0870B5164605460C467B
:10C870000846FBF729FD3346024621462846BDE817
:10C88000704095E60EB403B503AA52F8041B01925A
:10C89000FCF76DFA044B0549D86CFBF705FD02B0B7
:10C8A0005DF804EB03B07047886200249F930B0887
:10C8B0000049E7E787880B0838B50C460546154957
:10C8C0002046FBF72BFA30B9FDF7AAFE1248BDE867
:10C8D0003840FDF763BF11492046FBF71FFAA8B99E
:10C8E0000F4B83F8BD0183F8C50183F8A70283F8D5
:10C8F000AF0283F8910383F8990383F87B0483F8EC
:10C900008304084B83F821000748E0E72846BDE888
:10C910003840CDE796880B089C880B08B7880B0831
:10C9200088620024E8390024BF880B080049A9E781
:10C93000DB880B08F8B50C4606460846FCF728FCD1
:10C940002021054620465AF074FA044618B93046AC
:10C95000BDE8F840EAE7114F114E3B7832789A4231
:10C9600001D0FAF75FFD0F4B20461D6057F07EF9AE
:10C97000012201462046FAF7F3FC3B7832789A42CE
:10C9800001D0FAF74FFD204657F070F92A460146CC
:10C990000548BDE8F840FDF7A9BE00BF60240024AB
:10C9A000673200245C240024F2880B082DE9F04152
:10C9B0000D4688B006460846FCF7EAFB20210446EF
:10C9C00028465AF036FA20B9304608B0BDE8F041A2
:10C9D000ACE7FCF7DDFB2246054601460F48FDF7B4
:10C9E00085FE85B1202D2A466946204628BF202293
:10C9F000E846FAF75FFD00270646B74208DBAD1BA5
:10CA00003444002EEDD1FDF759FE08B0BDE8F081A9
:10CA100018F8010B0137FEF7D3F8EEE708890B0889
:10CA20002DE9FF47074608460D4657F01FF908282D
:10CA300046D105F1FF3801AE073531464246B146D1
:10CA400012F8010FFCF7B2FA01F8010BAA42F7D174
:10CA50000023DFF880A08DF80C30A84518D11C49C0
:10CA600048462BF063F81A4808231A4910F8012B9E
:10CA7000013B11F8014B02F110026A4402F80C4C20
:10CA8000F4D101A914488DF80C30FDF72FFE14E005
:10CA900018F8010FFCF78AFA0446014606F8010B64
:10CAA00050465AF0C6F928B1214630465AF0C1F92D
:10CAB0000028D2D03846FFF7FBFE04B0BDE8F0876F
:10CAC0000028D0D0384604B0BDE8F0472EE700BFBC
:10CAD00068370024801C0B0820890B0807B50093D9
:10CAE00013460A460249FFF7CDFE03B05DF804FB8A
:10CAF00027890B082DE9F04F06468BB00D46DFF86D
:10CB0000A082284657F0B2F8034638B90246964943
:10CB100001200BB0BDE8F04FFEF77CBC0522934925
:10CB20002846FCF749FA0446C8B9914D01467022DF
:10CB300005F5C4705AF066F9C5F8F841C5F8044225
:10CB4000C5F81042C5F81C42C5F82842C5F8344261
:10CB5000C5F84042C5F84C420BB0BDE8F08F042246
:10CB600041462846FCF728FA044628BB2846FBF72E
:10CB700002FC81460028EFD057F078F8DFF824B2A5
:10CB800082465BF8047B37B92A467A4930460BB0B7
:10CB9000BDE8F04F76E6524639464846FCF70CFAB7
:10CBA00040B92046744D29F0D3F839467348FDF753
:10CBB0009DFDA6E70134E4E7072271492846FCF70A
:10CBC000FBF9074600287AD1202128465AF031F98E
:10CBD000044670BB6B4D6C48FEF734FF21460134B0
:10CBE0002846FEF72FFF0E2CF8D10025DFF8B8916C
:10CBF000664FFDF763FDDFF8B4810C260024DFF8F3
:10CC0000B0A129466E434846FEF71CFF0123F259A6
:10CC10005F48A340013413420CBF41465146FEF722
:10CC200011FF0E2CF2D10135FDF748FD082DE4D19E
:10CC300092E702AC574D01AA56495AF0C0F80028B5
:10CC400048D0022F11D1029A072A07D8039C0D2C35
:10CC500004D80378722B13D06E2B25D00823002222
:10CC60004D493046FFF73AFF76E7FCF791FA01AA03
:10CC700044F8040B2946002001375AF0A0F8DEE7FB
:10CC80000C233B4903FB02110123D1F8F811A34007
:10CC90000B4337490C2000FB02123949C2F8F83126
:10CCA0003046FFF727FF57E7314B0C20012100FBEF
:10CCB0000233A140D3F8F83123EA0103E9E728461B
:10CCC000002402AD334F01AA32495AF078F880B1FE
:10CCD000082C03D13046FFF729FE3DE7FCF758FA50
:10CCE00001AA45F8040B3946002001345AF067F8D0
:10CCF000EDE7082CEED1029B0F2B30D8DDF80CE0CD
:10CD0000BEF1070F2BD8DDF810C0BCF10D0F26D8EF
:10CD1000059F07F16402C82A21D8069DFF2D1ED861
:10CD2000079864281BD80899642918D8884216DA0D
:10CD3000099C032C13D8C3EBC3020D4B134483F897
:10CD40008D1183F888E10C4983F889C183F88A71D1
:10CD500083F88B5183F88C0183F88E41A0E70F494B
:10CD60003046FFF78FFDF7E60875002440890B0871
:10CD7000807300244B890B08A1930B085C890B0876
:10CD800066890B086E890B0856980B087875002485
:10CD900073890B0877890B0879890B087F890B0841
:10CDA00046890B08C0A10A08E39F0B082E980B08C0
:10CDB0006C800B0810B504460748FDF7EFFCFAF746
:10CDC0007FFE20B10548BDE81040FDF7E7BC2046D6
:10CDD0000349BDE8104055E595890B089F890B086C
:10CDE000A7890B082DE9F04F8FB004460846B249D9
:10CDF00002AA59F0E4FF054640B903460246AF498E
:10CE00004120FEF7E1FB0FB0BDE8F08FAC49FAF727
:10CE100085FF064628BB02AAA74959F0D0FFFCF7B8
:10CE2000B7F90828054606D908233246A549204601
:10CE3000FFF754FEE7E7A44C94F8BC3683420CDCC1
:10CE400084F8BC56DFE731460136384637F064F8DF
:10CE500094F8BC36B342F6DCF2E7064604F2BC674F
:10CE6000F6E79A492846FAF759FF0646E0B902AABA
:10CE7000914959F0A4FFFCF78BF90828054603D91E
:10CE8000082332469249D2E78F4C94F8BD3683424C
:10CE900002DC84F8BD56B6E73046013629464CF030
:10CEA0009DFA082EF8D1F4E78A492846FAF736FFAA
:10CEB000064600BB02AA804959F081FF0028A2D093
:10CEC000FCF766F90828054603D90823324682494B
:10CED000ADE77D4C94F8A637834209DD014604F2A4
:10CEE000BC6037F05FF8294604F2BC6037F068F8A0
:10CEF00084F8A65787E779492846FAF70FFF0646D0
:10CF000018BB06AD704BDFF8B0910146A846102261
:10CF1000284693F8A67759F075FFBE4202AA80F220
:10CF20000A814946002059F04AFF10B93A466C4937
:10CF30000AE1FCF72DF9013628F8020BEDE7694C00
:10CF400095E80F0084E80F005DE767492846FAF787
:10CF5000E5FE0646C0BB5C4B06ADDFF85C9193F87E
:10CF6000A677BE4202AA80F2F3804946002059F01B
:10CF700026FF014610B93A465C49E5E0AA464FF063
:10CF80000008032228465AF03FF8284656F06EFE65
:10CF9000404502D801360435E3E79AF8000008F16D
:10CFA0000108FCF703F80AF8010BEEE7B6000446A7
:10CFB0004F4DB4423FF427AF06AB2819032219198D
:10CFC000043436F093FFF4E74A492846FAF7A6FE00
:10CFD0000746002840F0AC80DFF8EC8002AA364912
:10CFE00098F8BC6659F0EBFE00283FF40CAFFCF754
:10CFF000CFF8451E01D4AE4203DC334601223E4940
:10D0000015E72D4902AA002059F0D9FE0146002853
:10D010003FF4F9AE00260DF10C09082203A88DF8A3
:10D02000146059F0F1FF03A856F020FEB0421BD85F
:10D0300002AA2149002059F0C2FE00283FF4E3AEC5
:10D040000026037898F8BDA6B1460193564502AA7A
:10D0500019494FF0000080F2858059F0B0FE8346F8
:10D0600050B9524625496FE099F800000136FBF7A8
:10D070009DFF09F8010BD6E7A6B99BF80030303BBD
:10D08000092B0FD91E49FAF749FE38B11D495846F8
:10D09000FAF744FE70B15A461B4955E04FF00109BA
:10D0A0004FF0FF365846FCF773F8002830DA5A463E
:10D0B000164949E0B146F3E777890B084469002433
:10D0C000AE890B08B4890B0888620024BF890B085D
:10D0D000C8890B08D6890B08E2890B08F4890B086C
:10D0E000E38A0B08306A00241E8A0B08038B0B08A6
:10D0F000406A0024488A0B084D8A0B08238B0B08D2
:10D100002E7E0B08598A0B08608A0B08958A0B083B
:10D110000EAB03EB4603013623F8200C96E752468C
:10D120001F4911E033F8022B013724F8022F30E0B9
:10D130002A461C4908E01C49002059F040FE0028FE
:10D140003FF4FDAE3A4619492046FFF79BFB5AE6ED
:10D150001549002059F033FE00283FF427AF3A4626
:10D160001349F1E759F02BFE0028D8D105EBC50093
:10D17000104C082203A98230204404EB051436F039
:10D18000B5FE0198FBF712FF08EB050383F886074D
:10D1900006ABBE42C6DC454485F89E9733E600BF29
:10D1A000AA8A0B08CD8A0B0877890B08008A0B081E
:10D1B0002A8A0B0844690024154B1B682DE9F041AD
:10D1C000044688B0F3B11A6804A91846D56A6A46BD
:10D1D000A847064688B104AC6D460027DFF83C80BE
:10D1E000013735F8022B34F8021B4046FDF77EFA72
:10D1F000BE42F5DC08B0BDE8F08106492046FFF7E5
:10D2000041FBF7E7044908B0BDE8F041FFF73ABB3E
:10D21000183A0024628B0B087A8B0B08488B0B089A
:10D2200070B5054608460C4656F020FD024670B122
:10D230000C2804D12146094859F0D4FE38B12846BB
:10D24000064B074A0749BDE87040FFF71BBB03497F
:10D250000548BDE87040FDF749BA00BFEB850B08F3
:10D26000818B0B088C8B0B08B68B0B0870B50546B1
:10D2700008460C4656F0FAFC024670B1062804D166
:10D280002146094859F0AEFE38B12846064B074AF8
:10D290000749BDE87040FFF7F5BA03490548BDE806
:10D2A0007040FDF723BA00BFF8850B08C48B0B084C
:10D2B0008C8B0B08D48B0B082DE9F04307469BB0F1
:10D2C00008460C4656F0D2FC06462022002101A852
:10D2D00059F098FD36B3402E08D0402332463A49E3
:10D2E00038461BB0BDE8F043FFF7CCBA01AD04F1FE
:10D2F00040084FF0000902222146684659F084FE9A
:10D300000023102209A968468DF80290FBF790FED1
:10D31000099B0DF10202934223D1023405F8010B5F
:10D32000A045E8D109AC41220021284D204659F002
:10D3300069FD002E3CD095F85862D6B1202205F246
:10D34000592101A859F0B2FE98B105F259212046A1
:10D35000FBF79EFD23461E4A38461E49FFF792FA08
:10D3600004E01A7838461C49FFF78CFA1BB0BDE878
:10D37000F0831A4B1B79DBB9D6B901AB184E1A46AC
:10D38000083603CAA24246F8080C46F8041C1346A5
:10D39000F5D101232046124985F87932FBF778FD53
:10D3A0001048FDF757FA21460F48FDF79FF9DDE7D2
:10D3B00095F879321BB995F85832002BF3D008490B
:10D3C0002046FBF765FDEEE7E78B0B088073002432
:10D3D000258C0B088C8B0B08098C0B0888620024A9
:10D3E000D97500242F8C0B083E8C0B082DE9F74FC4
:10D3F000DFF82081834608460C4656F037FCD8F803
:10D400000070064628B1024633492046FBF7D4FD9A
:10D4100080B9394631484CF099F83149314821EA10
:10D4200007014CF093F83049304803B0BDE8F04FA5
:10D430004CF08CB823782D2B24D10134013E4FF0D1
:10D44000010A2B4B4FF000094FF0FF3553F8041B36
:10D4500051B1324620460193FBF7AEFD0028019BF7
:10D460000ABF4D460021012109F10109A9B9B9F10D
:10D470001D0FEBD122461F49584603B0BDE8F04FBF
:10D48000FFF700BA4FF0000ADBE73B431A49C8F840
:10D4900000301A4B12E01A4913E00123104AAB4046
:10D4A0001A40002AF7D007EA0302BAF1000FECD0C5
:10D4B00027EA03031349C8F80030134B002A18BFAA
:10D4C0001946124B124803EB8503D3F8A42703B087
:10D4D000BDE8F04FFDF70AB9B5840B08768C0B0850
:10D4E000BDD77718808C0B08422888E78C8C0B08F6
:10D4F0002CA20A084B890B086E8C0B08678C0B0852
:10D500004B8C0B08578C0B085E8C0B08889A0A080A
:10D51000FA7F0B084C3E00242DE9F74F0190084696
:10D520000E461746984656F0A1FB0446E8B9404D12
:10D530004048FEF787FA20460DF06CFA3B68184227
:10D5400006D020460DF078FA01462846FEF77AFA12
:10D550000134182CEFD13B6813B93748FDF7A6F812
:10D5600003B0BDE8F04FFDF7A9B802463349304695
:10D57000FBF722FD0546A8B92C46314D3148FDF791
:10D5800095F820460DF046FA10EA080F06D020461E
:10D590000DF052FA01462846FEF754FA0134192CD0
:10D5A000EFD1DDE733782D2B29D10136013C012560
:10D5B0004FF0000948F0807B48460DF03DFA2246C6
:10D5C000824601463046FBF7F7FC18BB48460DF093
:10D5D00021FA1BEA000F1DD09DB1B9F1180F02D03E
:10D5E0003B6840EA03081848C7F80080FDF75EF87A
:10D5F0005146134803B0BDE8F04FFDF777B800255A
:10D60000D6E7B9F1180F02D03D6825EA00050F48AA
:10D610003D60EBE709F10109B9F1190FCCD13246B0
:10D620000B49019803B0BDE8F04FFFF72BB900BFDD
:10D630002B840B089A8C0B08A48C0B08B5840B0860
:10D640002C840B08AB8C0B085E8C0B086E8C0B08C3
:10D650004B890B0840F20223004A5DE7A8390024F9
:10D660006FF07F43004A57E7A039002410B5044605
:10D670002AF0D0FA28B920460449BDE81040FFF747
:10D6800001B90348BDE81040FDF730B8B68C0B086F
:10D69000C58C0B08074B10B50446D3F87C0237F055
:10D6A000E3FB28B920460449BDE81040FFF7EAB87B
:10D6B00010BD00BF80730024D08C0B0870B50546E8
:10D6C00008461646FBF764FD0D4B041E1A780EDB68
:10D6D000944205DA21460B48FDF708F8204670BD54
:10D6E0002EB1FF2C03D10848FDF700F8F6E7013A08
:10D6F000064928464FF0FF34FFF7C4F8EEE700BFB5
:10D70000481C0020E68C0B08F78C0B080A8D0B08D0
:10D710002DE9F04F074691B082480E46824DFCF746
:10D72000E5FF002381494024062285F884323046F3
:10D7300001230978C5F880D285F8854208F0FCF805
:10D740000A20F9F799F995F884320C2BDAB240F2F5
:10D75000E4809DF80C60FE2E2CD0FF2E15BF0F2408
:10D76000152400250125944240F0D780611E6846AB
:10D77000C9B243F099FD04F140030DEB030414F822
:10D78000413C834240F0C4806A1E9DF80D30012A5E
:10D7900012D903F01F075C0961376548FCF786FF63
:10D7A000022D39D0013C042C34D8DFE804F00B2DD5
:10D7B0002F3331000225D6E79DF80E701E469DF8E6
:10D7C0000F40EAE75B486C464FF00008DFF8BC9179
:10D7D000FCF7E4FFDFF8B8A1DFF8B8B15648FCF772
:10D7E00065FF08F1010814F8011B4846FEF72AF905
:10D7F000B8F10C0F16D00AFB08F3B3F1553FF0D87F
:10D800005846FCF753FFECE74C48DCE74C48DAE7B6
:10D810004C48D8E74C48D6E700230DF11F008DF89F
:10D820003F30D0E7FCF74AFF022D3AD064223B4656
:10D830004648B6FBF2F102FB1162C9B2D2B2FCF764
:10D8400055FF85F001035B42DBB2012B59D8404AFA
:10D85000404B9DF81010404800290CBF1146194656
:10D860003E4EFCF743FF9DF811103D4B3D4800290B
:10D870000CBF31461946FCF739FF022D41D19DF806
:10D8800012403948FCF712FF8CB1FF2C1FD00A233D
:10D890003648B4FBF3F103FB1142D2B2FCF726FF8A
:10D8A00008E03A4631463248FCF720FFCFE73046E1
:10D8B000FCF774FF9DF813402E48FCF7F7FE44B1C7
:10D8C000FF2C21D021462C48FCF710FF04E02B4808
:10D8D000EEE72248FCF762FF0DF1130500241F4E0E
:10D8E0001F4FDFF8988015F8013F7BB1FF2B14BF65
:10D8F0003A464246214601342148FCF7F7FE042C03
:10D90000F1D111B0BDE8F08F1C48E3E73246F1E7F2
:10D910001C493846FEF7B6FFF3E71B48FCF73EFF0D
:10D92000EFE700BF508D0B0880730024481C0020D7
:10D93000618D0B086C8D0B08928D0B08738D0B0895
:10D940007B8D0B08838D0B08F9810B08A48D0B08C8
:10D95000398D0B08308D0B08DB8D0B08408D0B08C3
:10D9600071970B08F28D0B08F98D0B080D8E0B08C3
:10D97000C08D0B08158E0B08E39F0B08448D0B0818
:10D98000258E0B08308E0B08408E0B08447E0B084A
:10D99000ABAAAAAA089A0B082DE9F84307460C4639
:10D9A000DFF8A090204656F061F9064658B91D4BA5
:10D9B0001D481A781D4B03EB8203D3F83417BDE8DA
:10D9C000F843FCF793BE024649462046FBF7F4FABB
:10D9D00060B1DFF86080002558F8041BB1B9224619
:10D9E00038461349BDE8F843FEF74CBF114C124DC1
:10D9F0001248FCF75BFE54F8041B19B12846FEF7E9
:10DA000021F8F8E7BDE8F843FCF758BE3246204657
:10DA10000135FBF7D1FA0028DED1024B084C1D700E
:10DA2000C0E700BF2C380024498E0B08889A0A08EA
:10DA30004B890B08C0A10A082C840B08AB8C0B087F
:10DA4000A1930B08B5840B0838B50D460446052292
:10DA500019492846FBF7B0FA68B9184B93F85020DB
:10DA600022B9012183F8512083F850101448BDE8F1
:10DA70003840FCF793BE032212492846FBF79CFA74
:10DA8000A0B90E4D95F8503063B195F851304BB1B7
:10DA90000D492046FEF7F6FE002385F8503085F844
:10DAA000513038BD0948FCF779FEF5E720460849B2
:10DAB000BDE83840FEF7E6BEC8960B088862002431
:10DAC000538E0B081A980B08698E0B08A08E0B0852
:10DAD000B48E0B0870B5194C054694F850307BB1E4
:10DAE00094F8513063B11649FEF7CCFE284615492B
:10DAF000FEF7C8FE002084F8500084F8510070BD85
:10DB0000114B93F87922B2B193F858229AB903F2E3
:10DB1000592203F5227503F279261068083252F86B
:10DB2000041C2C46B24203C42546F6D1012283F8D8
:10DB3000C32209F0DFFA0120E1E700BF8862002478
:10DB4000698E0B08C38E0B08807300242DE9F04FFB
:10DB500080468BB008460D4656F088F8024670B3F2
:10DB6000A4492846FBF728FA044640BBFCF7A6FD6B
:10DB7000A14DA248A24FFCF711FEA24E1420DFF8DF
:10DB8000CC824BF03FFCE11004F007023846013133
:10DB9000FDF758FF2B7F6A7F06EB8303D3F844130E
:10DBA0004AB19948FCF7A2FD01342435102CEAD182
:10DBB0000BB0BDE8F08F4046FCF798FDF4E728462F
:10DBC00005AA924959F0FBF8054620B901464120C3
:10DBD000FCF759FEECE78E49FAF7A0F820B98D4919
:10DBE0004046FEF74FFEE3E700248B4E2746013701
:10DBF00031682846FAF792F8002808BF34460B2F00
:10DC000006F11006F3D154B984492846FAF786F88C
:10DC100028B12A4682494046FEF734FEC8E7002074
:10DC200005AA7A498DF8130059F0C9F80546002C69
:10DC300039D078B1FBF7ACFA461E08D4A37A9E42DD
:10DC400005DAE26842B101238340134204D12A4637
:10DC50007449E0E7744DFAE7E088002744F0B6F92C
:10DC6000724903970979D0E90223002918BF1A469F
:10DC7000217A637A06FB013302EB030B12F903A04E
:10DC800005AA6249002059F09AF88146A0BB0123F9
:10DC9000674944B39BF900202046CDE90031314665
:10DCA000FAF7AAFB84E768B10DF11301FBF74AFA12
:10DCB00028B19DF813603046F6F746FB20B92A4696
:10DCC0005C49A8E7584DFAE73046A346F4F77EFDD5
:10DCD0008246304608F0F6FB03903046264608F0B0
:10DCE00029FC0746CCE7CDE90031524639469DF87C
:10DCF0001300FAF7CDFB5BE74549FAF70FF8054645
:10DD000000282FD1ACB1F6B24B4F6AB23146207920
:10DD1000F4F730FD00283FF44BAF02882946037822
:10DD2000384601350093C2F30323120BFCF7DEFCE7
:10DD3000EBE738687979404C6AB2F4F763FD002864
:10DD40003FF436AF02882946037801352046009318
:10DD5000C2F30323120BFCF7C9FC102D3868797944
:10DD6000EAD125E735494846F9F7D8FF00283ED0E3
:10DD70004846FBF70DFA054642B26CB1F1B2207984
:10DD8000F4F7F8FCD8B9CDF80090731C22682C4940
:10DD90004046FEF777FD0BE7EBB2386879790F2B39
:10DDA00009D99DF8133027491A09CDF8009003F0DE
:10DDB0000F034032ECE7F4F725FD0028F1D006AF61
:10DDC00028463946FBF776F808A95046FBF772F863
:10DDD000554549D06DB2002C3AD08BF8005008ABB5
:10DDE0000097721C21681848FCF780FCE0E64FF0B1
:10DDF000FF35E4E7E18E0B08E0010024E68E0B0816
:10DE0000FC8E0B08889A0A086B900B0877890B0820
:10DE1000B5840B080D8F0B088405002443920B0872
:10DE2000218F0B08308F0B08A1930B088862002408
:10DE3000C5A60408408F0B08528F0B08A68C0B0850
:10DE4000738F0B08968F0B08BE8F0B082C840B0862
:10DE50009DF81320039B11090C489D7002F00F02DE
:10DE600008AB40310097BFE734B108AB721C2168A2
:10DE70000748FCF73BFC9BE69DF8132008AB0548E0
:10DE8000110902F00F024031F3E700BFE18F0B08E8
:10DE900009900B0824900B082DE9F04F07468DB030
:10DEA00008460D4655F0E2FE044630B90146012011
:10DEB0000DB0BDE8F04FFCF7EDBD0246A84928467D
:10DEC000FBF77AF830B9A74938460DB0BDE8F04FF6
:10DED000FEF7D8BC2246A4492846FBF76DF8002877
:10DEE00059D1FCF7EBFBA14FA1480E25DFF8C092FA
:10DEF000FCF754FCDFF8BC8217204BF083FA17F9CB
:10DF0000016B002E38D031464846FDF79BFD0023BB
:10DF10001C46A10030460393013489B208F040FB4F
:10DF2000834608F0C5FB02788246039BD2B10BB949
:10DF3000FCF7C4FB9BF806109AF800309AF8012011
:10DF400001F0020108EB8303CAB18A4800928A4AB1
:10DF5000D3F84433002908BF024621468748FCF71E
:10DF6000C5FB0123042CD4D113B98548FCF716FC5A
:10DF7000013D15F0FF05C2D10DB0BDE8F08F7D4821
:10DF80007D4AD3F84433002908BF024621467D4824
:10DF9000FCF7ACFBE5E7002407AA764928468DF894
:10DFA0001B4058F00CFF18B93846FEF781FCE3E738
:10DFB0000DF11B01FBF7C6F881460028F4D09DF84F
:10DFC0001B502846F6F7C0F920B96F493846FEF7CE
:10DFD00059FCD1E72346DFF8E0814FF0FF3403EB33
:10DFE000430218F8022095420BD0002C02DA002AD6
:10DFF00008BF1C460133152BF1D1002C16DA6349FA
:10E00000E4E71C4607AA5B49002058F0D8FE064604
:10E01000002800F097805249F9F780FE38BB04468B
:10E020005B4FDFF85481DFF8949117E04FF000095F
:10E03000E8E73068F5F776F9B1797379024611F0BF
:10E04000020F96F807A04FEA930348460CBF3946E3
:10E050004146013300915146FCF748FB0134284604
:10E06000214608F043FA06460028E2D184E74FEA49
:10E07000151A0222474930460AF1400A05F00F0BF3
:10E08000FAF79AFF002845D10390B01CFBF780F8FF
:10E09000039902460491013128460592039108F044
:10E0A00025FA059ADDE9031338B95B4652463A4929
:10E0B00000963846FEF7E6FB5EE7C0799042E9D16C
:10E0C0001F466300B9F1000F31D01A194244567847
:10E0D000013E7A1C23440AAC284614BF294600217D
:10E0E00008EB030208F803107B1C39465370FF232A
:10E0F00093702246FAF7EEFE08AA31462846FAF750
:10E10000E9FEB74216D108AB5A4651462348FCF700
:10E11000EDFA31E722493046F9F700FE20B15B46BF
:10E12000524620490096C4E74FF0FF37C9E74FF049
:10E13000FF36CEE708AB5A4651461B480094FCF721
:10E14000D5FA19E704EB4404184B02462846A044CC
:10E150000093012398F80110FAF7E2F90CE700BFE9
:10E16000B5840B080D8F0B08E18E0B08B8090B085E
:10E1700040900B0877890B08D7810B0860900B083B
:10E1800081900B0872900B0887900B089E900B08EB
:10E19000A1930B08C7900B08CA900B081C910B08A1
:10E1A000A68C0B08F6900B083A910B08C5A604083C
:10E1B00059900B08889A0A08C8270024B2900B08C7
:10E1C0002DE9F04F89B0074608469D4905AA58F049
:10E1D000F6FD054630B901464120FDF7ADFB09B01B
:10E1E000BDE8F08F9749F9F799FDDFF8A082044662
:10E1F00000283BD19448954DFCF7D0FA944E14205A
:10E20000DFF88C924BF0FEF829683046AA8801F1BD
:10E210002741AB79B2FA82F201F57E0108EB830364
:10E22000C2F11F02890AD3F844334131FDF70AFCD9
:10E23000E97911B14846FDF705FC0134FCF73EFAD7
:10E240000835902CE0D17E4905AA002058F0B7FD92
:10E250008049F9F763FD0028C1D138467949FFF7B5
:10E260001BFE78493846FFF771FCB8E7002408F533
:10E27000F27A1AF83430284608EB8303D3F8449333
:10E280004946F9F74BFD40B101342C2CF1D12A4617
:10E2900071493846FEF7F6FAA1E705AA684958F031
:10E2A0008EFD064688B3FAF773FF054608EBC408EF
:10E2B0004FEAC40B98F8EA314BBB002D29DC0AEB7E
:10E2C0000B03588893F804A093F8058043F07EFE72
:10E2D000EBB203FB0A88D0F808A00093002E00F0F0
:10E2E0009A803378002B00F0968006A93046FAF722
:10E2F00029FF002800F08C809DF818500DBB57486E
:10E300000AF80850FCF74AFA69E70546CEE7002DFF
:10E3100005DD012B1A4638BF0122954209DD012B8C
:10E320004FF001024E49384638BF0123FEF7D6FBB5
:10E3300055E705AA42490020013D58F040FD064638
:10E34000BDE72846F6F700F8814600285CD02B0987
:10E350000AF80850434F4FF000084033029305F08D
:10E360000F030393BB790026012B38BF01230193D0
:10E3700097F804B097F805A0788843F027FE06FBCD
:10E380000BA38268D15CA94222D1444504D10099F3
:10E39000B1421DD00021D1545FFA86FB32485FFAAA
:10E3A00088FADDE90212FDF74DFB59465046FDF7AC
:10E3B000C3FF444509D12D48FDF744FB504659465B
:10E3C000FDF7BAFF2A48FDF73DFB2A48FCF7E6F9BE
:10E3D0000136019BB342CBDC08F101080837B8F1E4
:10E3E0002C0FBFD1D9F80010B9F8042001F1274152
:10E3F0002148B2FA82F201F57E01C2F11F02890AB8
:10E400004131FCF773F9EAE63846FEF751FAE6E6E1
:10E4100032461A493DE71AF80830013573B11A0936
:10E42000174903F00F0306A84032FAF7CDFC06ABFC
:10E430002A4649461348FCF759F9D0E6124BF7E74C
:10E4400077890B08E18E0B0860910B08481D0024AA
:10E450009E910B08A9910B08AD910B08CF910B0869
:10E46000C9910B086C9C0A08E1910B08F0810B081C
:10E4700005920B081F990B080F920B082B920B08A3
:10E4800040810B0847920B08827D0B08889A0A0886
:10E49000E29F0B0820B10078B0FA80F04009704785
:10E4A000012070472DE9F74F81460846FFF7F2FF3C
:10E4B0000E46054670B1002401A9204601344BF0F8
:10E4C000D9F801464846FFF7EDFF122CF4D103B00E
:10E4D000BDE8F08F0846FAF75BFEC4B2112C72D883
:10E4E0003D4D701CF9F747FF3C4E05EB4408834651
:10E4F000670098F8C4A2B8B9AAF102014B424B4197
:10E500003D4495F8C422B25C002B55D095F8C53235
:10E51000192040F2EE2100FB03132146304803B0DE
:10E52000BDE8F04FFCF7E2B80178304658F081FCC6
:10E5300080B1032C2B49A0EB060394BF00220122DB
:10E5400002EB42020A4452FA83F393F818A8BAF194
:10E55000030F05D1484603B0BDE8F04FFEF7A8B958
:10E560005846F9F708FFF0B1BAF1020FF2D1FAF705
:10E570000FFE40F6CA0380B29842A8BF184640F288
:10E58000EE239842B8BF18461923A0F2EE20B0FB44
:10E59000F3F088F8C502AAF1020253425341EA1986
:10E5A00082F8C4A2ACE7BAF1020FF4D1484603B036
:10E5B000BDE8F04FFEF7BAB921460B4803B0BDE8FD
:10E5C000F04FFCF793B811232A460849484603B098
:10E5D000BDE8F04FFEF782BA807300246C1E0B0872
:10E5E0005B920B08889A0A086B920B0878920B08CA
:10E5F0002DE9F041054686B008460F46FFF74AFF71
:10E60000064640B100235C4901201A4606B0BDE829
:10E61000F041FCF7F7BA0846FAF7BAFD13280446AA
:10E6200000F3A08006258DF81760544E4543781CF2
:10E63000F9F7A1FE074660B1FAF7AAFDC0B213F0E0
:10E64000CBF930B17319027983F8182601238DF8BC
:10E6500017303846F9F78FFE074668B1FAF798FD8C
:10E660000D2809D8062303FB046383F819069DF8D7
:10E67000173001338DF81730DFF8FC80A91C0DF13D
:10E68000170238464144FAF787FDF9F774FE07464A
:10E6900068B1FAF77DFD012809D89DF817300622E8
:10E6A000013302FB04628DF8173082F81C063846ED
:10E6B000F9F761FE80B1FAF76BFDC0B213F08CF987
:10E6C00050B19DF817300622017902FB0462013334
:10E6D00082F81D168DF817309DF817200623042A9E
:10E6E0002FD103FB04630022A3F81C2606251CF08F
:10E6F00025FC05FB046595F8180614F0ABFD95F8AC
:10E700001B1695F81A7619234FF46172804695F816
:10E710001D0613FB012613FB072714F09BFD43790D
:10E72000214698F80520039395F81C361448009765
:10E73000CDE9016395F81936FBF7D8FF06B0BDE8BF
:10E74000F081052A05D103FB0463002283F81D260E
:10E75000CCE7062ACAD0002308EB050248F80530AA
:10E760009380C3E7132332460649284606B0BDE826
:10E77000F041FEF7B3B900BFA0680024886200240E
:10E78000937F0B08C9910B082DE9F04F80468DB09F
:10E790000846FFF77FFE054640B10023624901208D
:10E7A0001A460DB0BDE8F04FFCF7A4BA09AF0990C6
:10E7B00007915E49C7E9010007A858F0D3FA064659
:10E7C0004AF034FE431C04460CD12B460A2208A909
:10E7D0003046FAF72DFC089B1B781BB9C4B2132CEA
:10E7E00015D944B2A31CDBB2012B0AD94E4E00232B
:10E7F00096F90420A24200F08C8001330C360A2BDB
:10E80000F6D14046FEF754F80DB0BDE8F08F333432
:10E8100064B2E7E7002302250A221946FAF708FC4A
:10E8200009904FF0000BDFF80491DFF808A149468A
:10E8300007A858F097FA20B3FAF7AAFC3C4A00233D
:10E8400052F8041B884222D1DBB20AEB8302D2F8D1
:10E85000A421904215D1BBF1020F22D0BBF1030FCE
:10E8600024D05A1EBBF1010FD2B215D00B2A03D807
:10E870008DF829300135EDB20BF1010BBBF1040F1E
:10E88000D5D1052D18D84046FEF750F8BCE7013326
:10E89000102BD5D10023D8E7052AEDD88DF82A30E2
:10E8A000E8E7052BE8D88DF82C30E3E79A1E0D2A0F
:10E8B000E2D88DF82B30DDE797E8070086E80700FF
:10E8C00020464AF0C1FE1B4A9DF82B10034602EB7E
:10E8D0008101D1F8A41104919DF82C1002EB810163
:10E8E000D1F8A41103919DF82A1002EB8101D1F80F
:10E8F000A41102919DF8291002EB81020021D2F8A7
:10E90000A42108460192099A00920B4AFBF7DAFE0D
:10E910007AE7064907A88DF8284058F023FA00281E
:10E920007FF478AF01257CE76067002477890B08C6
:10E930002C9C0A08889A0A08AC7F0B082DE9F04F36
:10E940000346A1B00846FFF7A5FD054628B11846C5
:10E9500021B0BDE8F04FFDF7E9BFFF23DFF8C0921B
:10E9600007464FF0FF388DF82830D9F87C320B90ED
:10E9700093F83820ADF830000D908DF838200F90C6
:10E98000ADF8400011930991CDE90500934909A81C
:10E9900058F0E8F9044618BB01460AAC904F0B0149
:10E9A00090481A57002310F9016BB24240F0D28010
:10E9B0004E1C10464AF048FE024631463846FBF7E8
:10E9C00095FE022E4FF00101E9D19DF938A09DF985
:10E9D0002830534540F0C5808348FBF787FE4DE063
:10E9E0002378002BD2D0032FD4BF00260126062F78
:10E9F00000F2A980DFE807F0044750910447500077
:10EA0000042F10D079492046FAF7FAFA58B14FF49A
:10EA100080600CF065FA002800F0B58190F90400E0
:10EA2000012306930AE072492046F9F777F970B995
:10EA3000D9F87C3293F93800042F22D0119B11931E
:10EA400020AB03EB061606F8580C01379EE720466C
:10EA50004AF0ECFC0028EFDA01230A2212A9204632
:10EA6000FAF7E6FA40B2002803DB129B1B78002B72
:10EA7000E2D02246711C5F48FBF738FE21B0BDE8AA
:10EA8000F08F0023DBE72046FAF782FB20AB03EB95
:10EA9000061646F8540CD8E757492046FAF7B0FA5C
:10EAA000B0F1000A5549204618BF4FF0010AFAF7A5
:10EAB000A7FA08B14AF0020A3301DFF868C10793E8
:10EAC00020AB03EB0616BCE80F0006F850AC12AE04
:10EAD0000DF1480A0FC6BCE80F000FC6BCE80F00D6
:10EAE0000FC69CE8030086E803000026B346DAF868
:10EAF0000010204658F0C4FA10B19AF804301E43B2
:10EB00000BF1010B0AF1080ABBF1070FEFD1079BCC
:10EB100080336B4403F84F6C97E739492046F9F787
:10EB2000FDF8A0B137492046F9F7F8F800288CD055
:10EB30002046FAF72DFB0328804686D90146324845
:10EB4000FBF7D4FD9AE722460821304894E70123D9
:10EB500005937AE701330A2B7FF425AF01312C4866
:10EB60008AE70B9B1BB9AAF11402554255410023B9
:10EB70005F1CE368002B62D194F900B058460CF09A
:10EB800081F9D4F8049018B10668002E40F08B800B
:10EB9000B9F1000F237A14BF4E464FF46146666008
:10EBA00023B91C48FBF7A2FD03232372627A2AB122
:10EBB000394619480792FBF799FD079A0292584681
:10EBC000237ACDE9006300231A4619460CF0A2F916
:10EBD000E06048BB39461148B2E700BF77890B08AF
:10EBE000FC920B081C880A0819930B089B920B08CF
:10EBF000A6920B08AA920B08C5920B089E970B08C9
:10EC000040890B08A68C0B08C8920B08E0920B08F1
:10EC100007930B0832930B084D930B0868930B086E
:10EC200080730024A8A20A0858493346584A594814
:10EC3000B9F1000F18BF0A463946FCF703FF022F4F
:10EC400004F110044FF0010392D1119E0D9F4DB1BC
:10EC50005148FBF7A3FD33681B6A1BB13A464F4985
:10EC600030469847059B002B50D04D49474BBAF191
:10EC7000140F18BF19464B48FBF738FDBAF1140FB3
:10EC800009D1059B002B43D03368DB691BB10022FF
:10EC9000454930469847069B002B43D10022314618
:10ECA00038464AF0DBFBE660B9F1000F2CD049464C
:10ECB000304601F065FE3D4AB36839463C48FBF7F3
:10ECC00015FD94F80890B9F1000F0CD032799145F8
:10ECD00009D04B4639463748FBF708FD33684946AB
:10ECE00030469B699847637A23B172793946324836
:10ECF000FBF7FCFCF36A002BA1D039462F48FBF749
:10ED0000F5FC0023F3629AE7204AD5E71F49B2E7F2
:10ED1000B8F1000FBFDB3368DB69002BBBD0424684
:10ED20002749B6E7DFF89C900025DFF89CA04FF05C
:10ED3000030B07F0A9F80520F7F79EFE9AF80030BC
:10ED4000AB42ABD919F8014FC4B1204607F0F2FB32
:10ED5000804698B12046F5F7F7FA0446EBB210B1B9
:10ED600080F806B0C37120460121F4F77BFD98F8C6
:10ED700006302046DB0703D5F4F7ACFB0135DDE7B1
:10ED8000F4F7A2FBFAE74FF0FF3049E6A1930B0836
:10ED900080920B0884930B083A940B0881090508AC
:10EDA0008E920B0863940B088F83040889920B08DA
:10EDB000A2930B08C7930B08EA930B0821940B0846
:10EDC000498104082F310024481C00202DE9F0431C
:10EDD00080468BB008460F46FFF75CFB044640B107
:10EDE00000235E4901201A460BB0BDE8F043FCF752
:10EDF00005B80846FAF7CCF91D28054600F3A580AA
:10EE00000A268DF827404643781CF9F7B4FA10B16A
:10EE100001238DF82730F9F7AEFA514C074668B157
:10EE2000FAF7B6F90D2809D80A2303FB054383F83E
:10EE3000E8029DF8273001338DF82730DFF81C9168
:10EE4000711C0DF1270238464944FAF7A5F9F9F784
:10EE500092FA074668B1FAF79BF9232809D89DF87A
:10EE600027300A22013302FB05428DF8273082F851
:10EE7000EB023846F9F77FFA074668B1FAF788F9E6
:10EE80000D2809D89DF827300A22013302FB0542DC
:10EE90008DF8273082F8EC029DF82730062B0CD035
:10EEA000002309EB0602404649F8063053601381FF
:10EEB0000BB0BDE8F043FDF739BD0A260023384604
:10EEC00006FB0546A6F8EE32A6F8F032F9F753FA3B
:10EED000074618B1FAF75CF9A6F8EE023846F9F7DA
:10EEE0004AFA30B1FAF754F90A2303FB0543A3F8B1
:10EEF000F0021C4B4FF0FF324FF461705A600A234E
:10EF000003FB0542B2F8F0320693B2F8EE320593F5
:10EF100092F8EC32049392F8EB320393192392F8AF
:10EF2000EA1213FB0101029192F8E91213FB0103AB
:10EF300000210193084692F8E8320B4A00932B46D1
:10EF4000FBF7C0FB0BB0BDE8F0831D232246074949
:10EF500040460BB0BDE8F043FDF7C0BD6876002425
:10EF60008073002478050024C97F0B08C9910B0821
:10EF70002DE9F14F06460D46DFF890B12846FFF720
:10EF800089FA074640B10023594901201A4601B0C9
:10EF9000BDE8F04FFBF794BF052256492846FAF723
:10EFA0000BF860B9524B00221A601A611A621A6398
:10EFB0001A641A651A661A6701B0BDE8F08F042258
:10EFC00059462846F9F7F8FF04462846002C42D156
:10EFD000F9F7D1F907460028EED054F047FEDFF8E4
:10EFE00030A15FFA80F85AF8049BB9F1000F07D1FD
:10EFF0002A464149304601B0BDE8F04FFDF742BC1A
:10F000004246494638460134F9F7D6FF844600287F
:10F01000E9D1374A034600211546013342F8101B57
:10F02000082BFAD1354B03EBC40257682FB9494678
:10F030003348344DFBF75AFBA0E713F834E0F445AE
:10F04000F5DA07EB0C1305EB0C140CF1010C0FCBEC
:10F0500084E80F00F3E7FAF79BF8072804463DD849
:10F060002846F9F788F9074658B3F8F7F5FE204B1C
:10F07000012503EB041383ED000A3846F9F77BF909
:10F08000074638B1F8F7E8FE194B013503EB0413D6
:10F0900083ED010A3846F9F76EF9074638B1F8F7FB
:10F0A000DBFE134B013503EB041383ED020A3846F4
:10F0B000F9F761F938B9304601B0BDE8F04FFDF716
:10F0C00035BC0546D9E7F8F7C7FE094B032D03EB1E
:10F0D000041383ED030A3FF456AFECE707233A46E7
:10F0E0000949304601B0BDE8F04FFDF7F7BC00BF5D
:10F0F0003C38002440890B084B890B0828880A08F3
:10F100005C890B08A1930B08C9910B0846890B0871
:10F11000C0A10A082DE9F34105460846FFF7BAF9F0
:10F120000C46074640B10023334901201A4602B07D
:10F13000BDE8F041FBF75EBF30492046F8F7EEFD31
:10F1400070B904222C4B4FF47A704FF4FA61013AF3
:10F150001880598003F10403F9D102B0BDE8F081B1
:10F160002046FAF715F80328064641D82046F9F755
:10F1700002F9074698B1FAF70BF84FF00108044678
:10F180003846F9F7F8F820B1FAF702F8B8F1000FAD
:10F1900009D1284602B0BDE8F041FDF7C7BB40F2F7
:10F1A000EE248046ECE7A4F2EE2240F2DC539A42D1
:10F1B00003D8A0F2EE229A420AD940F6CA0340F2DE
:10F1C000EE220F49284602B0BDE8F041FDF786BCAB
:10F1D0000C4B00210C4A03EB8603A3F81444A3F85C
:10F1E00016043346CDE900400846FBF76BFAB4E756
:10F1F00003233A460549E5E79477002440890B0844
:10F2000086940B088073002400800B0878920B080A
:10F21000F0B5074689B008460E46FFF73BF90546AC
:10F2200040B100231A4901201A4609B0BDE8F04058
:10F23000FBF722BF0846F9F7ABFF1F2804461DD88D
:10F240003046F9F798F80146204636F013F878B1C1
:10F2500003AE0F48314600EB84004AF0A1F9234683
:10F260000C4A294628460096FBF72CFA09B0F0BD57
:10F27000384609B0BDE8F040FDF71ABB1F232A4607
:10F280000549384609B0BDE8F040FDF727BC00BF8E
:10F29000A477002411800B08C9910B08F0B507462C
:10F2A00085B008460E46FFF7F5F8054640B1002345
:10F2B0001D4901201A4605B0BDE8F040FBF724BF08
:10F2C0000846F9F765FF0F28044623DC3046F9F7B6
:10F2D00052F80146204636F0A7F8A8B104F1200202
:10F2E000124B2946284603EB820393F82724029207
:10F2F00093F826240192B3F824340D4A0093234650
:10F30000FBF7E0F905B0F0BD384605B0BDE8F040C8
:10F31000FDF7CEBA0F232A460649384605B0BDE8A8
:10F32000F040FDF7DBBB00BF24780024807300248D
:10F330001B800B08C9910B08F0B5054685B008463F
:10F340000B46FFF7A7F8044640B100231B490120F4
:10F350001A4605B0BDE8F040FBF71CBF01AE184FE0
:10F360006A461749184657F02AFD88B1032C04D184
:10F370002846FDF7DBFA05B0F0BDF9F709FF6A464C
:10F3800046F8040B39460020013457F018FDECE72D
:10F39000032CEDD1039FDDE901463A463146E0B248
:10F3A00036F07CF818B92846FDF782FAE3E73B46C9
:10F3B000324621460348FBF799F9DCE7A47700249D
:10F3C00077890B082D800B08F0B506468BB00846F0
:10F3D0000D46FFF75FF8044628B300233E4901209D
:10F3E0001A460BB0BDE8F040FBF76EBF2D2903D0E5
:10F3F000A1F13003092B49D8052C05DD30460BB0AF
:10F40000BDE8F040FDF792BA2846F9F7C1FE0AAB15
:10F41000621C03EB440424F80C0C15F8013F303B4C
:10F42000092BFAD9144629780029DFD1062CE5D119
:10F43000BDF81C20BDF91C30072ADFD8BDF91E50CD
:10F44000A5F5FA7292B2B2F5FA6F18D8BDF920702C
:10F45000A7F5FA7292B2B2F5FA6F10D8BDF922C0D0
:10F4600065450CDC67450ADBBDF924E00EF164025A
:10F4700092B2C82A03D8BDF92640112C11DD1749D4
:10F4800030460BB0BDE8F040FDF7FCB9202902D1B1
:10F4900001352246C6E730460BB0BDE8F040FDF727
:10F4A00007BA0C200E4A64B200FB03220846A2F8F9
:10F4B000FC51A2F8FE71A2F800C282F802E282F8C2
:10F4C0000342084A0095CDE903E4CDE9017CFBF74E
:10F4D000F9F80BB0F0BD00BF787500247F890B08E8
:10F4E0008073002441800B082DE9F04F074689B056
:10F4F00008468B46FEF7CEFF054640B100234D4936
:10F5000001201A4609B0BDE8F04FFBF7FFBF4A4B98
:10F51000084693F8BCA693F8BD9693F8A687F9F72A
:10F5200037FE092804467BDC06268DF81F50414D26
:10F5300046430BF10100F8F71EFF834638B1F9F797
:10F5400027FE0D2803D80123A8558DF81F305846F3
:10F55000F8F711FF834660B1F9F71AFE504508D855
:10F56000062303FB045358709DF81F3001338DF8B8
:10F570001F305846F8F7FFFE824660B1F9F708FEE3
:10F58000484508D8062303FB045398709DF81F30A4
:10F5900001338DF81F305046F8F7EDFE814660B11B
:10F5A000F9F7F6FD804508D3062303FB0453D87012
:10F5B0009DF81F3001338DF81F30311D0DF11F02F2
:10F5C00048462944F9F7E8FD9DF81F30062B09D07D
:10F5D0000023AA193846AB51938009B0BDE8F04F1B
:10F5E000FDF7A4B963434FF461761921EA18507905
:10F5F00011FB00600590107911FB00610491D17836
:10F600000391917802910021527808460192EB5CB7
:10F610000A4A00932346FBF755F809B0BDE8F08F7E
:10F6200009232A460649384609B0BDE8F04FFDF7E0
:10F6300055BA00BF303A0024886200248B800B0842
:10F64000C9910B082DE9F74F05460846FEF722FF42
:10F650000B46044618B9334A92F814752FB9284658
:10F6600003B0BDE8F04FFDF723B92646DFF8C89098
:10F67000DFF8C8A001AA2C49184657F0A0FB10B922
:10F6800006F00EFC08E056B9012201462846FEF7B6
:10F6900015F8421C04461AD103B0BDE8F08FF9F703
:10F6A00077FD2F28834636D80FB106F0EDFBBBF16E
:10F6B000060F13D01D4901235FFA8BF20978E0B2DF
:10F6C00006F03AF9002759464846FBF70FF801AA19
:10F6D00015490020013657F072FBD0E7DAF8003008
:10F6E0001B0114D5FF2C0ED0E1B22846FEF710F80E
:10F6F000E8E701372846FEF70BF8F9B298F8002042
:10F700008A42F6D8DEE70027DFF82080F5E70848D0
:10F71000FBF744F8D6E72F2206492846FDF7B2F852
:10F72000D5E700BF8073002477890B08481C0020B0
:10F73000B68C0B08A5940B0894940B08643700242E
:10F740002DE9F74307460846FEF7A4FE0B4604469C
:10F7500028B1384603B0BDE8F043FDF7E7B801AA89
:10F760002E491846264657F02AFBA0460546DFF8E4
:10F77000AC9065B92A4B3246A1B2D3F87C024CF06A
:10F7800045FD68BB27493846FDF77CF828E0B8F10D
:10F79000000F06D0B8F1010F25D03846FDF7C6F8A6
:10F7A0001EE0284654F062FA1F49064602462846E3
:10F7B000F9F702FC50B332461C492846F9F7FCFB26
:10F7C00030B332461A492846F9F7F6FB10B33246F1
:10F7D00018492846F9F7F0FBF0B13846FDF768F80C
:10F7E00003B0BDE8F083B31E294638465A425A4159
:10F7F000FDF764FF421C0446F2D001AA49460020EE
:10F8000008F1010857F0DBFA0546B2E74646F4E78F
:10F810000126F2E70226F0E70426EEE777890B08D7
:10F8200080730024D1940B08C5940B08C8940B086E
:10F83000CB940B08CE940B082DE9F743804608467D
:10F84000FEF728FE0B46054628B14046FDF76EF848
:10F8500003B0BDE8F08301AA2C4918462F4657F0A3
:10F86000AEFA2E460446DFF8A4907CB9022DECD106
:10F87000A7F57A73B3F57A7F21D94FF4FA634FF481
:10F880007A7223494046FDF729F9E1E74DB1012D90
:10F8900010D001AA49460020013557F090FA0446DD
:10F8A000E3E7012221464046FDF708FF431C0646D8
:10F8B000EFD1CDE72046F9F76BFC0746E9E7154B9A
:10F8C000B8B21B685B689847FCEEC07AFF2E124BFB
:10F8D00017EE902A0AD11149B6EEC00A0978A14262
:10F8E0000FDC11460E48FAF701FFB1E703EB860380
:10F8F00031460C48B6EEC00A83ED000AFAF7F6FE70
:10F90000A6E70134A3EC010AE9E700BF77890B08F9
:10F91000DF950B088C23002098780024481C0020D9
:10F92000FC940B08EF940B08F8B507460846FEF761
:10F93000B1FDD0B1204BD3F8C46001363046344617
:10F940000BF07AF80546F0B90134192CA8BF002451
:10F9500020460BF071F80546A8B9B442F4D13846F8
:10F960001649BDE8F840FCF78DBF0846F9F710FCD2
:10F9700004460BF061F8054628B921461048BDE859
:10F98000F840FAF7B3BE0C4BC3F8C4400BF0D4FBFD
:10F990002A4621460B48FAF7A9FE182C09D80A4B2B
:10F9A0000C2202FB043393F85808BDE8F8400BF032
:10F9B000F9BB0020F9E700BF780500240B950B0880
:10F9C0001F950B0835950B08889A0A0838B5044628
:10F9D000114D0846FEF75EFD68B1104B93F900101B
:10F9E0004B1C06D10E4B19780E48BDE83840FAF78B
:10F9F0007DBEC9B2F8E70846F9F7CAFB032804D868
:10FA0000C0B2FAF7D5FA2946E3E7204603220649B1
:10FA1000BDE83840FCF736BFA1930B0878050024F9
:10FA2000483700244E950B085E950B080329F0B566
:10FA3000054685B00C46164614D80B4F3970FAF7B8
:10FA40003DFE0A492846FFF7C1FF2246084901A8A2
:10FA5000F9F7BAF901AB324608212846FCF792FEC5
:10FA6000FF233B7005B0F0BD78050024A1930B087F
:10FA70004E950B0838B50446114D0846FEF70AFDB1
:10FA800068B1104B93F901104B1C06D10E4B5978FD
:10FA90000E48BDE83840FAF729BEC9B2F8E7084673
:10FAA000F9F776FB032804D8C0B211F0AFFF29465E
:10FAB000E3E7204603220649BDE83840FCF7E2BEF2
:10FAC000A1930B0878050024483700244A950B08B9
:10FAD00059950B080329F0B5054685B00C46164626
:10FAE00014D80B4F7970FAF7E9FD0A492846FFF759
:10FAF000C1FF224608496846F9F766F96B46324667
:10FB000010212846FCF73EFEFF237B7005B0F0BDB8
:10FB100078050024A1930B084A950B08444B2DE966
:10FB2000F74FDFF8289105461A785B78009189F83D
:10FB30000130404B89F800201B790BB905F0EAFB36
:10FB400000263D4C42F07CFAB0460D233A4A00991B
:10FB5000734352F803A05046F9F752FA002841D0F7
:10FB6000B8F1000F01DDFAF7A9FD51463348FBF764
:10FB700069FF002221462846FCF776FEFAF79EFD33
:10FB8000237903F01803082B45D0102B48D02046CA
:10FB9000FBF765FF0D22284B02FB0633B3F8090083
:10FBA00042F014FA8346D8B12046F8F797FA074690
:10FBB000DBE90221024401442046F8F727FA78B92C
:10FBC000514601901E48FBF73DFFDBF80810019AF3
:10FBD00028461346CA192146FCF7EAFCFAF76EFDDF
:10FBE00008F10108013640F281230D349E42ACD168
:10FBF0000020F8F752FAFF2389F8003089F8013025
:10FC0000B8F1000F11D1009A28460E4903B0BDE8A3
:10FC1000F04FFCF737BE0C492846FFF7D7FEB6E792
:10FC200009492846FFF726FFB1E703B0BDE8F08F8A
:10FC3000483700248862002408AB0A0881880B0832
:10FC400079950B084B890B08A1930B0878050024C4
:10FC50002DE9F74F804608460F4654F007F8044652
:10FC600020B1012824D13B782A2B21D1A94E00258F
:10FC70004FF00D0AA84FB14604F00104A748FAF767
:10FC80008DFD0AFB05F33846013559F80310FBF7E3
:10FC9000D9FE314622464046FCF7E6FD0D36FAF71E
:10FCA0000DFD40F281239D42EBD103B0BDE8F08F02
:10FCB0003D21384657F0BDF8002800F02481034666
:10FCC0009A4613F8012D202AFAD0AAEB070A013030
:10FCD000054610F8013B202BFAD05FFA8AFA4FF064
:10FCE0000009DFF830B20D235246384603FB09F312
:10FCF0005BF803100BEB03040091F9F75DF906467E
:10FD000070BB0099084653F0B1FF824528D127798E
:10FD100007F0E001402900F08A8012D871B36679BB
:10FD20007F4A002702EBC606BA463B4696F8BC243B
:10FD30000092009ABA4202D9BAF1000F63D02BB1F7
:10FD40002DE06029ECD0802900F0A580404675495F
:10FD5000FCF798FD204603B0BDE8F04FFBF77FBEEF
:10FD600009F1010940F281239945BCD13A466E4917
:10FD7000404603B0BDE8F04FFCF784BD07F0070331
:10FD8000042B1CD10B460A222846F9F751F9D4F866
:10FD9000053001468342D9D32046F8F7A9FA0D234E
:10FDA000624803FB09F95BF80910FBF74BFE0022E0
:10FDB0002146404603B0BDE8F04FFCF755BD052B8A
:10FDC0000DD101230A222846F9F732F9D4F805307B
:10FDD00001468342BADB5B428342B7DCDCE728465C
:10FDE000F9F7D6F917F0050F014607D1B4F8052049
:10FDF000B4F807309142A9DB9942EEE7B4F9052047
:10FE0000B4F90730F6E7D6F8B81451F8270060B116
:10FE100029460193F7F782FF019B30B94FF0010AA1
:10FE200039462046F8F764FA5346013781E707F070
:10FE300007076379013F0093009BB342AFDDAA46F9
:10FE400015F8013B202BFAD02046F8F73DFA05467D
:10FE5000042F04D8DFE807F0030E0E141D005046EF
:10FE6000F9F796F9A8552C21504656F0E2FF0136D5
:10FE7000451CE1E75046F9F78BF925F81600F2E743
:10FE800000230A2200215046F9F7D2F845F826004F
:10FE9000E9E70123F5E7284653F0E8FEE379064653
:10FEA00094F805A0DB07A7790AD52046F8F70CFAE5
:10FEB0000378014623B13246284657F093F8E0B95B
:10FEC000DEB1B74219D32046F8F7FEF93A460021D1
:10FED00056F098FFB2453FF662AF324614492846C5
:10FEE00057F080F800283FF45AAF2046F8F7ECF9B5
:10FEF0003246294656F028FF51E73A460D4940461A
:10FF0000FCF7C0FC22E73946404603B0BDE8F04F9D
:10FF100004E600BF08AB0A0881880B0889950B0826
:10FF2000889A0A08D7950B084B890B08CC950B08C3
:10FF3000089A0B089C950B0870B504460E460846B7
:10FF400053F094FE3146054602462046F9F734F850
:10FF500068B9635D1846F9F713F800B933B901358C
:10FF60002C44204601340378202BFAD070BD0020A9
:10FF7000FCE708B504460948FAF798FBFAF77AFB5C
:10FF8000074BD3F87C020BF067F805F01BFF012C40
:10FF900001D14CF0E3FBF4F74FFC00BFE5950B08F3
:10FFA0008073002410B5044608460B46FEF772FA2B
:10FFB00028B9032208491846F8F7FEFF28B9074870
:10FFC000FAF748FC0120FFF7D4FF20460449BDE8BA
:10FFD0001040FCF757BC00BFF1950B08F5950B08D6
:10FFE000B48E0B082DE9F74F4FF0000B064601AA1F
:10FFF00008462D495D4656F0E2FE01270446DFF82B
:020000040805ED
:10000000B880DFF8B890DFF8A0A014BBBBF1000FF8
:1000100027D1264C002D43D029462548FAF766FB08
:1000200023790BB905F076F942F00AF8002384F839
:100030005130FAF7F5FA15B12846F8F72EF89FB1C6
:100040003046FDF747FD78B1FAF740F90020FFF799
:1000500090FFBBF1000F0AD02046F9F799F885B25E
:10006000C5B93046FCF724FC03B0BDE8F08F41462B
:100070002046F8F7C5FF80B949462046F8F7C0FF8B
:100080000028EED05F4601AA5146002056F097FEA8
:100090000446BAE74FF0000BF5E74FF0010BF2E72B
:1000A0000448FAF7D7FBBFE777890B08886200247A
:1000B00020960B0843960B0817960B08FF960B0823
:1000C00010B50C46FDF706FD78B1084B01229A7376
:1000D000FAF7FCF80648FAF7BDFB06492046F7F7A1
:1000E0001DFE10B10020FFF744FF10BD483700246B
:1000F00059960B08477F0B082DE9F04F0E4693B039
:10010000A049174602903046FFF716FF0546002823
:1001100040F021819C493046FFF70EFF054600283C
:1001200040F01B8199493046FFF706FF054600283D
:1001300040F0158196493046FFF7FEFE054600283F
:1001400040F00F8193493046FFF7F6FE0028054640
:100150000ABF0124082435467F428F49284607F00C
:1001600010073C43FFF7E8FE002800F0FC8044F055
:1001700020048A4B1B790BB905F0CCF841F060FFE5
:1001800014F0090F00F04C838548FAF763FB002058
:10019000FCF726F814F48073059340F0EE80814854
:1001A000FAF758FB8048FAF7F9FA04F01803182B0D
:1001B00005D17E48FAF74EFB7D48FAF7EFFA0123A6
:1001C0000493FAF77BFA7B497B48FAF78FFA7B496D
:1001D0007B48FAF78BFA04F48473082B07D179492A
:1001E0000298FAF792FA77490298FDF765F814F049
:1001F000800307930ED1744B204693F8382503F5FE
:10020000A763002A714A06BF012113460021704AE4
:10021000FAF758FA6F492046FBF78EFB6E492046E5
:10022000FAF738FC6D492046FAF72DFB6C4B14F0B9
:100230001006D3F800A06B4B1D6840F0A0806A4800
:10024000FAF708FB0396694B4FF0000899460693AE
:100250006AEA0503099359F804BBBBF1000F21D0EA
:100260000127099B039A204607FA08F73B400CBF79
:10027000012100210893FAF7F9FA65EA0A035C4ABA
:10028000039020463B425B4614BF01210021FAF750
:10029000A1FC08995B46564A0039204618BF012147
:1002A000FAF710FA08F10108B8F11D0FD3D165EA89
:1002B0000A034FF00008DFF850910893069B53F8AB
:1002C00004BB0693BBF1000F24D0012707FA08F7FF
:1002D0003D420AD06AEA05034A4620463B425B4655
:1002E00014BF01210021FAF775FC1AEA070F11D09B
:1002F000089B2046039A1F400CBF01210021FAF7FA
:10030000B5FA391E03905B464A4618BF01212046C4
:10031000FAF7D8F908F10108B8F11D0FCED12A4D2E
:100320002046344B344A05F5B461FAF7E3FC079BE9
:10033000002B6BD0134B224618210298FCF722FAAF
:10034000049B002B00F0D2812C48FAF783FA2C484A
:10035000FAF724FACAE10124FEE60224FCE60424AA
:10036000FAE68124F8E627492846FFF7E5FD00284C
:100370003FF4FFAE44F48074FBE6002320E71A4B01
:10038000039360E77F960B0886960B088E960B0802
:1003900094960B08A9910B083A960B0888620024E2
:1003A000A2960B08AA960B08C2960B08CE960B08CD
:1003B000F6960B08EB850B08B68B0B08F8850B0837
:1003C000D48B0B08A1930B0880730024089A0B08A8
:1003D00006970B0813970B081D970B08CE820B0886
:1003E000404100244C3E002460960B082CA20A08D1
:1003F00023970B083A970B0860670024FE970B08B9
:1004000014980B089D960B082F970B08DFF8B8A3DC
:100410002046DFF8B8B39AF800209BF80030BB4FB5
:100420009A42BB4A13BF012100214FF001094FF04E
:100430000009FAF71BFA9BF800308046B54A07EB33
:10044000830349462046D3F83437FAF7C3FB9AF8BA
:1004500000304946AF4A07EB83072046D7F83437C8
:10046000AD4FFAF72FF9AD4A2046D7ED007AF5EEF9
:10047000407AF1EE10FA0CBF01210021FAF722F9BF
:1004800043463A46A6492046FAF71AFDA54B05F51C
:10049000FC7205F21C612046FAF716FF26B195F9A9
:1004A0008A31002B00F028819F48FAF7D3F99F4842
:1004B000FAF774F900239E4A20469E4F02F2F44157
:1004C0009D4DFAF7A7FF9D4B6FF07F4220460193A9
:1004D00000923A682968FBF7D9F940F20222984B5A
:1004E000204600920193BA68A968FBF7CFF9002E65
:1004F00040F004819348FAF7ADF93246924F012556
:1005000092480021DFF8C8C217F8013B10F8018BB0
:1005100003F1480EEE440EF8208C1CF801EB0EF1AE
:100520004809E94409F8108C002D00F0E980A3EB9C
:100530000E056B426B4101311D460829E4D10027AD
:1005400083F0010120468DF83070FAF78FF90EAB79
:100550007F4A294620468DF84070FAF73BFB0AABEC
:100560007B4A29462046FAF7ADF87A4A7A4B20466C
:1005700002F53271FAF780FD784A794B204602F590
:100580003271FAF7C1FD734A764B204602F532719B
:10059000FAF700FE744B754A20467549FAF732FBAC
:1005A000744A754B204602F26C51FAF727FC734AE5
:1005B000734B204602F26C51FAF71CFD714B724AE4
:1005C00020467249FBF700F8714B724A2046724987
:1005D000FAF79CFF002E40F09580B3466F48FAF77B
:1005E00039F96F4D0026DFF8EC81A5F5FD67394636
:1005F0000222284656F05AFD002895F800A05A46D7
:1006000014BF0121002120460CBF4FF001094FF01B
:100610000009FAF72BF9BAF1020F834640F0DC80AB
:100620007B784FF0190A40F2EE22494620461AFB29
:1006300003235C4A01933B7818F803300093334658
:10064000FAF7C8FA6B7840F2EE22494620461AFBC8
:100650000323544A01932B7818F803300093334650
:10066000FAF730F8013602350237122EBFD10021D9
:100670004D4B22460298FCF785F8210740F1C480D3
:100680000025E9B2013522460298FFF7CFF9042D83
:10069000F7D1464F464D3B782B70059B33B9454803
:1006A000FAF7D8F844490298FFF790F9FF2300269B
:1006B0002B70F1B2013622460298FFF70BFA042E96
:1006C000F7D17B786B70059B002B40F09A803B48FC
:1006D000FAF7C0F838490298FFF7CCF93848FAF72A
:1006E000B9F83848F9F7E2FFFF236B70002013B028
:1006F000BDE8F04FF7F7D1BC0B4BDCE6114AFDE645
:100700002B4618E7DFF894B06BE700BF889A0A0819
:100710006E960B0841970B083C3800244A970B084B
:100720007C3F002479890B0868960B0859970B08C1
:1007300008750024A03900246C41002466970B083A
:100740006D970B0874960B0828420024801C0B0838
:1007500020890B08A4770024728C0B0824780024CD
:1007600079970B0874970B087F970B08A0680024F3
:100770005C7B00246876002483970B089477002420
:100780008C970B0894970B0844690024107D002473
:100790009D970B08303A00244C40002478960B08B3
:1007A0002C7E00245B920B087F960B086C42002481
:1007B00078050024A1970B08A1930B08C4970B0898
:1007C000EB970B0801970B08144200242C380024E7
:1007D000683700246C1E0B083B7849461A4A2046AD
:1007E00018F8033000933346FAF7F4F92B78164AD9
:1007F000494618F80330204600933346F9F762FF64
:1008000030E7FF236B709BE5104D22460298297854
:10081000FFF70CF9224669780298FFF75BF98FE53C
:10082000A20706D5094B224602981978FFF7FEF871
:100830005CE763077FF55AAF044B2246029859786C
:10084000FFF748F952E700BF6B920B086C42002497
:10085000224BB0F5FA6F1A680346A8BF4FF4FA634B
:10086000B3F57A7FB8BF4FF47A73D20416D540F24D
:10087000DC52904215D040F2DB5207EE903A9042A3
:10088000F8EE677A1FD8DFED166A9FED167A77EEDD
:10089000E67A9FED150AA7EE870A7047B0F57A7FD2
:1008A00002D89FED120A704707EE903ADFED106A0A
:1008B0009FED107AF8EE677A9FED0F0A77EEE67AF1
:1008C000A7EE870A7047DFED0D6A9FED0D7A77EE90
:1008D000E67A9FED0C0AA7EE870A7047643700247A
:1008E00000007A44D62000C000E0824400000000EE
:1008F00000407A44661000400000404200A0BB4423
:10090000D620004000008344704700BF704700BFFE
:100910000020704701207047704700BF704700BF3C
:10092000704700BF704700BF9FED010A704700BFCE
:100930000000000000207047064B1B78834206D958
:1009400000EB4000044B03EBC003586970470020E4
:10095000704700BF000600203C05002000EB40006F
:10096000024B03EBC003587C704700BF3C050020DE
:10097000024B1878003818BF01207047000600208D
:1009800003681B6903B11847704700BF2DE9F04F9A
:10099000DFF878B00F4601F109080124BBF80030F8
:1009A00004339DB217F8011BAC464FF0000E04FA59
:1009B0000EF2ACF104030A409BB21BD103F1010A11
:1009C00000EB83091FFA8AF3C9F814209C45F5D17E
:1009D0000EF1010E0CF1040CBEF1080F1FFA8CFC95
:1009E000E5D120354745ADB2DCD10023ABF800306E
:1009F000BDE8F08F868903F1010900EB83021FFA3D
:100A000089F356616345F6D1E2E700BFB084002464
:100A10002DE9F047DFF87CA0884601F106090024A3
:100A2000BAF8023001260B331FFA83FE18F801CB07
:100A300071460025A1F10B039BB23DB1092D20D0D9
:100A40006A1E06FA02F212EA0C0F1AD0878900EB2E
:100A5000830201339BB257619942F8D10B1D0135D6
:100A60000C3100EB83030A2D89B25C60E2D10EF1F8
:100A7000780EC8451FFA8EFED8D1AAF80240BDE80C
:100A8000F0871A1D01339BB200EB82028B42546047
:100A9000F7D1E3E7B08400242DE9F8430E7804464B
:100AA000057B00F11003F64300F13802F6B243F87B
:100AB000045F9342FBD12822002104F13C0005276A
:100AC00056F0A0F94FF000084FF0140E46FA07F266
:100AD000734602F00102002A42440CBF4FF00A099B
:100AE0004FF0190917F0010F5FFA82F80EEB090CAD
:100AF00014BF284600201FFA8CFC591C04EB83020B
:100B00008BB250616345F8D1013FF1447B1C1FFA61
:100B100089FEDBD118F0010F734614BF19200A209B
:100B20000EEB0006B6B2591C04EB83028BB2556182
:100B3000B342F8D1421E0EF101030EF10200074943
:100B400092B2134402449BB292B204338A800021D1
:100B500004EB830359602261BDE8F883B08400246C
:100B600070B5094CA36873B10546002606E0996884
:100B70001A681E73A1609047A36823B15A6818468B
:100B8000AA1A002AF3DA70BDB084002470B5214C93
:100B90002378012B00D070BD1F4B1B68002BFAD0AF
:100BA0001E4D2B6828465B6898470028F3D01C4BE5
:100BB0001C4E1A68338892889A4219D31A49002227
:100BC000284609684968EA622A6803FB01F1D3688C
:100BD00098473388154A013352683380002ADAD0A7
:100BE000116893884A69134218BF1B048B6170BD5A
:100BF0000E4A00210E4B52681B782170002ACAD081
:100C0000C3F34003918812681B0101FA03F3936157
:100C100070BD00BF663200246424002468240024D0
:100C200060320024643200245C320024A0240024BA
:100C3000AC2400240022FFF75FBA0122FFF75CBA60
:100C40002DE9F84F002607460C461D4DB046DFF84B
:100C50007890DFF878A02046FDF71CFCD5F800B0AE
:100C600048B921465846F8F7CBF920B921466868BB
:100C7000F8F7C6F980B15846F9F718FD696811B15F
:100C80005046FAF7DFFEA96811B14846FAF7DAFED6
:100C90004FF00108F9F712FD013610353A2EDAD17E
:100CA0002046FDF7F7FB48B9B8F1000F06D1224600
:100CB00038460449BDE8F84FFBF7E4BDBDE8F88FBE
:100CC00098CB0A0858980B0852980B084C980B08B8
:100CD000F8B5354C2368002B53D00A2801D00D28D5
:100CE0004DD1324D2B7B0BB1F9F7E8FC304E23216F
:100CF000304656F09EF808B1801B20602368002221
:100D00006BB902B12360F9F7A5FC2B7BEBB1294845
:100D1000BDE8F840F9F7CABC01220B46F0E7591EBE
:100D2000705C2028F8D08AB90022234C204FF2545E
:100D30003B26013E0CD13146204B9C4211D2E36848
:100D4000206898476B7B002BDDD1F8BD2360EBE773
:100D500021683846FFF7F0F801460028ECD110343E
:100D6000E7E72B7B23B116491648FBF707FCCAE7D8
:100D70001548F9F79BFC0E48F9F710FDC3E7FF2B68
:100D8000E3D8A0F120025E2ADFD80BB92028DCD0FE
:100D90005A1C2260064AD054044B1B7B002BD4D033
:100DA000BDE8F840F9F70CBF946B0024B084002430
:100DB000926A0024427F0B0898CB0A0838CF0A08B1
:100DC0006C980B0888980B088E980B0808B5294B6F
:100DD0001B68DB041ED5B5EE400AF1EE10FA26D0F2
:100DE000DFED257AB4EEE70AF1EE10FA1FD49FED9D
:100DF000237AB4EEC70AF1EE10FA2AD870EE677AB9
:100E00009FED1F7A9FED1F0AA7EE870A54F064FF3B
:100E100080B208BDDFED187AB4EEE70AF1EE10FA01
:100E20000BDA9FED190A54F057FF80B208BD9FED11
:100E3000170A54F051FF80B208BD70EE677A9FED3B
:100E4000147A9FED140AA7EE870A54F045FF80B28A
:100E500008BDDFED117ADFED116A70EE677A9FED64
:100E6000107AA7EEA67AB0EE470A54F035FF80B2AA
:100E700008BD00BF643700240000404200E0824407
:100E800066BEFFBE0060BB4400007A440080BB44E5
:100E900038DFFF3E00407A440000834466BEFF3ED8
:100EA00000A0BB442DE9F843D14B1B6813F00405A7
:100EB0002DED048B40F0EC809FEDCE8ACE4C13F0EC
:100EC000200305D094F8DC3013F0020340F0A58035
:100ED00094F815212E46DFEDC98A12F0010294F82C
:100EE000141140F0B080002940F09280D4ED467A91
:100EF0009FEDC36ADFEDC36A67EE867A94ED487AA8
:100F000038EE477AE8EE267A84ED477AC4ED467AE1
:100F100063B1012194F82821D4F8E0308A4284F8A2
:100F20001611C4F8243118BFC4F81C31B64B1F7811
:100F30000D2F0BD1D4ED387A9FEDB47AB44B67EE18
:100F4000877AFDEEE77A17EE902A9A80B0EE489AFB
:100F500000259FEDA87ADFF8C882D4ED4D7AD4ED54
:100F60004E6A37EE677A94ED4C8AE6EE877A37EE72
:100F7000C87AC4ED4D7AA6EE878A84ED4C8A88ED56
:100F8000008A0DB184ED478AD4ED517A94ED4F7A01
:100F9000B0EE676ADFED9F5A38EE477AD4ED526AB9
:100FA00094ED500A84ED4F8A97EE256AE6EE867A34
:100FB00037EEC07AC4ED517AA6EE870A84ED500A66
:100FC00084ED530A54F088FE02B282EAE273A3EB86
:100FD000E2739BB2092B40F2FD80002AACBF0A38B5
:100FE0000A3005B20D2FA4F8505100F0DB80242FF9
:100FF00000F0C880382F05D1B0EE480A54F06CFEDE
:10100000834B988084F85261BDEC048BBDE8F88373
:1010100084F8162184F8142168E7D4ED3B7AB4F8FB
:10102000F030F8EEE77AC4ED387A002B74D1DFEDBA
:10103000738A94F81521012694F8141112F0010214
:1010400033463FF450AF00295ED0D4ED489A6E4A43
:1010500038EE699A94F816911778F3B1B9F1010F47
:1010600001D0002D72D1B9F1000F40F0BC800D2FDE
:10107000DFF8AC8100F0D880002D00F0B08094F84B
:101080002831012B94BFB0EE497A98ED007A64E7DD
:10109000594C012594ED348A11E70D2F49D0DFF822
:1010A0008081DFED548AB9F1000FE5D094F8283142
:1010B000002B40F0918098ED007A002D00F0918097
:1010C00077EE487A94F829319FED536A06EE903A0C
:1010D00077EEA97AF8EEE66AF0EEE77A67EEA67A9E
:1010E000F4EEC67AF1EE10FA03DD28EE866AC6EE5B
:1010F000278AF7EE007A77EEE87A67EE897AE8EEEB
:10110000877AB0EE677A28E7D4ED469A0122C4EDDB
:10111000489A84F814219AE707EE903ADFED3D6A89
:101120009FED3E7AF8EEE77AC6EEA78AC8FEC78A38
:101130007FE7DFF8EC80DFED3B7A98ED000A20EEE8
:10114000270A54F0C9FD324B9880AAE794ED380A7B
:10115000012370EE487A84F8163177EEA97AC4ED4F
:10116000497A30EE670ADFF8B8800D2F88ED000A63
:101170009CD1DFED2C7A20EE270A54F0ADFD244BF4
:10118000988093E7DFED277A94ED470A20EE270A4F
:1011900054F0A2FD1E4B84F852615880BDEC048BC4
:1011A000BDE8F883DFED1B7A9FED1E0A68EEA77A93
:1011B000174F29EE000AFDEEE77A17EE903A3B80D2
:1011C00054F08AFDFD80788084F85261BDEC048B78
:1011D000BDE8F883002505E7022B7FF44DAF98EDBD
:1011E000007A0125B9E694ED380AD4ED497AB8E7DA
:1011F000A46B002400000000B08400249A99993E5A
:10120000CDCC4C3FCDCC4C3E172900240AD7233CF3
:10121000182900240000C84200401C466666663F4C
:10122000643F0024CDCCCC3D5FED027A98ED000AFE
:1012300020EE270A54F050FD014B98801CE700BFB8
:10124000182900244E4B1B681B0600D470472DE95B
:10125000F0414C4CD4F860312DED048B84B013B1C7
:1012600004F5AA7098470023D4F8642169464648DB
:10127000CDE90033CDE902339047009BD4F87C21BF
:10128000BDF904609D1AA4F8686104D104B0BDECF6
:10129000048BBDE8F08194F88421F7EE007A9DED8F
:1012A000039AFFEE006A94ED627A002A374A67EEED
:1012B000498A9DED020A92ED008A47FEA67AB4F8AB
:1012C0008621E0EE088A29EE088AA0EE078A68EEF9
:1012D000A78A1AB394ED647AD4ED677A38EEC75AC8
:1012E00094ED656A78EE675AD4ED686AD4ED638A46
:1012F000A6EE057A94ED668AE6EEA57A37EE685A90
:1013000084ED647A77EEC85AC4ED677AE6EE058A12
:10131000A6EEA58AC4ED638A84ED668A1C4A84ED34
:101320005B0A127884ED5C9A1C2AC4ED5D8A84ED18
:101330005E8AC4F87C31A9D1DFED169A164C20EEF6
:10134000290A54F0C9FC29EE290A074654F0C4FCC6
:1013500028EEA90A804654F0BFFC002328EE290A93
:101360001A4666F30F0368F30F0267F31F4360F337
:101370001F42C4E9003254F0AFFC6581208185E74B
:10138000A46B0024B08400240486002440060024BA
:101390001729002400007A44182900242DE9F84375
:1013A000A84C2DED048BA36820469847002800F038
:1013B000BB80B4F90E30A17D06EE903AB4F910303E
:1013C000092907EE103AB4F91230F8EEE66A07EE92
:1013D000903AB8EEC77AF8EEE77AC4ED126A84ED77
:1013E000137AC4ED147A00F0A380974E04F14800FC
:1013F00029F03CFCB28DB36A002A40F0A580934AE4
:10140000934D1268520700F1E880B3F90020D4ED43
:10141000147A06EE102AB3F90220B3F9043006EE6E
:10142000902AB8EEC66A07EE103A8A4BF8EEE66AE2
:1014300094ED128AB8EEC77A93F86E75864B38EE43
:10144000468AD4ED138A93F8008037EEC79AB4F831
:10145000443078EEE68A84ED128A07EE903A3388BB
:10146000C4ED138AF8EEE79A84ED149A002B40F04D
:10147000FF80B8F1040F00F0D881D5ED747AD5ED76
:10148000756A95ED767A78EEE66A85ED748A39EEBE
:10149000477AC5ED758A38EE678A85ED769A66EEED
:1014A000A96A27EE297A28EE298AC4ED166A84ED06
:1014B000177A84ED158A94ED137AB8F1040FD4ED00
:1014C000167A27EE077AD4ED124A67EEA77A94EDE2
:1014D000155AD4ED145AA4EEA47A94ED176AE5EEE9
:1014E000057AD4ED006AA5EEA57AE6EE067AB1EEAD
:1014F000C70AB1EEE77A26EE800A84ED180A26EED6
:10150000878A84ED198A0CD1DFED548A544D20EE80
:10151000280A54F0E1FB28EE280AA88054F0DCFBEE
:101520002881012384F86830BDEC048BBDE8F88382
:10153000454E04F1200104F1480029F02FFBB28D43
:10154000B36A002A3FF45BAFB2F5C87F00F0518167
:101550003F4D4FF0000E94ED127A4FF0000CD5ED98
:10156000696A012AD4ED137AF8EEE66A94ED146AFA
:10157000C4F848E0A3F800C076EE876A95ED6A7A71
:10158000C4F84CE0B8EEC77AA3F802C0FDEEE66AF4
:10159000C4F850E0A3F804C037EE277AD5ED6B7A93
:1015A00016EE907AC5ED696AF8EEE77ABDEEC77A75
:1015B00077EE867A17EE100A85ED6A7AFDEEE77A05
:1015C00017EE901AC5ED6B7A00F01682013AB285DB
:1015D0001E4A126852077FF518AFB5F8B071322F66
:1015E00000F0C180002F40F0828195F8CE21002AC2
:1015F0003FF40BAF05F5E070DFF86CC0B4F80CE019
:10160000002707C88CFB0298D21785F8CE71C2EB71
:101610002812A2EB0E029A808CFB00E2C017C0EBEE
:1016200022108CFB012CC91701221880C1EB2C1150
:1016300059800C4BDF81C3F80A20F8F79FFEB36A8C
:10164000E3E600BF783500205C23002064370024E7
:10165000B0840024CC1D00201729002400007A4407
:1016600018290024846800241F85EB510AD7233CE5
:10167000002F00F0B380D6ED027AD6ED036A38EE83
:10168000678A96ED010A95ED747AE8EE267A37EED0
:10169000C06AC6ED027AA6EE260A30EE478A86EDCB
:1016A000010A84ED120A85ED740A28EE298A84ED78
:1016B000158A002F7FD0012F00F07981D6ED057AB1
:1016C000012F96ED067A78EEE78A96ED040A95EDFD
:1016D000758AE8EE877A77EEC06AC6ED057AA6EEDF
:1016E000870A30EE488A86ED040A84ED130A85EDF8
:1016F000750A28EE298A84ED168A00F03A81022FB5
:1017000000F04A8196ED087A022FD6ED096A79EE4B
:10171000477A96ED070A95ED768AA6EEA77A77EED8
:10172000407A86ED087AA6EEA70A30EE488A86ED62
:10173000070A84ED140A85ED760A28EE298A84EDDD
:10174000178A7FF4B8AEB8F1040F7FF4B4AE54F04A
:10175000C3FA1FED3A0ABB4D28EE000A688054F028
:10176000BBFAE880A7E6B84A0021D4ED126AD26835
:1017700094ED137AFDEEE66AC5F8BC211A68BDEE59
:10178000C77AD4ED147AC5F8B4219A88FDEEE77AC9
:10179000A164A5F8B8210022C5ED706A1A8085ED14
:1017A000717AE164C5ED727A5A8021659A80013FB1
:1017B000A5F8B07119E7B8F1040F7FF47FAF54F0CA
:1017C0008BFA9FEDA20ADFF87C9228EE000AA9F8B6
:1017D000020054F081FAA9F806006FE7B8F1040F8F
:1017E0007FF449AFB0EE480A54F076FA954B188072
:1017F00041E7D4ED126A002094ED137A0021D4ED74
:10180000147AFDEEE66ABDEEC77A914DFDEEE77AF9
:10181000A064C5ED696A198085ED6A7AE064C5ED5A
:101820006B7A598020659980D0E697B3D5ED747AAC
:10183000012F85ED748A38EE678A28EE298A84EDB7
:10184000158A00F0BF80D5ED757A022FC5ED758A37
:1018500078EEE77A67EEA97AC4ED167A3CD1B0EE5D
:10186000490A784E54F038FAD5ED767A9FED770A2A
:1018700000B279EE677A85ED769A3080708067EEF7
:10188000A97A27EE800AC4ED177A54F025FAF08081
:1018900011E6B0EE480A6B4E54F01EFAD5ED747A9C
:1018A0009FED6A0A00B278EE677A85ED748A30801F
:1018B000708067EEA97A27EE800AC4ED157A54F09D
:1018C0000BFAD5ED757AF08078EEE77AC5ED758A7A
:1018D00067EEA97AC4ED167AD5ED767A85ED769A1B
:1018E00079EE677A67EEA97AC4ED177AE3E5D5ED6C
:1018F000706A002194ED127A0022F8EEE66AD4EDC7
:10190000137A94ED146A012FA16476EE876A95ED3F
:10191000717A1A80B8EEC77AE164FDEEE66A5A8001
:10192000216537EE277AD5ED727AC5ED706AF8EE4B
:10193000E77A9A80BDEEC77A77EE867A85ED717A7E
:10194000FDEEE77AC5ED727A7FF431AF0B2085F8B2
:10195000CC2185F8CD7109F025FCB36AD5F8B42106
